:100000000C9403210C9434210C9434210C9434214D
:100010000C9434210C9434210C9434210C9434210C
:100020000C9434210C9434210C9434210C943421FC
:100030000C9434210D94D33A0C9434210C94342133
:100040000C9434210C9422D80C9434210C94342137
:100050000C9434210C9434210C94E9D40D94893AF5
:100060000C9434210C94314A0C94274A0C9434217A
:100070000C9434210C9434210C9434210C943421AC
:100080000C9434210C9434210C9434210C9434219C
:100090000C9434210C9434210C9434210C9434218C
:1000A0000C9434210C9434210C9434210C9434217C
:1000B0000C9434210C9434210C9434210C9434216C
:1000C0000C9434210C9434210C9434210C9434215C
:1000D0000C9434210C9434210C9434210C9434214C
:1000E0000C943421084AD73B3BCE016E84BCBFFD43
:1000F000C12F3D6C74319ABD56833DDA3D00C77FF8
:1001000011BED9E4BB4C3E916BAAAABE0000008090
:100110003F05A84CCDB2D44EB93836A9020C50B91F
:10012000918688083CA6AAAA2ABE000000803F004B
:100130000D941C340D940B340C94DE210C94268108
:100140000D94AC340C94BF4A0C94B7AF0D94F734B3
:100150000D9468330C9447810C945CC90D946C33F6
:100160000C94B0AE0C94FC770C9446780D948F33BD
:100170000C94C0AE0C9480AE0C941F7A0C94BA7F91
:100180000C94AE7F0C949E7F0C9436210C94747862
:100190000C9476C70C9460A70C94CA770C94D5C7BE
:1001A0000D947E340C94FB790C94A14A0D949D33EC
:1001B0000C9435770C946DC20C94694A0D945133AC
:1001C0000C944B960D94C0340C945F750D94703361
:1001D0000C94687D0C94E3910C941F880C9497BB4D
:1001E0000C945D780C940BB20C94F0830C94907981
:1001F0000C94C74A0C948B790C94F7840C9455801A
:100200000C94B47A0C94577B0C941B7A0C94E4BA3B
:100210000C94F67A0D94B6340C9483770C94537B3B
:100220000D9492340C9498AE0C94FD840D94D233BA
:100230000C94769F0C94C0C60C94CD7B0D94103416
:100240000D94C9460C946D800C9448A10D942C34E7
:100250000D946A130C946EAE0C94DDC60C949E77CC
:100260000C9400850C9484790C9498B20D9481338D
:100270000C9406B20C94EC790C94B67F0C94FF8A23
:100280000C94E0840C94BAC70C9486AE0C949181C3
:100290000C94EC800D9422340C9481850C94D87DC0
:1002A0000D94ED340C94B7770D94A7330C94988289
:1002B0000D9456330C9437780C9463850C94E99D17
:1002C0000D94B7330D9401350D94A3330C949579A7
:1002D0000C94E1930C94F1B50C94BB4A0C94467BBE
:1002E0000C94F4890C949EAE0C9437BB0C94D64AB3
:1002F0000C94E8830C94B6BB0C94FE790D948B336C
:100300000C947A810C9456BB0C9410810C94A27FAF
:100310000C94B6AE0D9458460C9470770C943D9C9A
:100320000C94A1800D94D9340C945D7B0C94867947
:100330000C9474AE0C9465C80C94B74A0C94C27FAC
:100340000C94BE7F0C94F1840C9465800C945B7BC0
:100350000D9488340C9478750C941C770C94D78188
:100360000C9420750C9492AE0C9480970D94E33409
:100370000C94167A0C94557B0C9439210C944022E1
:100380000C94F4840C94EE840C9423B20C9420907E
:100390000D94CA340C94FA840C940D850C946685E3
:1003A0000C945A790D949C340C9413790C94CB4A88
:1003B0000C94C34A0D9474330C9446360C94679A8B
:1003C0000C946F790C944F7B0C94A4AE0C94607DCC
:1003D0000D9487330C94BA800C9447A40C94A67F98
:1003E0000C947E750C9405850C94E94A0C94058157
:1003F0000C9415750C94057B0C94B04A0D94A434A0
:100400000C9419980C94E2830C94E1960D94993312
:100410000C948CAE0C9492C80C94647D0C94AA7FBE
:100420000C94D2B20C94B27F0C94AAAE0C94127DB0
:100430000C94CF4A0C946EC20C94C1C30C94B52199
:100440000C940A850C94F9830D94AB460C94DF9DB3
:100450000D9479340C94017A0C94067D0C946B9570
:100460000C9455C70D941B130C9453C80C947E8D9B
:100470000C9401B20C94D3800C94E14A0D94713425
:100480000C94E3770C94628C0C941E780C94048486
:100490000C947AAE0C94F6980C94E3310C94672289
:1004A0000C948C750D9495330C94597B0C94D279E3
:1004B0000C94B5AB0C945D770C94C5BA0C94EB849A
:1004C0000C94FCB10C9441C60C940B780D94481319
:1004D0000C9463790C943C210D9437340C942FA622
:1004E0000C9407850C94EBC10D9477330C948B78A6
:1004F0000D947D330C94E0BB0C949A790C944E7758
:100500000C9482790C94F2740C94047A0D940B354B
:100510000C94924A0C94517B4E414E494E49545989
:10052000494E46CDCCCC3D0AD7233C17B7D13877BE
:10053000CC2B329595E6241FB14F0A0000204100D4
:1005400000C84200401C4620BCBE4CCA1B0E5AAE1E
:10055000C59D7400407A10F35A00A0724E1809002D
:1005600010A5D4E80000E87648170000E40B540218
:100570000000CA9A3B000000E1F505000080969853
:1005800000000040420F000000A0860100000010A3
:100590002700000000E803000000006400000000E5
:1005A000000A00000000000100000000002C76D8C6
:1005B00088DC674F0823DFC1DFAE59E1B1B796E5AC
:1005C000E3E453C63AE651997696E8E6C28426EB10
:1005D000898C9B62ED407C6FFCEFBC9C9F40F2BA23
:1005E000A56FA5F490055A2AF75C936B6CF9676DBB
:1005F000C11BFCE0E40D47FEF520E6B500D0ED9010
:100600002E0300943577050080841E080000204EDC
:100610000A000000C80C333333330F986E12831175
:1006200041EF8D2114893BE65516CFFEE6DB18D14C
:10063000844B381BF77C1D901DA4BBE4242032841E
:10064000725E228100C9F124ECA1E53D27434F4DA4
:100650004D554E49434154494F4E0044525952550D
:100660004E004552524F525300494E464F004543AB
:10067000484F004572726F722077726974696E67B5
:1006800020746F20454550524F4D210A0053544F5E
:10069000505045442E20005072696E74657220736C
:1006A000746F707065642064756520746F20657266
:1006B000726F72732E2046697820746865206572A7
:1006C000726F7220616E6420757365204D393939FF
:1006D00020746F20726573746172742E20285465C3
:1006E0006D706572617475726520697320726573CF
:1006F00065742E2053657420697420616674657278
:100700002072657374617274696E67290A004E6F96
:1007100020436865636B73756D2077697468206C1E
:10072000696E65206E756D6265722C204C61737404
:10073000204C696E653A20004E6F20436865636BFC
:1007400073756D2077697468206C696E65206E75AD
:100750006D6265722C204C617374204C696E653A31
:100760002000636865636B73756D206D69736D61DF
:100770007463682C204C617374204C696E653A2058
:10078000004C696E65204E756D626572206973203C
:100790006E6F74204C617374204C696E65204E75C9
:1007A0006D6265722B312C204C617374204C696E24
:1007B000653A20004D3131300053657269616C201B
:1007C000737461747573206D69736D617463680A05
:1007D00000776169740A0053442072656164206582
:1007E00072726F720A00486F74656E642049646C9F
:1007F000652054696D656F757400486F74656E642B
:100800002049646C652054696D656F75740A002118
:1008100021204B494C4C20636175736564206279DB
:10082000204B494C4C20627574746F6E2F70696E4A
:100830000A002121204B494C4C206361757365648B
:1008400020627920746F6F206D75636820696E6116
:1008500063746976652074696D65202D20637572F7
:1008600072656E7420636F6D6D616E643A20004D29
:10087000656469612052656D6F766564004D6564DD
:10088000696120496E736572746564004D31303062
:10089000305300627573793A207061757365642016
:1008A000666F7220696E7075740A00627573793AAA
:1008B0002070617573656420666F72207573657250
:1008C0000A00627573793A2070726F636573736999
:1008D0006E670A00506C65617365205265736574BC
:1008E000005052494E5445522048414C5445440012
:1008F00025533A20255300706F7765726F66660046
:100900004B494C4C45442E20005072696E74657200
:100910002068616C7465642E206B696C6C282920DA
:1009200063616C6C6564210A006563686F3A004519
:1009300072726F723A000A4D656173757265642058
:10094000706F696E74733A0A00357835206D65737F
:10095000682E205A206F66667365743A20005072C4
:10096000696E74696E67204F626A6563740025530F
:10097000202569002F2F616374696F6E3A007374CC
:1009800061727400656E6400486F74656E642074F3
:100990006F6F20636F6C640A0053656E64204D3185
:1009A000303820746F20726573756D650A00496E6A
:1009B000736572742066696C616D656E7420616E1A
:1009C000642073656E64204D3130380A00526568CA
:1009D00065617420446F6E65005265686561746975
:1009E0006E672E2E2E005265686561740048656141
:1009F0007465722054696D656F75740053656E641B
:100A0000204D31303820746F2068656174206E6F1E
:100A10007A7A6C650A004E6F7A7A6C652050617242
:100A20006B65640070617573656400506175736512
:100A300000726573756D656400526573756D696EDE
:100A400067004732362043616E63656C656400471A
:100A500032362048656174696E67204E6F7A7A6C11
:100A600065004732362048656174696E67204265CB
:100A7000640057616974696E6720666F72206865EB
:100A8000617475702E0A004669786564204C656E45
:100A9000677468205072696D6500446F6E65205000
:100AA00072696D696E67004D616E75616C20707260
:100AB000696D696E672E2E2E004C656176696E67D2
:100AC00020473236003F537065636966696564206C
:100AD000582C5920636F6F7264696E617465206F62
:100AE0007574206F6620626F756E64732E0A003F06
:100AF00028522965706561742076616C7565206E79
:100B00006F7420706C61757369626C653B206D75E4
:100B10007374206265206174206C65617374203188
:100B20002E0A003F537065636966696564206E6FC5
:100B30007A7A6C652074656D706572617475726522
:100B4000206E6F7420706C61757369626C652E0A1B
:100B5000003F5370656369666965642066696C610E
:100B60006D656E742073697A65206E6F7420706C89
:100B700061757369626C652E0A003F537065636925
:100B800066696564207072696D65206C656E677456
:100B900068206E6F7420706C61757369626C652E6D
:100BA0000A003F537065636966696564206E6F7AF9
:100BB0007A6C652073697A65206E6F7420706C6141
:100BC000757369626C652E0A003F526574726163C9
:100BD00074696F6E204D756C7469706C69657220F4
:100BE0006D757374206265207370656369666965ED
:100BF000642E0A003F53706563696669656420521C
:100C0000657472616374696F6E204D756C74697080
:100C10006C696572206E6F7420706C6175736962A7
:100C20006C652E0A003F53706563696669656420D0
:100C30006C6179657220686569676874206E6F748D
:100C400020706C61757369626C652E0A0043292EF1
:100C50000A003F5370656369666965642062656474
:100C60002074656D7065726174757265206E6F7445
:100C700020706C61757369626C65202834302D00BA
:100C8000473236207374617274696E672E2E2E0A95
:100C9000004F46460A0046616465204865696768FA
:100CA000742000426564204C6576656C696E67202F
:100CB000004661696C656420746F20656E61626CCA
:100CC0006520426564204C6576656C696E670A0034
:100CD0004D65736820426564204C6576656C2064C0
:100CE0006174613A0A00496E76616C6964206D65D1
:100CF00073682E0A00206E6F7420656E74657265CD
:100D0000642E0A0050726F62696E6720506F696EC0
:100D1000740025532025692F256900206F66200067
:100D20004D424C2047323920706F696E7420002983
:100D30000A004A206F7574206F662072616E6765C5
:100D40002028302D00290A0049206F7574206F6615
:100D50002072616E67652028302D004732384C3094
:100D6000004D6573682070726F62696E6720646FF2
:100D70006E65004D6573682070726F62696E6720E2
:100D8000646F6E652E0A005374617274206D657312
:100D9000682070726F62696E6720776974682022BC
:100DA000473239205331222066697273742E0A004B
:100DB0004732395332004732384C300A47323953C0
:100DC0003200686173206E6F20646174612E0A00C6
:100DD0004D65736820426564204C6576656C696E6C
:100DE00067200053206F7574206F662072616E67F4
:100DF000652028302D35292E0A004D657368207036
:100E00006F696E74206F7574206F662072616E67F3
:100E1000650A004D34323120696E636F727265630A
:100E20007420706172616D6574657220757361679D
:100E3000650A004F4646004F4E0020204D61783A2B
:100E40002000200020204D696E3A2000536F667408
:100E500020656E6473746F70733A20004D323420D5
:100E600053256C642054256C64004739322E392098
:100E700045257300473120462564004739322E3915
:100E8000205A2573004731205A3020463230300036
:100E90004731205825732059257320463330303090
:100EA000004D34323020532569205A2573004D31CE
:100EB00030362050256920532569004D32303020CE
:100EC0004425730047323852305859004739322E82
:100ED00039204530205A300A47315A2573004D31A8
:100EE000303920532569004D3139302053256900B0
:100EF0004D343230205330205A300020496E766114
:100F00006C6964206578747275646572200047327C
:100F10002F47332062616420706172616D65746572
:100F200072730A00536C6565702E2E2E004D65732A
:100F30006820706F696E74206F7574206F66207200
:100F4000616E67650A004D302053746F70004D313B
:100F50002053746F7000436C69636B20746F205270
:100F60006573756D652E2E2E004E6F204D6F766564
:100F70002E00456E642066696C65206C6973740A86
:100F800000426567696E2066696C65206C697374E0
:100F90000A004E6F206D656469610A0052657375C1
:100FA0006D696E6720534400286E6F2066696C651A
:100FB000290043757272656E742066696C653A200B
:100FC000005072696E742074696D653A20000A538E
:100FD000746174733A2046696C616D656E74207536
:100FE0007365643A20002C204C6F6E676573742023
:100FF0006A6F623A2000546F74616C2074696D6589
:101000003A200053746174733A20002C20466169C1
:101010006C65643A20002C2046696E6973686564CB
:101020003A20005072696E74733A200053746174F0
:10103000733A2000436F6F6C696E672E2E2E004846
:10104000656174696E672E2E2E0045202553006F52
:101050006B006F6666006E06690662065B064D06EB
:1010600044454255473A004D3131332053004265E3
:101070006420436F6F6C696E672E2E2E004265648C
:101080002048656174696E672E2E2E005375506579
:10109000522043522D3230204F46462E002F2F0033
:1010A0004D31343520533C696E6465783E206F7550
:1010B00074206F662072616E67652028302D31299B
:1010C0000A00205200416363656C65726174696F48
:1010D0006E3A2050005741524E494E4721204C6FE6
:1010E00077205A204A65726B206D6179206C6561AA
:1010F0006420746F20756E77616E74656420706112
:10110000757365732E0A004D3230362058004652F2
:101110003A0020466C6F773A20004D424C204164E3
:101120006A757374205A0020643A0020693A0020DE
:10113000703A00496E76616C6964206578747275E6
:101140006465720A0020643A0020693A0020703A0F
:10115000004C434420436F6E74726173743A2000F4
:1011600064697300656E0043290A0061626C6564FE
:1011700020286D696E2074656D702000436F6C646B
:101180002065787472756465732061726520004F04
:10119000666673657473204170706C6965640045A0
:1011A00072723A20546F6F206661722100546F6F23
:1011B000206661722066726F6D2072656665726569
:1011C0006E636520706F696E740A00454550524F1A
:1011D0004D204F4B0A002E0A002028302D31302997
:1011E000002076616C7565206F7574206F662072C3
:1011F000616E676500416476616E6365204B3D00FA
:10120000506F7765722D6C6F7373207265636F76A4
:1012100065727920004D383400446F6E652070721D
:10122000696E74696E672066696C650A004D3737B0
:10123000004D3331004361703A004D4541545041F7
:10124000434B00434F4F4C45525F54454D50455220
:101250004154555245004348414D4245525F544523
:101260004D50455241545552450042414259535404
:10127000455050494E470041524353004D4F544949
:101280004F4E5F4D4F44455300544845524D414CDD
:101290005F50524F54454354494F4E004C4F4E47B8
:1012A0005F46494C454E414D45004155544F5245CE
:1012B000504F52545F53445F53544154555300535D
:1012C000445F5752495445005245504541540053DC
:1012D00044434152440050524F4D50545F53555077
:1012E000504F525400454D455247454E43595F506B
:1012F000415253455200434153455F4C494748547E
:101300005F4252494748544E45535300544F474754
:101310004C455F4C494748545300534F465457413E
:1013200052455F504F574552004255494C445F501B
:10133000455243454E54004C4556454C494E475F37
:1013400044415441005A5F50524F42450052554E5D
:101350004F5554004155544F4C4556454C00505242
:10136000494E545F4A4F420050524F4752455353E3
:10137000004155544F5245504F52545F54454D50C3
:1013800000564F4C554D4554524943004545505227
:101390004F4D0042494E4152595F46494C455F54BA
:1013A00052414E534645520053455249414C5F58B5
:1013B0004F4E5F584F4646004649524D57415245A1
:1013C0005F4E414D453A4D61726C696E20322E3050
:1013D0002E375F4457372E3320544D334420325339
:1013E0004D444E4E2028417072203234203230322B
:1013F000312032303A35383A31322920534F555264
:1014000043455F434F44455F55524C3A687474708E
:10141000733A2F2F6769746875622E636F6D2F4959
:101420006E73616E6974794175746F6D6174696F03
:101430006E2F4D61726C696E2F747265652F4372E9
:1014400065616C6974794477696E5F322E30205023
:10145000524F544F434F4C5F56455253494F4E3AAB
:10146000312E30204D414348494E455F5459504537
:101470003A53755065522043522D3230204558540E
:1014800052554445525F434F554E543A31205555BD
:1014900049443A63656465326132662D34316132A4
:1014A0002D343734382D396231322D63353563367A
:1014B000326633363766660A0043616E6E6F74209B
:1014C0006F70656E207375626469722000256973A0
:1014D0000025696D20256973002569682025696DDF
:1014E0002025697300256964202569682025696DB8
:1014F000202569730025697920256964202569689C
:101500002025696D202569730023646566696E6511
:101510002044454641554C545F00626564004B646D
:1015200020004B6920004B70200050494420417539
:10153000746F74756E652066696E69736865642181
:101540002050757420746865206C617374204B7032
:101550002C204B6920616E64204B6420636F6E7396
:1015600074616E74732066726F6D2062656C6F7744
:1015700020696E746F20436F6E666967757261745F
:10158000696F6E2E680A00504944204175746F746B
:10159000756E65206661696C6564212074696D658E
:1015A0006F75740A00504944204175746F74756EEC
:1015B00065206661696C6564212054656D70657293
:1015C000617475726520746F6F20686967680A00BE
:1015D000204B643A2000204B693A2000204B703A9F
:1015E000200020436C617373696320504944200AD2
:1015F00000204E6F206F76657273686F6F740A00FB
:101600002054753A2000204B753A2000206D6178F7
:101610003A2000206D696E3A200020643A200020B4
:10162000626961733A2000504944204175746F74B7
:10163000756E652073746172740A005049442041CC
:1016400075746F74756E65206661696C65642120C0
:1016500054656D706572617475726520746F6F206A
:10166000686967680A00504944204175746F747551
:101670006E6500504944204175746F74756E652025
:101680006661696C656421204261642068656174EB
:1016900065722069640A004572723A207574663872
:1016A00020666F6E74206E6F7420696E6974696154
:1016B0006C697A65642E004572723A2075746638DA
:1016C00020666F6E74206E6F7420696E6974696134
:1016D0006C697A65642E004572723A2075746638BA
:1016E00020666F6E74206E6F7420696E6974696114
:1016F0006C697A65642E00FFE0FFD140A0C8A6A205
:101700002FF80023AC00AF10FFFEFF05FFD0FFE075
:10171000FFC1FFD1E240A0C8A6A22FF80023812775
:10172000AC00AFFFD0FF64FFD1A5FFD0FF64FF6422
:10173000FFD1A4FFD0FF16FFFE000C0F00FE070232
:101740002503BB017FFE08FE08FE05080806000011
:1017500040F0C88888987810050808060000C0F88E
:101760008888888888F80505050600012030F8304B
:10177000200508080600002070F820202020E00541
:1017800009090600FF2070A8A8B8888870200705FE
:1017900005070001D86C366CD80509090600FFF86A
:1017A000A88888888888A8F8050A0A0600FE2050BC
:1017B00050505088A8A8887003030306000340A077
:1017C00040FFFFFFFFFFFFFFFFFFFFFFFFFFFFFFE8
:1017D000FFFFFFFFFFFFFF0000000605FF010707F7
:1017E00006020080808080800080030303060105DC
:1017F000A0A0A005060606000050F85050F85005BD
:1018000009090600FF2070A8A07028A8702005070D
:1018100007060000C8C81020409898050707060072
:101820000040A0A040A89068010303060205808044
:10183000800309090601FF2040408080804040204D
:101840000309090601FF8040402020204040800518
:10185000070706000020A8702070A82005050506CF
:1018600000012020F820200203030601FFC0408071
:10187000050101060003F8020202060100C0C005CE
:1018800007070600000810102040408005070706E3
:101890000000708898A8C8887003070706010040F8
:1018A000C040404040E0050707060000708808106F
:1018B0002040F8050707060000F808103008887077
:1018C00005070706000010305090F81010050707B4
:1018D000060000F880F00808887005070706000079
:1018E000304080F0888870050707060000F808106F
:1018F000102020200507070600007088887088885F
:1019000070050707060000708888780810600205D7
:1019100005060100C0C000C0C00206060601FFC0E7
:10192000C000C04080030505060101204080402022
:10193000050303060002F800F8030505060101800F
:101940004020408005070706000070881020200016
:10195000200507070600007088B8A8B88070050742
:1019600007060000708888F8888888050707060041
:1019700000F04848704848F00507070600007088E6
:101980008080808870050707060000F048484848B6
:1019900048F0050707060000F88080F08080F80511
:1019A0000707060000F88080F080808005070706A2
:1019B00000007088808098887005070706000088FE
:1019C0008888F8888888030707060100E0404040BF
:1019D0004040E00507070600003810101010906026
:1019E0000507070600008890A0C0A090880507079B
:1019F000060000808080808080F8050707060000D0
:101A000088D8A8888888880507070600008888C8BD
:101A1000A898888805070706000070888888888845
:101A200070050707060000F08888F08080800507B1
:101A30000706000070888888A890680507070600D8
:101A400000F08888F0A090880507070600007088DD
:101A50008070088870050707060000F82020202005
:101A60002020050707060000888888888888700578
:101A70000707060000888888885050200507070659
:101A8000000088888888A8A85005070706000088F5
:101A90008850205088880507070600008888502055
:101AA000202020050707060000F80810204080F8D5
:101AB0000309090601FFE080808080808080E005C6
:101AC000070706000080404020101008030909069F
:101AD00001FFE020202020202020E0050303060055
:101AE000052050880501010600FEF80303030601E6
:101AF00005804020050505060000700878887805F7
:101B000007070600008080F0888888F00505050634
:101B100000007080808870050707060000080878BC
:101B2000888888780505050600007088F0807005B3
:101B30000707060000304840E04040400507070620
:101B400000FE708888887808700507070600008006
:101B500080F0888888880307070601004000C0409D
:101B60004040E00409090601FE100030101010107A
:101B7000906005070706000080808890E090880349
:101B80000707060100C04040404040E0050505064B
:101B90000000D0A8A8A8A8050505060000B0C888C0
:101BA0008888050505060000708888887005070785
:101BB0000600FEF0888888F080800507070600FE92
:101BC00078888888780808050505060000B0C88070
:101BD000808005050506000078807008F00507077D
:101BE0000600002020F8202020180505050600002A
:101BF0008888889868050505060000888888502030
:101C00000505050600008888A8A8500505050600FA
:101C10000088502050880507070600FE88888850F5
:101C2000204080050505060000F8102040F8030953
:101C3000090601FF20404040804040402001090942
:101C40000602FF80808080808080808003090906F2
:101C500001FF8040404020404040800503030600D3
:101C60000248A890FF554E4C4F41442046494C41F4
:101C70004D454E54004C4F41442046494C414D4542
:101C80004E540046494C414D454E54204348414E28
:101C900047450042656400456E636C6F73757265FD
:101CA000002568753A253032687500253032687530
:101CB0003A25303268750020202020202020002086
:101CC000202020001FE020102010201010201020C5
:101CD0002010201030300840048003001FE03FF047
:101CE0003FF03FF01FE01FE03FF03FF03FF00FC03C
:101CF000078003003FFFF038007030FC3020FC10FC
:101D00002078102030102C00D02E31D02F7BD02FF7
:101D10007BD02E31D02C00D020301020781020FC29
:101D20001030FC303800703FFFF03FFFF03800709B
:101D30003186302387102787902F87D02F03D0201C
:101D400030102078102078102030102F03D02F87EB
:101D5000D02787902387103186303800703FFFF0FE
:101D60001FFFF81FFFF8041040020820020820049B
:101D7000104008208010410010410008208004100D
:101D8000400000001FFFF81FFFF8FFFFFF80000169
:101D90008E00E19F01F19381399F81F99F81F99F25
:101DA000B9F98F28F18038018000019FFFF9917403
:101DB000999B06A99B54A99B56A99B54999FFFF9EF
:101DC000FFFFFF6E6F74696669636174696F6E20EF
:101DD0000063616E63656C005072696E74204162CD
:101DE0006F72746564004469736D6973730055495B
:101DF0002041626F72746564004D323520500A4D87
:101E0000323400526573756D650055492050617517
:101E100073650050617573696E672E2E2E007265B2
:101E200073756D65004D3234004C6F6164206D6DCB
:101E300000556E6C6F6164206D6D0046696C2E20DC
:101E40004469612E004520696E206D6D5E3300414E
:101E50006476616E6365204B004D3330332055311D
:101E60002045256920532569005049442041757457
:101E70006F74756E65202A005049442D44202A0055
:101E80005049442D49202A005049442D50202A0011
:101E900020082046616374002008204D61780020EE
:101EA00008204D696E004F6666004F6E00417574E4
:101EB0006F74656D70005654726176204D696E00C6
:101EC000566D696E00566D6178204500566D6178DB
:101ED000205A00566D6178205900566D617820585F
:101EE00000416D6178204500416D6178205A0041C4
:101EF0006D6178205900416D6178205800412D5462
:101F0000726176656C00412D526574726163740074
:101F1000416363656C0056652D4A65726B00565AC5
:101F20002D4A65726B0056592D4A65726B005658E2
:101F30002D4A65726B00452073746570732F6D6D4B
:101F4000005A2053746570732F6D6D0059205374BF
:101F50006570732F6D6D00582053746570732F6D0D
:101F60006D00416476616E636564205365747469C5
:101F70006E6773003F0043616E63656C00496E6974
:101F800074004D34323800496E697469616C697A45
:101F90006520454550524F4D0046696C616D656E38
:101FA000740054656D706572617475726500537468
:101FB0006570732F6D6D004A65726B0041636365D8
:101FC0006C65726174696F6E0056656C6F636974DD
:101FD000790053657420486F6D65204F66667365A0
:101FE000747300436F6E66696775726174696F6EB2
:101FF000003F004E65787420506F696E7400446F26
:102000006E65004E657874004C6576656C696E6728
:1020100020446F6E6521004D6F7665205A0047326F
:10202000395332004E65787420506F696E74002504
:1020300069202F2025750047323953310047323946
:10204000533200436C69636B20746F20426567698B
:102050006E00486F6D696E672058595A005A2056B5
:10206000616C756500496E646578205900496E643D
:10207000657820580053746F7265205365747469D5
:102080006E6773004C6F61642053657474696E678A
:1020900073004C6576656C20436F726E65727300D9
:1020A000426564205A004661646520486569676836
:1020B00074004F6666004F6E00426564204C657682
:1020C000656C696E670045646974204D65736800CE
:1020D0004C6576656C20426564004D6F74696F6E67
:1020E000003F0043616E63656C204F626A656374F4
:1020F000004E4F005945530043616E63656C204F9D
:10210000626A656374203D004D61696E00426564DA
:10211000004E6F7A7A6C650046616E20537065657B
:102120006400436F6E66696775726174696F6E00F3
:10213000526573746F72652044656661756C747363
:10214000004C6F61642053657474696E677300534B
:10215000746F72652053657474696E677300507292
:102160006568656174202420436F6E66004F666663
:10217000004F6E00506F776572204F757461676510
:10218000004C434420436F6E747261737400416469
:1021900076616E6365642053657474696E6773005D
:1021A0004D61696E004D37303220542564004D3644
:1021B000303020423020542564004D373032203BEF
:1021C0002564004D37303120542564004D373032BE
:1021D000004D373031004D363030204230004D61F7
:1021E000696E005075726765206D6F726500436F90
:1021F0006E74696E756500524553554D45204F50BC
:1022000054494F4E533A005052494E542050415574
:102210005345440020204E6F7A7A6C653A20005076
:1022200061726B696E672E2E2E0000005761697413
:1022300020666F720066696C616D656E74206368FC
:10224000616E676500746F2073746172740057610A
:10225000697420666F720066696C616D656E7420CA
:10226000756E6C6F616400004E6F7A7A6C652068E1
:10227000656174696E6700506C6561736520776194
:1022800069742E2E2E00005072657373206275746F
:10229000746F6E00746F2068656174206E6F7A7A57
:1022A0006C650000496E736572742066696C616DBF
:1022B000656E7400616E6420707265737320627560
:1022C00074746F6E00746F20636F6E74696E7565E1
:1022D000005761697420666F720066696C616D6594
:1022E0006E74206C6F6164000050726573732042DD
:1022F0007574746F6E00746F20726573756D6520F0
:102300007072696E7400005761697420666F722084
:102310007072696E7400746F20726573756D652ECE
:102320002E2E00005761697420666F720066696C1A
:10233000616D656E7420707572676500003E2000E7
:10234000256C642E25696D0045787472756465642A
:1023500020546F74616C003E20004C6F6E67657393
:1023600074204A6F622054696D65003E2000546FEE
:1023700074616C205072696E742054696D650043FD
:102380006F6D706C65746564003A20005072696E00
:102390007420436F756E74003A200031353000357B
:1023A000004245443A204154432031303447542DB3
:1023B000320052756E617761792057617463683AB3
:1023C000204F4E004D61782054656D7000343530DB
:1023D000004D696E2054656D7000350045313A201E
:1023E000536C696365456E6720343530C2B0430075
:1023F0005053550047656E657269630050726F7483
:102400006F636F6C00312E300042617564003235AD
:102410003030303000437265616C69747933442028
:1024200052414D5053004D657368204C6576656C84
:10243000696E670045787472756465727300310067
:1024400074696E796D616368696E657333642E6358
:102450006F6D0053755065522043522D323000325B
:102460003032312D30342D313800322E302E375F5E
:102470004457372E33004D61726C696E005072699B
:102480006E74657220537461747300546865726D64
:102490006973746F727300426F61726420496E6673
:1024A0006F005072696E74657220496E666F004DE0
:1024B00061696E004D313030300053746F702050C0
:1024C00072696E7400526573756D65205072696E25
:1024D0007400506F776572204F7574616765003FB7
:1024E000004261636B0053746F70005072696E74C8
:1024F0002066726F6D204D65646961004368616E8E
:102500006765204D65646961004D32310041626F3D
:102510007574205072696E746572004368616E67ED
:10252000652046696C616D656E7400436F6E666907
:102530006775726174696F6E0054656D7065726164
:1025400074757265004D6F74696F6E00486F7374B7
:10255000205374617274004E6F204D656469610090
:10256000526573756D65205072696E740043616EBB
:1025700063656C204F626A6563740054756E650014
:1025800053746F70205072696E740050617573657A
:10259000205072696E7400496E666F2053637265D5
:1025A000656E003F005374617274205072696E74DE
:1025B0000043616E63656C005072696E7400436124
:1025C0006E6E6F7420656E746572207375626469D7
:1025D000723A2000022E2E004D61696E00210048E3
:1025E0006F74656E6420746F6F20636F6C6400425B
:1025F00061636B0050726F63656564004F666600CF
:102600004F6E00536F667420456E6473746F707301
:10261000004D6F74696F6E0044697361626C652070
:102620005374657070657273004D38340042656490
:10263000204C6576656C696E6700486F6D65205A41
:10264000004732385A00486F6D65205900473238CC
:102650005900486F6D652058004732385800417561
:10266000746F20486F6D6500473238004D61696EA8
:102670000050726568656174202420456E640050C6
:102680007265686561742024204265640054656D3C
:10269000706572617475726500436F6F6C646F77FB
:1026A0006E005072656865617420240046616E207A
:1026B0005370656564207E00426564004E6F7A7ACF
:1026C0006C65004D61696E0042616279737465707A
:1026D000205A00416476616E6365204B00466C6F42
:1026E000770046616E205370656564207E00426508
:1026F00064004E6F7A7A6C6500426564205A00531C
:1027000070656564004D61696E00486F6D696E6744
:10271000204661696C6564006F70656E00545249B3
:10272000474745524544003A20007A5F6D696E0084
:10273000795F6D696E00785F6D696E005265706FCC
:102740007274696E6720656E6473746F7020737441
:10275000617475730A0020746F6F206C6F6E672050
:10276000657874727573696F6E2070726576656EC8
:102770007465640A0020636F6C64206578747275F8
:1027800073696F6E2070726576656E7465640A0099
:102790000000000000000000000000005761726EA1
:1027A000696E673A20486F6D696E672042756D707B
:1027B0002044697669736F72203C20310A0002025E
:1027C00004000070430000704300007A43000000E2
:1027D0004100000041000000400000000100000036
:1027E0000100008000555555000000400033333390
:1027F00000AAAA2A004992240000002000C7711CE8
:102800000099991900D1451700555515003BB11392
:10281000002449120011111100000010000F0F0FC9
:1028200000E3380E0043790D00CCCC0C00C3300C13
:1028300000E8A20B0064210B00AAAA0A00703D0A5E
:10284000009DD80900427B090092240900DCD308CE
:1028500000888808001042080000000800F0C10746
:10286000008787070075500700711C07003EEB06C4
:1028700000A1BC06006990060066660600703E0670
:10288000006118060017F4050074D105005BB0055F
:1028900000B29005006272050055550500783905B3
:1028A00000B81E0500050505004EEC040087D404A1
:1028B00000A1BD040090A7040049920400C17D045A
:1028C00000EE690400C7560400444404005C32046E
:1028D000000821040041100400000004003FF00340
:1028E00000F8E0030026D20300C3C30300CCB50305
:1028F000003AA803000A9B0300388E0300C081033E
:10290000009F750300D0690300505E03001D530350
:102910000034480300913D030033330300162903BC
:1029200000381F030097150300300C030003030356
:10293000000BFA020049F10200BAE802005CE00272
:10294000002DD802002DD0020059C80200B0C002EC
:102950000031B90200DAB10200AAAA0200A0A30263
:1029600000BC9C0200FA9502005C8F0200DF880226
:102970000082820200457C02002776020027700256
:1029800000436A02007C640200D05E02003F5902EC
:1029900000C8530200FFFDFCFAF8F6F4F2F0EEEC8A
:1029A000EAE9E7E5E3E1E0DEDCDAD9D7D5D4D2D055
:1029B000CFCDCBCAC8C7C5C3C2C0BFBDBCBAB9B7EB
:1029C000B6B4B3B2B0AFADACAAA9A8A6A5A4A2A153
:1029D000A09E9D9C9A99989795949392908F8E8D96
:1029E0008B8A8988878684838281807F7E7D7B7ABB
:1029F000797877767574737271706F6E6D6C6B6ABF
:102A0000696867666564636261605F5E5D5C5B5AAE
:102A10005958585756555453525150504F4E4D4C8B
:102A20004B4A4A4948474646454443424241403F53
:102A30003E3E3D3C3B3B3A3938383736353534330A
:102A400032323130302F2E2E2D2C2B2B2A292928B3
:102A5000272726252524232322212120201F1E1E4F
:102A60001D1C1C1B1B1A19191818171616151514DE
:102A7000131312121111100F0F0E0E0D0D0C0C0B63
:102A80000A0A0909080807070606050504040303DE
:102A90000202010000000070430000704300007A51
:102AA00043000000000000000000000000536574B7
:102AB00074696E67732053746F7265640045455086
:102AC000524F4D20496E697469616C697A65640A78
:102AD000003B200020204D36303320002055004C94
:102AE0000046696C616D656E74206C6F61642F7552
:102AF0006E6C6F6164206C656E677468733A002059
:102B0000204D393030204B004C696E656172204198
:102B10006476616E63653A0020204D343133205372
:102B200000506F7765722D4C6F7373205265636F21
:102B3000766572793A0020204D3235302043004CC2
:102B4000434420436F6E74726173743A00204400F2
:102B500020490020204D33303420500020440020F4
:102B6000490020204D33303120500050494420731B
:102B7000657474696E67733A00204600204800202F
:102B8000204D3134352053004D6174657269616C9C
:102B90002068656174757020706172616D6574651F
:102BA00072733A002020473239205334205A0020D3
:102BB0004A00202047323920533320490020204D3D
:102BC0003432302053004D65736820426564204CD8
:102BD0006576656C696E673A0020204D323036208C
:102BE0005800486F6D65206F66667365743A002003
:102BF000580020530020204D3230352042004164DF
:102C000076616E6365643A20423C6D696E5F736500
:102C1000676D656E745F74696D655F75733E205393
:102C20003C6D696E5F66656564726174653E2054D3
:102C30003C6D696E5F74726176656C5F6665656434
:102C4000726174653E20583C6D61785F785F6A659B
:102C5000726B3E20593C6D61785F795F6A65726B7B
:102C60003E205A3C6D61785F7A5F6A65726B3E20E8
:102C7000453C6D61785F655F6A65726B3E0020540C
:102C80000020520020204D32303420500041636338
:102C9000656C65726174696F6E2028756E697473F6
:102CA0002F7332293A20503C7072696E745F6163F1
:102CB00063656C3E20523C726574726163745F613F
:102CC0006363656C3E20543C74726176656C5F6131
:102CD0006363656C3E0020204D3230312058004D3A
:102CE0006178696D756D20416363656C65726174AF
:102CF000696F6E2028756E6974732F7332293A00DC
:102D000020204D3230332058004D6178696D756D4B
:102D1000206665656472617465732028756E6974D8
:102D2000732F73293A005374657073207065722095
:102D3000756E69743A0020440020204D32303020F6
:102D400053002044697361626C65640A0046696CD3
:102D5000616D656E742073657474696E67733A0093
:102D600020204D3134392043203B20556E69747347
:102D700020696E2043656C736975730A0020286DA5
:102D80006D29002020473231202020203B20556E25
:102D900069747320696E206D6D0000803B44008073
:102DA0003B4400002041000096420000A042000089
:102DB000A0420000C8430000BE42D0070000D00778
:102DC0000000640000004B00000024F4D43050C325
:102DD0008E20C2A24017828B7011127A910D816CE5
:102DE000D90AA861E108C7586607615143061E4B1E
:102DF0005D05C145A7041A411104093D98037139C5
:102E000031034036DB0265339102D4305402802E08
:102E10001D02632CEE01752AC501B028A001102700
:102E200081018F2564012B244B01E0223401AC2168
:102E30001F018D200D01801FFC00841EED00971DD9
:102E4000DF00B81CD200E61BC600201BBC00641AC1
:102E5000B200B219A8000A19A0006A189900D11787
:102E6000910040178B00B516840031167E00B31513
:102E700079003A157300C7146F0058146A00EE13F6
:102E800066008813630025135E00C7125B006C1296
:102E9000570015125400C111510070114F0021113B
:102EA0004B00D61049008D10470046104400021018
:102EB0004200C00F4000800F3E00420F3C00060F52
:102EC0003B00CB0E3800930E37005C0E3500270E0A
:102ED0003400F30D3200C10D3100900D3000600D53
:102EE0002E00320D2D00050D2C00D90C2B00AE0C40
:102EF0002900850C29005C0C2700350C27000E0CDE
:102F00002600E80B2400C40B2400A00B23007D0B3B
:102F100023005A0B2100390B2100180B2000F80A5E
:102F20001F00D90A1E00BB0A1E009D0A1D00800A50
:102F30001D00630A1C00470A1B002C0A1B00110A13
:102F40001A00F7091A00DD091900C4091900AB09B4
:102F50001900920917007B091800630917004C0932
:102F6000160036091600200916000A091500F50892
:102F70001500E0081400CC081400B8081400A408D8
:102F80001400900813007D0812006B081300580805
:102F9000120046081200340811002308110012081C
:102FA000110001081100F0071000E0071000D00721
:102FB0001000C0071000B0070F00A1071000910714
:102FC0000E0083070F0074070F0065070E005707F8
:102FD0000E0049070E003B070D002E070E002007CC
:102FE0000D0013070D0006070D00F9060C00ED0695
:102FF0000D00E0060C00D4060C00C8060C00BC0650
:103000000C00B0060C00A4060B0099060C008D06FF
:103010000B0082060B0077060B006C060B006106A6
:103020000A0057060B004C060A0042060A00380642
:103030000A002E060A0024060A001A060A001006D4
:10304000090007060A00FD050900F4050900EB0563
:103050000900E2050900D9050900D0050900C705E6
:103060000900BE050900B5050800AD050800A50565
:1030700009009C050800940508008C0508008405DB
:1030800008007C050800740508006C05070065054C
:1030900008005D050700560508004E0507004705B6
:1030A00007004005080038050700310507002A051C
:1030B0000700230507001C050600160507000F057D
:1030C00007000805060002050700FB040600F504DA
:1030D0000700EE040600E8040600E2040700DB0433
:1030E0000600D5040600CF040600C9040600C30488
:1030F0000600BD040600B7040600B1040500AC04D8
:103100000600A6040600A00405009B040600950422
:103110000500900406008A0405008504050080046B
:1031200006007A04050075040500700405006B04B0
:10313000050066040500610405005C0405005704F1
:103140000500520405004D04050048040500430431
:1031500005003E0404003A0405003504050030046F
:1031600004002C04050027040400230405001E04A9
:1031700004001A04040016040500110404000D04E0
:103180000400090405000404040000040400FC0316
:103190000400F8030400F4030400F0030400EC034B
:1031A0000400E8030400E4030400E0030400DC037B
:1031B0000400D8030400D4030400D0030400CC03AB
:1031C0000400C8030300C503030024F404D9201B32
:1031D000C40C5C0E9804C4095F0265077101F40514
:1031E000F900FB04B30048048700C10369005803D9
:1031F000550003034500BE023A0084023100530229
:103200002A002902250004022000E4011C00C80154
:103210001900AF0117009801140084011300710117
:1032200010006101100051010E0043010D00360134
:103230000B002B010B0020010B00150109000C01F4
:10324000090003010800FB000800F3000800EB0080
:103250000700E4000600DE000600D8000600D200E9
:103260000600CC000500C7000500C2000500BD0037
:103270000400B9000400B5000400B1000400AD0072
:103280000400A9000400A5000300A20003009F00A1
:1032900004009B00030098000300950002009300C7
:1032A0000300900003008D0002008B0003008800E3
:1032B00002008600020084000300810002007F00FB
:1032C00002007D0002007B0002007900020077000E
:1032D000010076000200740002007200010071001B
:1032E00002006F0002006D0001006C0002006A0025
:1032F000010069000200670001006600010065002E
:103300000100640002006200010061000100600031
:1033100001005F0002005D0001005C0001005B0035
:1033200001005A0001005900010058000100570037
:103330000100560001005500010054000100530037
:103340000000530001005200010051000100500034
:1033500001004F0001004E0000004E0001004D0032
:1033600001004C0001004B0000004B0001004A002E
:10337000010049000100480000004800010047002A
:103380000100460000004600010045000000450025
:10339000010044000100430000004300010042001E
:1033A0000000420001004100000041000100400017
:1033B00001003F0000003F0001003E0000003E0011
:1033C00001003D0000003D0001003C0000003C0009
:1033D00000003C0001003B0000003B0001003A00FF
:1033E00000003A00010039000000390001003800F7
:1033F00000003800000038000100370000003700EE
:1034000001003600000036000000360001003500E3
:1034100000003500000035000100340000003400D9
:1034200000003400010033000000330000003300CE
:1034300001003200000032000000320001003100C3
:1034400000003100000031000100300000003000B9
:103450000000300001002F0000002F0000002F00AE
:1034600000002F0001002E0000002E0000002E00A2
:1034700001002D0000002D0000002D0000002D0097
:1034800001002C0000002C0000002C0000002C008B
:1034900001002B0000002B0000002B0000002B007F
:1034A00001002A0000002A0000002A0000002A0073
:1034B0000100290000002900000029000000290067
:1034C000000029000100280000002800000028005A
:1034D000000028000000280001002700000027004D
:1034E0000000270000002700000027000100260040
:1034F0000000260000002600000026000000260034
:103500000100250000002500000025000000250026
:103510000000250000002500010024000000240018
:10352000000024000000240000002400010023000B
:1035300000002300000023000000230000002300FF
:1035400000002300000023000100220000002200F0
:1035500000002200000022000000220000002200E3
:1035600001002100000021000000210000002100D6
:1035700000002100000021000000210001002000C7
:1035800000002000000020000000200000002000BB
:1035900000002000000020000000200001001F00AB
:1035A00000001F0000001F0000001F0000001F009F
:1035B00000001F0000001F0001001E0000001E0090
:1035C00000001E0000001E000000232C0000B82296
:1035D0000000561800003A0F0000B8080000B104BF
:1035E0000000710200003E01000020436F756E7400
:1035F00020583A0042656400453100626564002C41
:103600002073797374656D2073746F7070656421B5
:10361000204865617465725F49443A2000486561DD
:1036200074696E67204661696C6564004865617401
:10363000696E67206661696C6564004D31313220C6
:1036400053687574646F776E001000C90210012C06
:10365000014001220170011801B0010E01F00104C6
:10366000015002FA00B002F0003003E600D003DCA3
:10367000009004D2007005C800A006BE000008B487
:1036800000B009AA00D00BA000600E960060118C5B
:10369000000015820020197800C01D6E00A0226471
:1036A00000B0275A00902C500000314600E0343C16
:1036B0000010383200903A2800603C1E00A03D14F3
:1036C00000803E0A00203F0000544845524D414CC6
:1036D0002052554E4157415900546865726D616CD6
:1036E0002052756E61776179004572723A204D41C2
:1036F0005854454D50004D415854454D502074721A
:1037000069676765726564004572723A204D494E7B
:1037100054454D50004D494E54454D5020747269EA
:1037200067676572656400202F002042403A0020E0
:10373000403A0020573A0020573A00496E76616CB3
:1037400069642065787472756465720A007C3C3E19
:103750005E2B3D3F2F5B5D3B2C2A225C0043616E5C
:103760006E6F74206F70656E20737562646972206D
:1037700000534420496E6974204661696C005344CB
:103780002063617264206F6B0A006F70656E526F08
:103790006F74206661696C65640A00766F6C756D84
:1037A000652E696E6974206661696C65640A004EF5
:1037B0006F20534420636172640A000A4D32340062
:1037C0004D32332025730041425300504C41002EAE
:1037D0000A006F70656E206661696C65642C204616
:1037E000696C653A200046696C652073656C656399
:1037F0007465640A002053697A653A200046696C52
:1038000065206F70656E65643A2000454E44205314
:103810005542524F5554494E450A002220706F734D
:10382000002220706172656E743A22005355425234
:103830004F5554494E452043414C4C2074617267AA
:1038400065743A220053756263616C6C204F766533
:1038500072666C6F77004578636565646564206D9A
:10386000617820535542524F5554494E4520646566
:103870007074683A002E0A0044656C6574696F6E56
:10388000206661696C65642C2046696C653A20008D
:1038900046696C652064656C657465643A005344E0
:1038A000207072696E74696E672062797465200099
:1038B0004E6F74205344207072696E74696E670A8B
:1038C000002F6175746F25632E67005772697469E4
:1038D0006E6720746F2066696C653A2000667265B9
:1038E000736800646F696E67002066696C653A20D2
:1038F000004E6F77200002FD55555555555FFFFF6F
:10390000FFFFFFFFFFFFFFFE00000000003FFFFF83
:10391000FFFFFFFFFFFFFFFD000007FFFFFFFFFFAF
:10392000FFFFFFFFFFFFFFFE07C00555555555552B
:103930005FFFFFFFFFFFFFFC0A2006000000000002
:103940003FFFFFFFFFFFFFFE141005000007FFFF12
:10395000FFFFFFFFFFFFFFFC28080607C0055555C6
:103960005555555FFFFFFFFE5404040A2006000072
:103970000000003FFFFFFFFC60040614100500007C
:1039800007FFFFFFFFFFFFFE50040428080607C0E3
:103990000555555555555FFC6004065404040A202E
:1039A0000600000000003FFE54041C6004061410D2
:1039B0000500000000001FFC28082E500404280801
:1039C0000607C00001F03FFE1410546004065404C2
:1039D000040A200002081FFC0A206654041C60042C
:1039E0000614100005043FFE07C05428082E50049A
:1039F000042808000A021FFC00002E141054600462
:103A00000654040015013FFE00001C0A2066540401
:103A10001C60040018011FFC00000607C0542808A1
:103A20002E50040014013FFE00000400002E14106C
:103A30005460040018011FFCFFFFFE00001C0A2058
:103A40006654041C15013FFED5555400000607C0FE
:103A50005428082A0A021FFC8410460000040000B3
:103A60002E14105105043FFEC41044FFFFFE000059
:103A70001C0A206102881FFC841046D555540000A2
:103A80000607C05101F03FFE841044841046000038
:103A90000400002A00001FFCC41046C41044FFFFAD
:103AA000FE00001C00003FFE841044841046D555E3
:103AB0005400000000001FFCD555568410448410AB
:103AC0004600000000003FFCFFFFFCC41046C4108D
:103AD00044FFFFFFFFFF9FFE000006841044841098
:103AE00046D555555555BFFD555554D55556841099
:103AF0004484104104109FFFFFFFFCFFFFFCC41033
:103B000046C410410411BFFFFFFFFE0000068410F1
:103B10004484104104109FFFFFFFFD555554D555B7
:103B20005684104104109FFFFFFFFFFFFFFCFFFFC3
:103B3000FCC410410411BFFFFFFFFFFFFFFE0000A8
:103B40000684104104109FFFFFFFFFFFFFFD555546
:103B500054D555555555BFFFFFFFFFFFFFFFFFFF32
:103B6000FCFFFFFFFFFF9FFFFFFFFFFFFFFFFFFFC8
:103B7000FE00000000003FFFFFFFFFFFFFFFFFFF11
:103B8000FD55555555555FFFFFFFFFFFFFFFFFFF39
:103B9000FFFFFFFFFFFFFFFFFFFFFFFFFFFFFFFF35
:103BA000FFFFFFFFFFFFFFFFFFFFFFFFFFFFFFFF25
:103BB000FFFFFFFFFFFFFFFFFFFFFFFFFFFFFFFF15
:103BC000FFFFFFFFFFFFFFE02EFB7DFBFBCFC1DF11
:103BD000BB3EC0E1FE3C1FFDEE7B39F9F3CF9EDF1B
:103BE000BB3EDFDEFCDDE7FDEE3BBBF9EBD7BF5FA5
:103BF000BB5EDFDEFDEDF7FDEEBBD3FAEBB73FDFDB
:103C0000BB4EDFDFFFCDF3FDEEDBC7FAEBBB7FC0C2
:103C10003B6EC0E3FF1DF3FDEECBEFFADBBB7FDFB6
:103C2000BB66DFF8FFCDF3FDEEEBEFFB5B033F5F21
:103C3000BB76DFFE7FEDF3FDEEF3EFFB5B79BEDFDE
:103C4000BB7ADFDE7DEDF7FDEEF3EFFBBAFD9EDF25
:103C5000BB7CDFDEFDCDE7FDEEFBEFFBBAFDC1DF98
:103C6000BB7EC0E0FE1C1F6D61726C696E66772EB4
:103C70006F726700322E302E375F4457372E330075
:103C80001FFFFFFFFFFFFF600000000001FF40007B
:103C900000000000FF8000000000007F83CF0000D4
:103CA0000C303F87FF80000C301F867980000C00AD
:103CB0000F8C30C7838C30E78C30CFC7CC31F38C7E
:103CC00030DCECEC33B98C30D86C6C33198C30D0E0
:103CD0006C0C33198C30D86C0C33198C30DC6C0EB6
:103CE0003B198C30CF7C079F198C30C77C038F1910
:103CF00040000000000002600000000000061FFFFE
:103D0000FFFFFFFFF86001F4017001EA019001E09C
:103D100001B001D601D001CC010002C2013002B8CD
:103D2000016002AE019002A401D0029A012003902A
:103D30000170038601C0037C0130047201A0046895
:103D40000120055E01B005540160064A01200740CC
:103D500001F0073601F0082C01100A2201500B185F
:103D600001C00C0E01500E04013010FA002012F0B8
:103D7000005014E600C016DC007019D200501CC8B8
:103D800000501FBE007022B400B025AA00F028A089
:103D900000202C9600302F8C0010328200A0347846
:103DA00000F0366E00E0386400803A5A00403B551F
:103DB00000E03B5000F03C4600C03D3C00603E321D
:103DC00000E03E2800303F1E00503F1900703F14B5
:103DD00000A03F0A00C03F0000D03FF6FFE03FECEC
:103DE000FF2020506C616E6E65724275666665726A
:103DF00042797465733A20002046726565204D65EE
:103E00006D6F72793A2000436F6D70696C65643A2A
:103E10002041707220323420323032310A00204C7E
:103E200061737420557064617465643A2032303275
:103E3000312D30342D3138207C20417574686F72FB
:103E40003A2054696E794D616368696E65733344D5
:103E50000A00322E302E375F4457372E330A004D7A
:103E600061726C696E0020536F66747761726520B1
:103E700052657365740A00205761746368646F67E4
:103E80002052657365740A002042726F776E206F4E
:103E900075742052657365740A00204578746572E4
:103EA0006E616C2052657365740A00506F7765729D
:103EB00055700A0073746172740A00473238585999
:103EC000004D31303031006572726F722077726947
:103ED00074696E6720746F2066696C650A00446FB0
:103EE0006E6520736176696E672066696C652E0A5F
:103EF000004D323900456E6473746F707300255342
:103F000020256320256320256320256300205A3A5D
:103F10000020593A0020583A00656E6473746F703F
:103F200073206869743A200000000A0B02090C0D26
:103F30000E0807030401000000000000000000005C
:103F40000000000000000000000000000000000071
:103F5000000000001211100000000000000000002E
:103F60000000000000000000000000000000004D04
:103F70006F76652025736D6D004D6F766520302E50
:103F8000316D6D004D6F766520316D6D004D6F7632
:103F9000652031306D6D004D6F7665204178697315
:103FA000004578747275646572004D6F7665205AAD
:103FB000004D6F76652059004D6F7665205800CB17
:103FC00037C7374368616E67652046696C616D6508
:103FD0006E7400556E6C6F61642046696C616D652E
:103FE0006E74004C6F61642046696C616D656E741F
:103FF000005072656865617420437573746F6D005D
:10400000507265686561742024004261636B00FF33
:10401000FFFF486F6D652025732573257320466962
:104020007273740070726F6D70745F0073686F7775
:1040300000627574746F6E00626567696E0050751A
:104040007267654D6F7265005061757365640043FA
:104050006F6E74696E7565004C6F61642046696CA3
:10406000616D656E74205400496E736572742066CC
:10407000696C616D656E7420616E642073656E6439
:10408000204D3130380A00220A00556E6B6E6F7772
:104090006E20636F6D6D616E643A202200204200D5
:1040A0002050006F6B0053755065522043522D32E3
:1040B000302052656164792E005072696E74696EA9
:1040C000672E2E2E005072696E74205061757365D4
:1040D0006400204500205A00205900204D3932202C
:1040E000580020453A00205A3A0020593A00583AE0
:1040F0000020746F6F206C6F6E6720657874727526
:1041000073696F6E2070726576656E7465640A00FF
:1041100020636F6C6420657874727573696F6E20AC
:1041200070726576656E7465640A00526573656EBB
:10413000643A20006E6F74696669636174696F6EBA
:10414000200000002200250028002B002E00310056
:10415000340002010000050108010B0100002100EC
:10416000240027002A002D00300033000101000048
:10417000040107010A0105050505070508080808E7
:10418000020202020A0A08080404040401010101EF
:1041900001010101030303030303030304070707EA
:1041A0000C0C0C0C0C0C0C0C02020202060606068F
:1041B000060606060B0B0B0B0B0B0B0B010210205C
:1041C000200808102040102040800201020108044D
:1041D00002010102040810204080804020100804E1
:1041E000020180040201804020100804020108043A
:1041F000020101020408102040800102040810207E
:1042000040802001240211241FBECFEFD1E2DEBF87
:10421000CDBF00E00CBF13E0A0E0B2E0E2E1FAEBBA
:1042200002E00BBF02C007900D92AC36B107D9F780
:1042300028E1ACE6B3E001C01D92A63DB207E1F76C
:1042400011E2C2E0D1E200E006C021970109802F0F
:10425000FE010F946659C130D10780E00807A9F725
:104260000F941C480D94F75C0C940000FC018491A1
:104270000895FC018081089590E080E00895CF9337
:10428000DF93DB01F9019C919130C1F0943080F013
:1042900094509C938830D1F480819181009771F083
:1042A000019791838083480F591FEA01188206C045
:1042B0008C3539F49C5F9C93943041F4DF91CF911D
:1042C00008958B3339F781E08C93F8CF20813181C9
:1042D000B9016F5F7F4F71836083420F531FEA0103
:1042E0008883808191818F3591056CF7E7CF0F939B
:1042F0001F9381E00091BD161091BE162091BF164C
:104300003091C0164091B9165091BA166091BB1603
:104310007091BC16041715072607370708F480E0CC
:104320001F910F91089590E080E00895282F9091BB
:104330006608833021F495FD0FC094FD0FC0892FCE
:1043400090E0B0E0A0E004C0B695A795979587955A
:104350002A95D2F78170089581E0089580E008954C
:10436000129A0895269A2E9A0895EF92FF920F932B
:104370001F93CF93DF93EC018B017A018A859B8594
:104380008617970731F0888199810F94683D1B87C4
:104390000A87B701888199810F942D2F2E813F8143
:1043A000820F932F911D9F838E8390E080E0DF9199
:1043B000CF911F910F91FF90EF9008959F92AF9230
:1043C000BF92CF92DF92EF92FF920F931F93CF9302
:1043D000DF93EC018B01942EA52E8A859B85861791
:1043E000970731F0888199810F94683D1B870A8770
:1043F00088859985019649F5BC800A818E81080FD0
:10440000C880D980D6015596ED91FC91C6011995C9
:10441000B80EE92CFA2C10E0F70121917F0121114F
:1044200027C08E819F81810F911D9F838E8390E095
:1044300080E0DF91CF911F910F91FF90EF90DF907F
:10444000CF90BF90AF909F9008950E811F81692DEE
:104450007A2D888199810F942D2F800F912F911D96
:10446000288539852817390738F681E090E0E1CFB3
:104470004B2D602FC6010F94C03D080F180FCCCFF5
:10448000DF92EF92FF920F931F93CF93DF93EC0194
:10449000D62E1CAD0BAD7C0184E0E80EF11CE98D3D
:1044A000FA8DC7011995412F480F2D2D602FC70197
:1044B0000F94C03D9BAD890F8BAF81E090E0DF9101
:1044C000CF911F910F91FF90EF90DF900895AF92E1
:1044D000BF92DF92EF92FF920F931F93CF93DF93E0
:1044E0008C01EB01D42E79018FE0481709F486C0C6
:1044F000A5E14A17B1F1BAE04B130EC0EC81FD8182
:1045000030E020E042E061E0C80119954CE057E15D
:10451000BE01C8010F946B3E0A80DB81C02DF2E31F
:10452000DF1609F4E2C0FD1508F491C085E1D81644
:1045300009F4E0C0A7E1DA1609F4EFC0B4E1DB1238
:104540007BC0EE81FF818D8190E0880F991F8E0FD7
:104550009F1F11928E179F07E1F7CE010F94883BA2
:104560006BC0AA80BB8047EF56E1C8010F946B3E39
:10457000F5014481440F406BBE01C8010F94533EC6
:1045800041E0BE01C8010F945B3ED50116962D9106
:104590003C911797EC81FD8115964C9166E0C8011E
:1045A000199540E0BE01C8010F94633E47EF56E104
:1045B000BE01C8010F946B3EF5014481440F4F5F6B
:1045C000406BBE01C8010F94533E41E0BE01C801DB
:1045D0000F945B3ED50115964C91159716962D912B
:1045E0003C91240F311DEC81FD8166E0C8011995D5
:1045F00040E0BE01C8010F94633E8ECF41E0C80188
:104600000F94633E40E0BE01C8010F945B3E41E859
:10461000BE01C8010F94533EF701408150E055950B
:10462000479555954795BE01C8010F94533E40E00C
:10463000BE01C8010F94633E81E0DF91CF911F91CD
:104640000F91FF90EF90DF90BF90AF900895E6E458
:10465000DE1609F471C0F7E4DF1609F471C08BE3CC
:10466000D812EACFD70111969C91119713968C918D
:1046700038E0390F813031F0833011F0392F02C02A
:10468000392F985021E04B81491708F420E041E090
:10469000391708F040E091E05A81351708F490E0AE
:1046A000322F342B932311F4242331F2F70112819A
:1046B00000E0D12C843048F490E0FC01E855FD4F37
:1046C000D0808C559D4FDC010C9117FF04C0B701C1
:1046D000CE010F948F3BF70180818D0D8083818106
:1046E000800F8183110F89F7A7CFB701CE010F94F7
:1046F0008F3BA2CFCE010F94723B882309F49DCF4C
:10470000EE81FF818D8190E0880F991F8E0F9F1F92
:1047100011928E179F07E1F78FCFD7011C928A81E4
:1047200011968C9311978D81815012968C931297CC
:104730008B8113968C9380CF8D81F70180837CCF02
:104740008981D7018C9378CFAB01BC014093BD1612
:104750005093BE166093BF167093C01686E298E120
:104760000C94AACE809323028032B8F5909107056D
:10477000891724F091E0980F909307054091030565
:10478000509104056091050570910605082E04C03E
:1047900076956795579547950A94D2F7417040935F
:1047A000521087FD1DC0282F082E000C330B3F939D
:1047B0008F938EE599E09F938F938EE699E09F9378
:1047C0008F931F920E9439B28DB79EB707960FB68E
:1047D000F8949EBF0FBE8DBF089510925210E1CF86
:1047E0000D9482420F931F93CF93DF9300D01F92BB
:1047F000CDB7DEB79C0105E318E090E1EDE9F0E10B
:10480000D80101900D929A95E1F7F901208131814B
:1048100042815381F80160857185828593850F946B
:104820006F59F801608771878287938780E090E0F5
:10483000A0EAB0E489839A83AB83BC83CE0101965E
:104840000E9451F90F900F900F900F90DF91CF9130
:104850001F910F9108952F923F924F925F926F9206
:104860007F928F929F92AF92BF92CF92DF92EF9200
:10487000FF921F93CF93DF93CDB7DEB72C970FB680
:10488000F894DEBF0FBECDBF7A011901DC012D9176
:104890003D914D915C912D833E834F835887FB0161
:1048A000408051806280738080909D1090909E1017
:1048B000A0909F10B090A010A50194016D817E8101
:1048C0008F8198850F947D5281110EC011E0A30154
:1048D00092016091A1107091A2108091A31090910B
:1048E000A4100F947D52811110E0D1012D913D91C2
:1048F0004D915C9129873A874B875C87F701C0808F
:10490000D180E280F3802091090230910A02409127
:104910000B0250910C02C701B6010F947D528823FF
:1049200009F44EC0C0920902D0920A02E0920B0232
:10493000F0920C028091A9109091AA10A091AB1056
:10494000B091AC104091A1105091A2106091A310B1
:104950007091A4108092350890923608A092370882
:10496000B09238084093390850933A0860933B0856
:1049700070933C08C0923D08D0923E08E0923F08F8
:10498000F09240088093410890934208A093430816
:10499000B093440820E030E040E05FE36091801095
:1049A0007091811080918210909183100F94E35246
:1049B00069837A838B839C83CE0101960E9451F98F
:1049C0002D813E814F8158852093350830933608DC
:1049D00040933708509338084092390850923A086B
:1049E00060923B0870923C08D1012D913D914D9110
:1049F0005C916091410870914208809143089091C8
:104A000044080F946F596093410870934208809353
:104A100043089093440811112FC020E030E0A90111
:104A200069857A858B859C850F947D52811133C071
:104A300060E070E088EC92E469837A838B839C83E6
:104A4000CE0101960E9451F92C960FB6F894DEBF64
:104A50000FBECDBFDF91CF911F91FF90EF90DF9000
:104A6000CF90BF90AF909F908F907F906F905F900E
:104A70004F903F902F9008952AEF3EE74AE25FE380
:104A800060918410709185108091861090918710AC
:104A90000F94E352D1CF60E070E080EA91E4CCCF94
:104AA0008091BF049091C004009731F04AE050E03B
:104AB00070E060E00D94985060E070E0CB010895E4
:104AC00080915F0982FF0BC063E682E49AE00E9456
:104AD00054B20F947C350E9419B981E0089580E0AA
:104AE00008958091BF049091C004009731F04AE08E
:104AF00050E070E060E00D946A4F60E070E0CB0140
:104B00000895AF92BF92CF92DF92EF92FF920F93F0
:104B10001F93CF93DF93EC015B018A01FB01199591
:104B200087FD16C0C82ED12CF12CE12C2196F8015E
:104B3000C082D182E282F382CE01DF91CF911F91B8
:104B40000F91FF90EF90DF90CF90BF90AF900895BE
:104B5000982F907E903CA9F48F7190E0B0E0A0E097
:104B60006C017D0156E0CC0CDD1CEE1CFF1C5A953F
:104B7000D1F7CE010196F50119958F73C82A2296B7
:104B8000D6CF982F907F903E11F58F7090E0B0E0D7
:104B9000A0E06C017D0136E0CC0CDD1CEE1CFF1C9E
:104BA0003A95D1F7CE010196F50119958F73C82A70
:104BB00046E0CC0CDD1CEE1CFF1C4A95D1F7CE0163
:104BC0000296F50119958F73C82A2396B0CF982FB6
:104BD000987F903F79F5877090E0B0E0A0E06C019D
:104BE0007D0186E0CC0CDD1CEE1CFF1C8A95D1F704
:104BF000CE010196F50119958F73C82A96E0CC0C69
:104C0000DD1CEE1CFF1C9A95D1F7CE010296F50132
:104C100019958F73C82A26E0CC0CDD1CEE1CFF1CF6
:104C20002A95D1F7CE010396F50119958F73C82AFD
:104C300024967DCF982F907C903841F4807C8038EA
:104C400069F42196CE01F5011995F8CF8E7F8D3F3D
:104C500028F02196CE01F5011995F8CFC12CD12C61
:104C6000760165CF9CE0899F802D112491E0980FFB
:104C7000909308052CE0280F20932F0830E02E5F3A
:104C80003F4F409187164217130619F014F080E049
:104C90000895209189169217D0F7662341F08E5F10
:104CA0000F94823C80912F088E5F0F94823C8091FC
:104CB0002F0890918716891750F3209189169091AB
:104CC0000805291720F310928A1680938B1681E02D
:104CD00008952091F904022E000C330B821713065D
:104CE00041F08093F90469E377E183E596E10D945F
:104CF000683D08951F93CF93DF931F92CDB7DEB722
:104D00008F3F910519F014F08FEF90E088379105EF
:104D100014F488E790E09093520280935102182F88
:104D200080918C16811105C081E080938C160F94C0
:104D3000A93B609155167091561619839E012F5FFD
:104D40003F4F4FE083E596E10F94A53B0F90DF9135
:104D5000CF911F910895CF938091FA0481114FC094
:104D600010928A1610928B1610928C16109258166A
:104D70001092571610925A161092591610925C16ED
:104D800081E080935B1682E280935D16109262163A
:104D900010926116E6E7F6E124E836E18FEF8193A1
:104DA0002E173F07E1F7C1E0C093731628E231E008
:104DB0003093691620936816C0936A1610926B168A
:104DC00010926C1690E490936D1610926E1626E673
:104DD00032E0309385162093841626E132E030933A
:104DE00056162093551699E1909378169BE190936F
:104DF0007716809376160F94A93BC093FA0480919E
:104E00005102909152020E947A2681E08093FB0425
:104E100087EF96E19093C6158093C5151092C8153B
:104E20001092C715CF910895CF92DF92EF92FF9223
:104E30000F931F93CF93DF93CDB7DEB72C970FB6A9
:104E4000F894DEBF0FBECDBF6F3F710581059105A0
:104E500009F0D0F48FE496E10E944022E0915716C9
:104E6000F09158163196849190E02C960FB6F894F4
:104E7000DEBF0FBECDBFDF91CF911F910F91FF908D
:104E8000EF90DF90CF900895F0908A16E0908B1607
:104E90002091FB0421110FC047ED56E16E2D8F2D9F
:104EA0000F942C3E90E080E0F80EF0928A16E0928B
:104EB0008B169927DACFC0905716D090581623E555
:104EC00036E13A8329832F2D30E03C832B832E2D2E
:104ED00030E03E832D8318861F822FEF3FEF3A8705
:104EE00029871C861B860EED11E29E012F5F3F4F26
:104EF000AB01BC01C6010F946925B60183E596E1BB
:104F00000F94683D8F819885CFCFCF93DF93FC01BD
:104F100025AD211104C021E025AF0F94A93BC0911C
:104F20005516D0915616E0918416F091851682E0C0
:104F30001995E0918416F091851681E0199530E07D
:104F400020E044E1BE0183E596E10F94A53B26E80D
:104F500036E147E1BE0183E596E10F94A53BE09180
:104F60008416F091851680E0DF91CF911994CF924D
:104F7000DF92EF92FF920F931F93CF93DF93CDB702
:104F8000DEB72C970FB6F894DEBF0FBECDBFF09002
:104F90008A16E0908B162091FB0421111DC047EB6F
:104FA00056E16E2D8F2D0F942C3E90E080E0F80E90
:104FB000F0928A16E0928B1699272C960FB6F894E9
:104FC000DEBF0FBECDBFDF91CF911F910F91FF903C
:104FD000EF90DF90CF900895C0905716D09058165C
:104FE00023E536E13A8329832F2D30E03C832B8360
:104FF0002E2D30E03E832D8318861F827A876987A5
:105000001C861B860EED11E29E012F5F3F4F46E38B
:1050100051E2BC01C6010F942D26B60183E596E14D
:105020000F94683D8F819885C2CF6FEF7FEF0C940E
:10503000B727CF92DF92EF92FF920F931F93CF93F8
:10504000DF93CDB7DEB72C970FB6F894DEBF0FBE57
:10505000CDBFF0908A16E0908B162091FB042111B1
:105060001DC047E956E16E2D8F2D0F942C3E90E028
:1050700080E0F80EF0928A16E0928B1699272C9613
:105080000FB6F894DEBF0FBECDBFDF91CF911F9159
:105090000F91FF90EF90DF90CF900895C09057163A
:1050A000D090581623E536E13A8329832F2D30E03E
:1050B0003C832B832E2D30E03E832D8318861F8268
:1050C0007A8769871C861B860EED11E29E012F5F91
:1050D0003F4F49E351E2BC01C6010F942D26B601B2
:1050E00083E596E10F94683D8F819885C2CFBF928A
:1050F000CF92DF92EF92FF920F931F93CF93DF93A4
:105100008B01F42EE90141FB662760F90E943226EB
:10511000882309F45AC0B12C0115110521F0C801EA
:105120000E94EAB9B82EE12C209721F0CE010E940E
:10513000D5BBE82E80E8C82ED12CF0FE1EC085E13C
:1051400090E08B199109B7FC93958E199109E7FCB2
:10515000939597FD019695958795F82E30E8C32E87
:10516000D12CFA94F7FC09C060E270E080E090E096
:105170000E941427C81AD90AF4CFBB2099F0C6019F
:1051800066E070E00F943E59262F4091310850910F
:10519000320860913008C8010E942AB996E0899FC0
:1051A00060011124EE2031F0B601CE010E941928D1
:1051B000C81AD90A87E0C816D10438F060E270E056
:1051C00080E090E00E941427F3CFDF91CF911F91F0
:1051D0000F91FF90EF90DF90CF90BF9008956FEF09
:1051E0007FEF0C941928AF92BF92CF92DF92EF928B
:1051F000FF920F931F93CF93DF935C016B010E948B
:10520000EAB9E82EC6010E94D5BBF12C03E110E0FB
:10521000081B1109C5E20E151F050CF4CFE18C2FF8
:1052200090E09C012E5F3F4F409187164217130676
:1052300009F0CCF5099720918916281719069CF1D9
:1052400040913108509132086091300810928A16CE
:10525000C0938B1625E1C5010E942AB9D1E0C11483
:10526000D104B1F06AE370E080E090E00E9414277E
:105270000E151F05D4F4C45F80918716C81740F03F
:10528000209189164C2F4950550B241715067CF494
:10529000DF91CF911F910F91FF90EF90DF90CF9012
:1052A000BF90AF900895D0E0DACFDD2389F3802F4F
:1052B000880F080F000F00938A16C0938B1660E2C8
:1052C00070E080E090E00E941427C601DF91CF914A
:1052D0001F910F91FF90EF90DF90CF90BF90AF9014
:1052E0000C94EF288F929F92AF92BF92CF92DF9251
:1052F000EF92FF920F931F93CF93DF93CDB7DEB75B
:105300002C970FB6F894DEBF0FBECDBF982F862F17
:105310005A017901D02E692F0E943226882309F480
:1053200089C0C701002391F10E94EAB9C82E80907C
:105330005716909058168091FB04811145C01FEFBD
:1053400023E12C19409131085091320860913008C6
:10535000C5010E942AB9CC2009F46CC0B6E08B9F2D
:10536000500111246AE370E080E090E00E9414276D
:1053700057E0A516B10408F444C060E270E080E094
:1053800090E00E941427A81AB90AF2CF0E94D5BB58
:10539000C82E80905716909058168091FB04882351
:1053A00071F2FE0133968AE0DF011D928A95E9F7DA
:1053B00083E596E19A83898305EB11E29E012F5FD5
:1053C0003F4F49E351E212C0FE0133968AE0DF010C
:1053D0001D928A95E9F783E596E19A83898305EB27
:1053E00011E29E012F5F3F4F46E351E2B701C40136
:1053F0000F942D26B40183E596E10F94683D1F813B
:105400009FCF40912F08212F30E0A6E0CA9EC00117
:1054100011242E5F3F4F281739070CF49C0180E8B8
:10542000821B80938A1640938B16C701DD20A9F05A
:105430000E9415282C960FB6F894DEBF0FBECDBF84
:10544000DF91CF911F910F91FF90EF90DF90CF9060
:10545000BF90AF909F908F9008950E94EF28EACF61
:10546000EFE4F6E183AF64AFCA010C94EF282F920A
:105470003F924F925F926F927F928F929F92AF92E4
:10548000BF92CF92DF92EF92FF920F931F93CF9331
:10549000DF93D62FC72FFC0180809180A280B3803C
:1054A000C501B40120E831E541E050E00F94C15856
:1054B000C9016DE671E00F943E596B017C01C50195
:1054C000B40120E13EE040E050E00F94C158CA0131
:1054D000B90128E130E040E050E00F94C158362E89
:1054E000272E062F172F8CE3482E512C612C712C60
:1054F000C501B401A30192010F94C158B62EA72E85
:10550000CA01B901A30192010F94C158CB01C11482
:10551000D10479F1AF92BF927F936F932F923F9214
:10552000FF92EF92DF92CF9285EF94E19F938F935A
:10553000CF93DF930F9414528DB79EB70E960FB68C
:10554000F8949EBF0FBE8DBF8D2F9C2FDF91CF9102
:105550001F910F91FF90EF90DF90CF90BF90AF9091
:105560009F908F907F906F905F904F903F902F9083
:105570000895E114F104C9F0AF92BF927F936F9345
:105580002F923F92FF92EF9285EE94E19F938F933B
:10559000CF93DF930F941452EDB7FEB73C960FB63E
:1055A000F894FEBF0FBEEDBFCFCF012BB9F0AF9285
:1055B000BF927F936F932F923F9289ED94E19F93D7
:1055C0008F93CF93DF930F9414528DB79EB70A96A3
:1055D0000FB6F8949EBF0FBE8DBFB6CF892BA9F032
:1055E000AF92BF927F936F9381ED94E19F938F93DE
:1055F000CF93DF930F941452EDB7FEB738960FB6E2
:10560000F894FEBF0FBEEDBF9FCFAF92BF928DEC5F
:1056100094E19F938F93CF93DF930F9414520F9045
:105620000F900F900F900F900F908ECF8F929F92B0
:10563000AF92BF92CF92DF92EF92FF920F931F93A0
:10564000CF93DF931092F8041092F7042FE3209386
:10565000F6041092F5041092F4041092F3041092E0
:10566000EF041092F0041092F1041092F2049C01E5
:10567000F90190812F5F3F4F9032D1F39E34C9F4EE
:10568000818190ED980F9A3020F08D3211F08B329D
:1056900081F432969F012F5F3F4F808180538A3083
:1056A00008F47BC09F012F5F3F4F8081803209F457
:1056B00076C0F0935308E09352088F010F5F1F4F9D
:1056C000C0816AE270E0C8010F94BD5C009731F0C0
:1056D000FC01319780818032E1F31182CD3429F0D1
:1056E000C43519F0C73409F04BC0F80180810F5F51
:1056F0001F4F8032D1F380538A3008F041C0C093ED
:10570000F60430E020E04AE0DF011196429FC0013C
:10571000439F900D11249C01205331098081280F53
:10572000311D87FD3A95818190ED980F9A30C8F12F
:105730003093F5042093F4048E3261F4329690E0B5
:105740004AE0DF0131968C9150ED580F5A3058F1F4
:105750009093F304CD01DC0101964C914032D9F3D2
:10576000CD3489F52E31310539F018F52731310561
:1057700019F02C31310539F5B093F804A093F704F2
:10578000DF91CF911F910F91FF90EF90DF90CF901D
:10579000BF90AF909F908F900895F9017BCFF90152
:1057A00081CFFD01B1CF949F800D112490ED980F12
:1057B000C8CF2537310538F027373105E8F2203AD0
:1057C00083E03807C9F2D091520840E050E0BA01B6
:1057D00010E000E0C12CD12C7601C394FD0131967C
:1057E0008C91882309F47FC08132E1F4CD34D1F467
:1057F00020323105B9F44093EF045093F0046093E4
:10580000F1047093F204F093F804E093F70463E278
:1058100070E0CF010F94BD5C009709F4B1CFFC019B
:105820001082AECF81548A3108F058C0DF019D91BB
:10583000903291F0A0EDA90FAA30E8F09E3271F4F9
:10584000918190539A30B8F00115110519F48F0128
:105850000150110990E013C0FD01E8CF9D3211F015
:105860009B3291F79181A0EDA90FAA3020F09E32D2
:1058700059F79281E6CF9E2F9D1B309759F3A82FA1
:10588000B0E04601570104C0880C991CAA1CBB1C3F
:105890008A95D2F7482959296A297B29AB52BB4FEF
:1058A0009C9380818154DF018A3108F497CFDF0116
:1058B0008191882309F492CF90ED980F9A30B8F334
:1058C00093ED980F923098F38B3289F3CD010196C6
:1058D000EC91E03209F082CFDC01F8CF011511051F
:1058E00001F78D01DECF1093F8040093F704409385
:1058F000EF045093F0046093F1047093F20440CFEE
:105900009B01AC01485F5F4FBC016C5F7F4F0C9403
:105910002B240F931F93CF93DF9300D000D01F92BF
:105920001F92CDB7DEB7FC018B0183A5811112C098
:1059300081E083A784819581A681B781B05889834E
:105940009A83AB83BC83BE016F5F7F4F85E398E092
:105950000E94802C1D821E821F82188620E030E06B
:1059600040E05FE36091A5107091A6108091A710B0
:105970009091A8100F946F5969837A838B839C83CD
:105980009E012B5F3F4FAE014F5F5F4F61EA70E1B9
:105990008DE990E10E942B241D821E821F821886B1
:1059A00020E030E040E05FE3F801608571858285AA
:1059B00093850F946F5969837A838B839C83B80195
:1059C0006C5F7F4F9E012B5F3F4FAE014F5F5F4F7C
:1059D000C8010E942B2428960FB6F894DEBF0FBE94
:1059E000CDBFDF91CF911F910F9108952F923F92DC
:1059F0004F925F926F927F928F929F92AF92BF92DF
:105A0000CF92DF92EF92FF920F931F93CF93DF938A
:105A1000CDB7DEB7A2970FB6F894DEBF0FBECDBFED
:105A20008C011B015E834D8340909D1050909E1011
:105A300060909F107090A0108090A1109090A21084
:105A4000A090A310B090A410DB018D919D910D90BA
:105A5000BC91A02D8F87988BA98BBA8B9C01AD012F
:105A6000C301B2010F946E596B017C01D1011496F0
:105A70008D919D910D90BC91A02D8B8B9C8BAD8BAE
:105A8000BE8B9C01AD01C501B4010F946E596F8BA3
:105A9000788F898F9A8FAD81BE818D919D910D9068
:105AA000BC91A02D8F839887A987BA879C01AD01EF
:105AB000C301B2010F946E596B8F7C8F8D8F9E8FB7
:105AC000AD81BE8114968D919D910D90BC91A02DBC
:105AD0008B879C87AD87BE879C01AD01C501B40152
:105AE0000F946E596F8F78A389A39AA3A70196018B
:105AF000C701B6010F94E3526B017C012F89388DE9
:105B0000498D5A8DCA01B9010F94E3529B01AC0132
:105B1000C701B6010F946F594B015C012F8538897D
:105B200049895A896F81788589859A850F946E593C
:105B30002B013C012B893C894D895E896B857C85D5
:105B40008D859E850F946E596B017C01A301920196
:105B5000C301B2010F94E3522B013C01A70196014E
:105B6000C701B6010F94E3529B01AC01C301B2011E
:105B70000F946F590F941D5C6B017C012B8D3C8D34
:105B80004D8D5E8DCA01B9010F94E3522B013C018A
:105B90002F8D38A149A15AA1CA01B9010F94E3522E
:105BA0009B01AC01C301B2010F946F599B01AC0181
:105BB000C501B4010F94CF5B1816B4F520E030E0B6
:105BC000A901C701B6010F94CF5B87FF2AC0C701A7
:105BD000B601905820E030E040EA50E40F94CF5BEB
:105BE000181614F5A1016D817E81C8010E94F62C62
:105BF000A2960FB6F894DEBF0FBECDBFDF91CF9156
:105C00001F910F91FF90EF90DF90CF90BF90AF90DA
:105C10009F908F907F906F905F904F903F902F90CC
:105C20000895C701B601D6CF20E030E040E050E44F
:105C3000C501B4010F94CF5B181624F4B101C8015B
:105C40000E94892C19821A821B821C82BE016F5FFE
:105C50007F4FC1010E94802C2DEC3CEC4CEC5CE3AE
:105C6000C701B6010F94E3529B01AC01F8016081BA
:105C70007181828193810F94E35269837A838B834C
:105C80009C83C8010F945F2EBE016F5F7F4F8D8193
:105C90009E810E94802CACCF4F925F926F927F9238
:105CA0009F92AF92BF92CF92DF92EF92FF920F93AB
:105CB0001F93CF93DF93CDB7DEB768970FB6F894F5
:105CC000DEBF0FBECDBFFB019080342F390D3530C4
:105CD00008F026C1E180022F0E0D053008F020C12A
:105CE000EE2DF0E0EA54FB4F4080512C712C612CDA
:105CF000092C04C076946794579447940A94D2F779
:105D000040FE0EC110E0F801EA54FB4F4080512CD8
:105D1000712C612CC32ED12C04C0769467945794B7
:105D200047943A95D2F740FEFBC0F22E642F5C01F7
:105D3000660F770B072E000C880B990B0F9484527B
:105D40002B013C01892D94E08902F0011124EE55CC
:105D5000F94EA301920160817181828193810F9438
:105D60006F596D877E878F87988BF601EE0FFF1F27
:105D7000EE0FFF1FEE55F94EA30192016081718174
:105D8000828193810F946E5969837A838B839C837C
:105D90006F2D660F770B072E000C880B990B0F9455
:105DA00084522B013C018E2D94E08902F0011124D4
:105DB000E257F94EA3019201608171818281938142
:105DC0000F946F59698B7A8B8B8B9C8B000F111FF3
:105DD000000F111FF801E257F94EA30192016081F3
:105DE0007181828193810F946E596D837E838F833D
:105DF0009887F50180859185A285B38589879A87E3
:105E0000AB87BC878D8B9E8BAF8BB88F4FEE50E0EE
:105E100061E070E0CE0141960E94ECD54FEE50E07B
:105E200061E070E0CE0105960E94ECD54FEE50E0A7
:105E300061E070E0CE010D960E94ECD54FEE50E08F
:105E400061E070E0CE0101960E94ECD5C988DA8845
:105E5000EB88FC8827E137EB41ED58EBC701B60131
:105E60000F94CF5B87FD5CC027E030E040E753E450
:105E7000C701B6010F947D5218160CF451C0CD84A1
:105E8000DE84EF84F88827E137EB41ED58EBC7015A
:105E9000B6010F94CF5B87FD43C027E030E040E7B9
:105EA00053E4C701B6010F947D521816CCF1CD8092
:105EB000DE80EF80F88427E137EB41ED58EBC70136
:105EC000B6010F94CF5B87FD2BC027E030E040E7A1
:105ED00053E4C701B6010F947D5218160CF1C98026
:105EE000DA80EB80FC8027E137EB41ED58EBC7010E
:105EF000B6010F94CF5B87FD13C027E030E040E789
:105F000053E4C701B6010F947D5218164CF0AE0150
:105F10004F5F5F4FBE01635F7F4FC5010E94F62C4C
:105F200068960FB6F894DEBF0FBECDBFDF91CF915C
:105F30001F910F91FF90EF90DF90CF90BF90AF90A7
:105F40009F907F906F905F904F9008958C3891054F
:105F500014F08CE890E090937208809371080C9490
:105F600041C60E94712597FD0CC00E9471256F3FAC
:105F700071058105910509F034F40E947125862F81
:105F8000089580E008958FEF08958091BF04909167
:105F9000C004892B41F00E94B12F91E0811101C012
:105FA00090E0892F089591E0FCCF0E947125CB01EC
:105FB00008950F931F93CF938091BF049091C004D5
:105FC0000097E9F0FC018F01C1912C2F2F7D81F00A
:105FD000C53411F0C536B9F7F801108270E060E001
:105FE0000F940C4EF801C083CF911F910F9108952B
:105FF00070E060E0CF911F910F910D940C4E60E026
:1060000070E0CB01F1CF2FEB280F2A3108F047C009
:10601000E22FF0E08091EF049091F004A091F10460
:10602000B091F20404C0B695A795979587952A95E7
:10603000D2F780FD02C081700895EB52FB4FE081E2
:10604000EE2341F18091520890915308E80FF92F07
:10605000F11D808190ED980F9A3030F08E3251F41E
:10606000818180538A3098F4F093C004E093BF0498
:1060700081E008958D3211F08B3249F4818190EDE9
:10608000980F9A3088F38E3211F48281EACFF0E0D3
:10609000E0E0EACF1092C0041092BF04E9CF80E0A4
:1060A00008950E940330882341F081E02091BF04CD
:1060B0003091C004232B09F480E00895CF93DF933F
:1060C000EB010E945130882319F00E947125EB01E9
:1060D000CE01DF91CF910895CF92DF92EF92FF92A0
:1060E0006A017B010E945130882331F0FF90EF90CC
:1060F000DF90CF900C94D92FC701B601FF90EF909D
:10610000DF90CF9008954F925F926F927F928F921F
:106110009F92AF92BF92CF92DF92EF92FF921F9326
:10612000CF93DF9300D01F92CDB7DEB719821A82CA
:106130001B821C82CE0101964C018DE9C82E80E1A4
:10614000D82E95E3E92E98E0F92E2FE4A22E29E02F
:10615000B22E10E088E5810F0E945130F401819346
:106160004F01882341F00E94D92F2B013C018091DF
:106170005210882359F0F60180819181A281B38168
:10618000F70180839183A283B38314C0812F0E947F
:106190009621882309F4D0C0F60120813181428103
:1061A0005381C301B2010F946F59F701608371836A
:1061B000828393831F5FF4E0CF0ED11C84E0E80E4E
:1061C000F11C94E0A90EB11C133021F685E40E9465
:1061D00051308C83882309F4B9C00E94D92F6B01F8
:1061E0007C0183E00E949621882371F02091A91000
:1061F0003091AA104091AB105091AC10C701B6017C
:106200000F946F596B017C01C0924108D0924208F3
:10621000E0924308F09244088091CE05882359F11A
:106220008091C11682FF27C08C81882321F189814A
:10623000811103C08A818823F1F02DEC3CEC4CE401
:106240005DE36091A6087091A7088091A8089091DD
:10625000A9080F946F599B01AC016091A510709132
:10626000A6108091A7109091A8100F94CF5B1816DC
:1062700014F40F94C23F40E050E0BA0186E40E945B
:106280006C3020E030E0A9010F94CF5B181684F445
:106290000E94D92F20E030E040E752E40F94695A81
:1062A0006093790270937A0280937B0290937C02D0
:1062B0008091531083FD2CC080915210811128C011
:1062C0008091AF07882321F12091A9103091AA1065
:1062D0004091AB105091AC10609141087091420810
:1062E00080914308909144080F946E592091BC0707
:1062F0003091BD074091BE075091BF070F946F5971
:106300006093BC077093BD078093BE079093BF074F
:106310000F900F900F900F90DF91CF911F91FF90F2
:10632000EF90DF90CF90BF90AF909F908F907F9035
:106330006F905F904F900895F501208131814281E7
:106340005381C301B2010F946E592FCF8091A910D0
:106350009091AA10A091AB10B091AC10809341081D
:1063600090934208A0934308B093440855CFCF932D
:10637000DF93EB010E945130882321F0DF91CF9110
:106380000C94D52FCE01DF91CF910895CF93DF9359
:10639000C82FD62F0E945130882321F0DF91CF9152
:1063A0000C94C52F8C2F0E940330811101C08D2FBA
:1063B000DF91CF910895EDE9F8E082EBDF011D92C6
:1063C0008A95E9F708958091CE05811104C00E9455
:1063D000DB310D9487418091C11682FD0D94C23F3F
:1063E000089580919D08882361F090914E0989134A
:1063F00008C08091C11683FF04C08BED98E00D9416
:10640000924180E00895FC01238121110C9406D271
:106410000895CF92DF92EF92FF920F931F93CF9345
:1064200090912402913009F461C0662351F01092DA
:10643000A20410929E0410929F041092A004109245
:10644000A104C82F0F944335C0909E04D0909F04A0
:10645000E090A004F090A1049B01AC012C193D092F
:106460004E095F0969017A01F7FC40C02091A2043E
:10647000C7FD15C04C2F0C2E000C550B4C5F5F4F09
:10648000E22F022E000CFF0B4E175F077CF144EF4A
:10649000C42EDD24D394E12CF12C2C1734F438EEE7
:1064A000C32E33E0D32EE12CF12CC60ED71EE81EEE
:1064B000F91EC0929E04D0929F04E092A004F09234
:1064C000A104022F017010E084E2809FB001819F3F
:1064D000700D701B112460597C4F82E390E00E9484
:1064E0001E7D8091A2048F5F8093A204CF911F91A3
:1064F0000F91FF90EF90DF90CF9008950F931F932F
:1065000001E010E020E030E0082E04C0000F111F71
:10651000221F331F0A94D2F74091030550910405BE
:106520006091050570910605402B512B622B732B52
:106530004093030550930405609305057093060589
:1065400090912302891303C081E0809352101F9120
:106550000F9108951092330610923406109235066A
:1065600010923606EFECF5E084E6DF011D928A9585
:10657000E9F7089590919C109817B1F00E94C6DC3D
:1065800080919C10882341F08DE990E10E94E9DC24
:1065900010929C100C9461F281E080939C108DE924
:1065A00090E10E941BDCF6CF08954F925F926F92AC
:1065B0007F928F929F92AF92BF92CF92DF92EF9293
:1065C000FF921F93CF93DF93EC01162F2091670862
:1065D000309168084091690850916A086881798112
:1065E0008A819B810F947D52882309F4AEC0B090BC
:1065F0009C1080E00E94BA32C880D980EA80FB807B
:1066000020E030E0A901C701B6010F94CF5B181656
:106610001CF0C12CD12C7601C0926708D09268087A
:10662000E0926908F0926A082DEB37E346E855EBF3
:10663000C701B6010F94CF5B87FD0BC02DEB37E38D
:1066400046E855E3C701B6010F947D5218160CF0C9
:1066500078C0A701960160E070E080E89FE30F94A6
:10666000695A6093B2057093B3058093B405909313
:10667000B50580EF9FEFA9E7B4EC8093B605909342
:10668000B705A093B805B093B905BB2009F45DC068
:1066900040909D1050909E1060909F107090A010A0
:1066A0008090A1109090A210A090A310B090A41080
:1066B000C090A510D090A610E090A710F090A81060
:1066C00081E00E94BA32112309F43FC020919D104D
:1066D00030919E1040919F105091A010C301B201C3
:1066E0000F947D5281111CC02091A1103091A210F5
:1066F0004091A3105091A410C501B4010F947D5294
:1067000081110EC02091A5103091A6104091A710C4
:106710005091A810C701B6010F947D528823A9F0AB
:10672000DF91CF911F91FF90EF90DF90CF90BF90BE
:10673000AF909F908F907F906F905F904F900C9450
:1067400009FB60E070E0CB018CCFDF91CF911F910E
:10675000FF90EF90DF90CF90BF90AF909F908F9081
:106760007F906F905F904F900895EF92FF920F93FC
:106770001F93CF93DF930FEC15E0C5E07801D5E0D0
:10678000F70161917191819191917F0120E030E059
:10679000A9010F947D5281110EC0D15089F7C150CB
:1067A0000C5E1F4FC111EACFDF91CF911F910F9166
:1067B000FF90EF90089581E0F7CFEFE6F0E0808161
:1067C0008260808308958091490890914A08892BBE
:1067D00079F48091490890914A08892B49F42091D5
:1067E000490830914A0881E0232B19F480E008958C
:1067F00081E00895CF92DF92EF92FF926B017C01CE
:1068000083E3C816D104E104F10470F082E3C81AEE
:10681000D108E108F10862E370E080E090E00F94B5
:1068200010350E9463F2ECCFC701B6010F9410350A
:10683000FF90EF90DF90CF900C9463F280914E0622
:1068400081110AC080916508813041F08091C116A4
:1068500082FB882780F9089580E0089581E00895FB
:106860005F9A8091C3078E7F8093C3078A9A809135
:10687000C3078D7F8093C307809108018095817045
:10688000809306018091C3078B7F8093C3070C948C
:10689000B0219091C11693FB882780F993FF06C021
:1068A00081E090912918911101C080E008958091B4
:1068B0004E06811110C080916508823061F00E94FF
:1068C0004934882349F08091C11682FB882780F9DA
:1068D00091E08927089581E008950E94573481113D
:1068E0000DC0109203051092040510920505109238
:1068F0000605109207058FEF0E94B2230C9446FE06
:10690000EDE8F9E010821182089581E008958F92F8
:106910009F92AF92BF92CF92DF92EF92FF920F932E
:10692000CF93DF931F92CDB7DEB75C017B014901A6
:106930006B01C40ED51EF501808191810F949B5887
:106940008983002311F0F7018083BE016F5F7F4FC1
:10695000C4010F945325F5018081918101969183A3
:106960008083FFEFEF1AFF0AEC14FD0421F780E0AB
:106970000F90DF91CF910F91FF90EF90DF90CF902C
:10698000BF90AF909F908F9008959091C00095FF19
:10699000FCCF8093C6000895CF93DF93EC018991DB
:1069A000882319F00E94C534FACF8DE00E94C534C7
:1069B0008AE0DF91CF910C94C534CF92DF92EF92B1
:1069C000FF92CF936B017C01C42F4A3069F4F7FE2C
:1069D0000BC0F094E094D094C094C11CD11CE11C75
:1069E000F11C8DE20E94C5344C2FC701B601CF9136
:1069F000FF90EF90DF90CF900D94243FCF93DF93E3
:106A0000EC01FE0184912196882319F00E94C5347F
:106A1000F8CFDF91CF9108950F931F93CF938C01FF
:106A2000C62F85E392E10E94FE34C8010E94FE3425
:106A30008AE30E94C53480E38C0F0E94C5348AE04B
:106A4000CF911F910F910C94C53488EB93E10E9474
:106A5000FE3460E088EA93E10E940C3560E083E94F
:106A600093E10E940C3561E08CE893E10E940C35C3
:106A700061E081E893E10E940C3561E081E793E1F8
:106A80000E940C3560E088E693E10E940C3561E0DD
:106A90008EE593E10E940C3560E084E593E10E946D
:106AA0000C3560E08DE493E10E940C3560E085E4F4
:106AB00093E10E940C3561E087E393E10E940C357D
:106AC00061E089E293E10E940C3560E08AE193E1A4
:106AD0000E940C3560E08CE093E10E940C3560E090
:106AE00086EF92E10E940C3561E085EE92E10E9412
:106AF0000C3561E086ED92E10E940C3561E08FEC8F
:106B000092E10E940C3560E088EC92E10E940C3525
:106B100061E08FEB92E10E940C3561E08AEA92E13C
:106B20000E940C3561E08CE992E10E940C3561E035
:106B300089E892E10E940C3560E08CE792E10E94C6
:106B40000C3561E087E792E10E940C3561E08AE64E
:106B500092E10E940C3560E086E592E10E940C35DE
:106B600060E083E492E10E940C3560E085EC96E100
:106B70000E949321682F61708AE392E10C940C3596
:106B80000E94C53485EF9CE00C94FE340F931F9354
:106B9000CF938C01C62F84E799E00E94FE34C80190
:106BA0000E94FE34CC2331F08AE0CF911F910F91E7
:106BB0000C94C534CF911F910F91089560E084E249
:106BC00090E40E94C63584E899E00E94FE348AE091
:106BD0000C94C534EF92FF920F931F93CF937C01D7
:106BE0008B01C42F60E084E290E40E94C635C701A7
:106BF0000E94FE3480E20E94C534C8010E94FE3427
:106C0000CC2319F08C2F0E94C5348AE0CF911F91BC
:106C10000F91FF90EF900C94C534DF92EF92FF92AA
:106C20000F931F93CF93DF93D82E7B018A01E90145
:106C30000E94DE35D0924D0840E0B70188E390E431
:106C40000E94EA350115110531F040E0B80181E3F9
:106C500090E40E94EA35209731F040E0BE0181E3E4
:106C600090E40E94EA3560E084E290E40E94C63538
:106C70008CE290E40E94FE348AE0DF91CF911F9174
:106C80000F91FF90EF90DF900C94C53461E08EE798
:106C900099E00C94C635AF92BF92CF92DF92EF92FB
:106CA000FF920F931F93CF93DF9389E499E00E94A3
:106CB000FE346091330670913406809135069091D0
:106CC000360645E00F948C0786E399E00E94FE3477
:106CD000C0E0D9E0D15021F080E20E94C534FACF63
:106CE0008C2F0F948B3FCF5FC53099F78AE00E94BD
:106CF000C5340FEC15E0C0E080E20E94C5348C2F53
:106D00000F948B3F5801D5E080E20E94C534F50115
:106D1000C080D180E280F380A7019601C701B6014F
:106D20000F94615C81112CC020E030E0A901C70103
:106D3000B6010F94CF5B87FD03C08BE20E94C53480
:106D400045E0C701B6010F948C07D15084E1A80E2D
:106D5000B11CD111D9CF8AE00E94C534CF5F0C5F3E
:106D60001F4FC53049F68AE0DF91CF911F910F91F7
:106D7000FF90EF90DF90CF90BF90AF900C94C53410
:106D8000F12C80E20E94C534F3948DE3F8E0FF1209
:106D9000F9CFDBCF811107C083E39EE00E94FE3470
:106DA0008AE00C94C53487E39EE0F8CFCF93DF935D
:106DB000EB010E94FE34CE01DF91CF910D94923F02
:106DC000CF93C62F0E94FE348C2FCF910D948B3F12
:106DD000CF92DF92EF92FF926A017B010E94FE3414
:106DE00042E0C701B601FF90EF90DF90CF900D9485
:106DF0008C07CF92DF92EF92FF926A017B010E9493
:106E0000FE344AE0C701B601FF90EF90DF90CF90CB
:106E10000C94DD342F923F924F925F926F927F924B
:106E20008F929F92AF92BF92CF92DF92EF92FF929A
:106E30000F931F93CF93DF93CDB7DEB7C654D1091D
:106E40000FB6F894DEBF0FBECDBF70E060E085E402
:106E50000E94B731182F8F3F09F483C08823E9F0CF
:106E600083E796E1CA5BDF4F0FB6F894DEBF0FBE33
:106E7000CDBFDF91CF911F910F91FF90EF90DF90E9
:106E8000CF90BF90AF909F908F907F906F905F90CA
:106E90004F903F902F900C94FE3424EB30E03A83D7
:106EA000298383E50E945130882321F00E94D52F49
:106EB0009A83898365E070E083E40E94B7318AA7F2
:106EC00060E085E50E94C63125968FAF259760E08A
:106ED00086E696E10E9454B2A981BA81BD01BB0F3A
:106EE000880B990B0F9484526D837E838F83279632
:106EF0009FAF27970F944335688B798B8A8B9B8B39
:106F00001F3F09F045C420E030E04CE053E46D81C0
:106F10007E818F8127969FAD27970F94CF5B1816A0
:106F20000CF0AAC18BE396E10E94FE34CA5BDF4FEE
:106F30000FB6F894DEBF0FBECDBFDF91CF911F918A
:106F40000F91FF90EF90DF90CF90BF90AF909F9008
:106F50008F907F906F905F904F903F902F900D9407
:106F6000824246E450E05A8349839BCF1FAEAFC1B3
:106F70002496EEADFFAD2497808383C2FBEE4F2EA7
:106F8000512C612C712C04C384E190E0A0E0B0E0AE
:106F90008C8B9D8BAE8BBF8BE4E14E2E512C612CE4
:106FA000712C04C34C8A5D8A6E8A7F8AFFC2249644
:106FB000EEADFFAD24978083D4C389819A81AB81E4
:106FC000BC8129A93AA94BA95CA9821B930BA40BEC
:106FD000B50BB7FD59C08FAD0F9430088AE00E9401
:106FE000C53489819A81AB81BC818053984FAF4F62
:106FF000BF4F89AB9AABABABBCAB9DA9911177C02E
:107000002EA93FA948AD59ADB101802F26969FAD5D
:1070100026970F94CF5B18160CF053C020E030E099
:1070200040E050E4B101802F26969FAD26970F9443
:107030006F596EAB7FAB88AF99AF2CA53DA54EA520
:107040005FA589819A81AB81BC81280F391F4A1FB6
:107050005B1F2AAF3BAF4CAF5DAF20E030E040ECB0
:1070600050E46D817E818F8127969FAD27970F9485
:107070006E599101402F26965FAD26970F947D5251
:10708000881F8827881F8DAB88899989AA89BB8921
:10709000C816D906EA06FB0610F4D701C6012981F5
:1070A0003A814B815C81281B390B4A0B5B0BDA015F
:1070B000C90181389F44A241B105A8F187E895E153
:1070C0000EC289819A81AB81BC812AAD3BAD4CADAA
:1070D0005DAD821B930BA40BB50B4DE156E36CE247
:1070E00076E3B7FDD1CF812F0E942ED6CDCF20E001
:1070F00030E040EF51E46D817E818F8127969FAD16
:1071000027970F946E599B01AC01B101802F2696F1
:107110009FAD26970F947D5287FFB6CF49EC56E37B
:1071200069ED76E3E0CF4AA55BA5888D998D481778
:1071300059070CF09EC003970CF49BC08AE295E1BE
:107140000E94FE341F3F09F076C0AAE1B5E1BA8380
:10715000A98389E095E10E94FE3489819A810E9489
:10716000FE34488559856A857B8586E295E10E94D3
:10717000E8368AE00E94C53489E095E10E94FE3439
:1071800089819A810E94FE3449A15AA16BA17CA1F8
:1071900082E295E10E94E8368AE00E94C53489E0E7
:1071A00095E10E94FE3489819A810E94FE34B501E6
:1071B000A4018EE195E10E94E8368AE00E94C53480
:1071C0002596FFAD2597FF2391F12CEA35EC47E298
:1071D0005EE369A17AA18BA19CA10F94E3526B019C
:1071E0007C012CEA35EC47E25EE3C501B4010F9463
:1071F000695A288539854A855B851F3F09F52093A3
:107200007408309375084093760850937708C092BD
:107210007808D0927908E0927A08F0927B0860931F
:107220007C0870937D0880937E0890937F0881E0AE
:10723000809362027BCEEEE6FFE3FA83E98389CF97
:107240002093D8153093D9154093DA155093DB1558
:10725000C092DC15D092DD15E092DE15F092DF15BC
:107260006093E0157093E1158093E2159093E31518
:10727000DECF0E945EB680C087E296E10E94FE34B7
:107280000E9421D58FE78093730824EB30E0A8EEAD
:10729000B3E00F9415596CA77DA78EA79FA72889E7
:1072A00039894A895B89260F371F481F591F2AAF22
:1072B0003BAF4CAF5DAF1092620281E080937102F0
:1072C00032E0310F3EAF323008F450CE1FAFC888E5
:1072D000D988EA88FB88C9AADAAAEBAAFCAA812C79
:1072E000912C540189A29AA2ABA2BCA2888699864D
:1072F000AA86BB868FE790E0A0E0B0E08C8B9D8BE8
:10730000AE8BBF8B1C8690E49A8FACE1AB8FB6E45A
:10731000BC8F1D8E1E8E1F8E18A23FE7432E512C50
:10732000612C712C1DAA8EAA9FAAA8AEB9AE1EA26E
:107330001FA218A619A6E1E0EDA3198E188E212C24
:10734000312C00E026961FAE2697F5E11F02C00102
:1073500011249C0121533A4E22963FAF2EAF229723
:10736000285F3F4F24963FAF2EAF24974AA5042EA7
:10737000000C550B5BA74AA780917102882309F482
:10738000B0C00F94433569837A838B839C8350917B
:107390004C0658AB552309F48BC00E94D4D560919C
:1073A0006F08709170081F3F39F02296AEADBFADE7
:1073B000229714966D917C91072E000C880B990BE7
:1073C0000F9484521B01082F26969FAF26972D8D70
:1073D0003E8D4F8D58A126969FAD26970F94CF5B7B
:1073E00018163CF42D8E3E8E0F8F2696BFAD269735
:1073F000B8A32C853A8D4B8D5C8DB101802F2696DC
:107400009FAD26970F947D5287FF07C02C863A8E3A
:107410000B8F2696EFAD2697EC8FFDA19101402FA3
:1074200026965FAD26976D817E818F8127969FADD1
:107430002797FF2309F45AC00F947D5287FF38C065
:1074400049815A816B817C814C195D096E097F09E4
:10745000DB01CA0188589341A109B109B7FD28C0D1
:107460008C899D89AE89BF8984199509A609B709B8
:10747000B595A795979587951F3F09F079CD80938E
:1074800073084EA35FA368A779A7FD81FD8F2E81A6
:107490002E8F3F813F8F27964FAD279748A3898135
:1074A0009A81AB81BC81888B998BAA8BBB8B1DA2E7
:1074B00020E030E040EF51E46D817E818F8127969E
:1074C0009FAD27970F946F599101402F26965FAD7E
:1074D00026970F947D5287FF70CD85EA95E10E9433
:1074E000FE34109271020E9421D5A1CE0F94CF5B81
:1074F0001816F4F689819A81AB81BC812889398973
:107500004A895B89821B930BA40BB50BAC01BD01AF
:10751000485853416109710977FDCACF488D598D8B
:10752000452B09F40DC1CEA0DFA0E8A4F9A4C80E34
:10753000D91EEA1EFB1E2EA13FA148A559A5281B56
:10754000390B4A0B5B0BC301B2010F94B158A70171
:1075500096010F94E3584C885D886E887F88420EB0
:10756000531E641E751E54E14516510461047104D6
:107570000CF40ACD8CEE48165104610471040CF031
:10758000FDCC90E849165104610471040CF40ACD55
:107590004C8A5D8A6E8A7F8A2EEF30E040E050E0B0
:1075A000241935094609570929013A014C895D8991
:1075B0006E897F898FE196E10E94F936B301A201BD
:1075C0008AE196E10E94F9364C855A8D6B8D7C8D4F
:1075D00083E196E10E94E8364D8D5E8D6F8D78A136
:1075E0008CE096E10E94E836A88DB98D13970CF4D3
:1075F000A7C0C301B2010F94845220E030E040E8FC
:1076000050E40F94E3524B015C012C853A8D4B8D75
:107610005C8D6D8D7E8D8F8D98A10F946E592BEDA5
:107620003FE049E450E40F94E35220E030E040E0D2
:107630005FE30F94E3529B01AC01C501B4010F94C9
:10764000695A6C877D878E879F87C701B6010F9423
:1076500084522FE632E143E85AE30F94E3526B0180
:107660007C011E3F59F02AE939E949E15FE3812CA9
:10767000912CA12C6EE3B62E1F3F59F42DEC3CEC5F
:107680004CE45EE37BEA872E7AEA972EA92C7EE310
:10769000B72E6C857D858E859F850F94E352688714
:1076A00079878A879B879B01AC010F946F59A7014B
:1076B00096010F94695A69A37AA38BA39CA328858A
:1076C00039854A855B85C701B6010F94E352A50150
:1076D00094010F94E3524B015C014C855D856E85EE
:1076E0007F8586E096E10E94E836B701A60180E03A
:1076F00096E10E94E8368AE00E94C534BEAD81EF73
:1077000095E1B23010F082EE95E10E94FE3448859A
:1077100059856A857B858CED95E10E94E83649A103
:107720005AA16BA17CA186ED95E10E94E836B501D6
:10773000A40180ED95E10E94E8368AE00E94C534FC
:107740008C899D89AE89BF89840D951DA61DB71DA5
:10775000B595A795979587951F3F09F028CC8093FD
:107760007308288D398D2F5F3F4F398F288F3D81CA
:107770003C874E814A8F5F815B8F27968FAD27971D
:107780008C8FC980DA80EB80FC8098A99DA390CE75
:10779000E12E012E000CFF08F70183E0EE0FFF1F22
:1077A0008A95E1F7E759FD4F668177816F5071093E
:1077B000072E000C880B990B0F9484529B01AC018F
:1077C0006D817E818F8127969FAD27970F94CF5B28
:1077D00018160CF4A7CB87E296E10E94FE340E94B3
:1077E00021D585E18E9DF0018F9DF00D1124E1538F
:1077F000FA4E8FE7808722E330E049CDCF93DF93C5
:10780000EB010E94FE34CE01DF91CF910D940A2747
:107810002F923F924F925F926F927F928F929F92A0
:10782000AF92BF92CF92DF92EF92FF920F931F938E
:10783000CF93DF93CDB7DEB7C058D1090FB6F89418
:10784000DEBF0FBECDBF80E89CE00E94FE340F94E7
:10785000A44281118FC084E50E945130882329F011
:107860000E94D52F81110E94D7D480E090E0A0E83B
:10787000BFE389839A83AB83BC838D839E83AF836D
:10788000B8878DEC9CECACE4BEE389879A87AB8724
:10789000BC8780E090E0A0E2B1E48D879E87AF874F
:1078A000B88B8CE390E09A8B898B8DEC90E09C8B6D
:1078B0008B8B8DEC9CECACECBEE38D8B9E8BAF8BFD
:1078C000B88F80E090E0A0EEBFE3898F9A8FAB8FF6
:1078D000BC8F1BA61CA64AE959E969E97EE38FE43F
:1078E0000E946C306D8F7E8F8F8F98A360E083E451
:1078F0000E94C63189A360E08BE40E94C6318AA34E
:1079000089E40E94513010E0F12CE12C8823C1F071
:107910000E94B12F90E01816190614F481E090E04F
:1079200011E0180F212F2150330BC90126E0289FA9
:10793000F001299FF00D1124E75FF74FE280F380FB
:1079400082E40E945130882319F00E94D52F7C01D7
:10795000E114F10459F1C70188978536910520F1AA
:107960006CE870E082E59CE00E94FE3B8DE49CE0C8
:107970000E94FE34C058DF4F0FB6F894DEBF0FBE32
:10798000CDBFDF91CF911F910F91FF90EF90DF90CE
:10799000CF90BF90AF909F908F907F906F905F90AF
:1079A0004F903F902F900895FA8AE98A8CE40E94C4
:1079B00051308823E1F00E94D92F6B017C01C986E8
:1079C000DA86EB86FC8620E030E0A9010F94CF5BDD
:1079D00087FD0AC020E030E040E050E4C701B60176
:1079E0000F947D5218161CF485E29CE0C1CF81E50E
:1079F0000E940330882331F18091BF049091C0042C
:107A0000892BE9F00E94D92F6B017C01CD82DE82A7
:107A1000EF82F8862DEC3CEC4CE45DE30F94CF5BF9
:107A200087FD0AC020E030E040E751E4C701B6011D
:107A30000F947D52181634F484EF9BE099CF89ECB3
:107A40009BE096CF83E50E9451308823E9F00E94A5
:107A5000D92F6B017C01CD8ADE8AEF8AF88E2DEC5E
:107A60003CEC4CEC5DE30F94CF5B87FD0AC020E05B
:107A700030E040E050E4C701B6010F947D52181683
:107A80001CF482EA9BE074CF80E50E9403308823D7
:107A900041F08091BF049091C004892B29F58FEFAC
:107AA0008BA786E40E945130882309F43DC00E94D0
:107AB000D92F6B017C01C98EDA8EEB8EFC8E20E013
:107AC00030E040E85FE30F94CF5B87FD0AC020E021
:107AD00030E040E850E4C701B6010F947D5218161B
:107AE0001CF581E59BE044CF8BA58F5F8BA70E949F
:107AF000D92F6B017C01CD86DE86EF86F88A20E0E7
:107B000030E0A9010F94CF5B87FD0BC020E030E08F
:107B100048EC51E4C701B6010F947D5218160CF0E1
:107B2000C0CF8AE79BE024CFC98CDA8CEB8CFC8C2D
:107B30008D889E88AF88B88CA7019601C701B601D1
:107B40000F94E3529B01AC0160E070E084E490E4A8
:107B50000F94695A29813A814B815C810F94E352D9
:107B60002B013C01A5019401C501B4010F94E3521E
:107B7000A70196010F94E3522CEE31E548EB5DE34B
:107B80000F94695A9B01AC01C301B2010F94E352F7
:107B900069837A838B839C83112309F1412F4150A0
:107BA000550B26E0249FF001259FF00D1124E75F7F
:107BB000F74F0081118188E40E945130882319F029
:107BC0000E94D52F8C010115110571F0C801855A4D
:107BD00091098F30914030F083E29BE0C9CE10E0F4
:107BE00000E0E9CF1C8B0B8B85E50E9403308823D6
:107BF000C9F00F944335611571058105910511F0A8
:107C00000F94034E8091BF049091C004892BC9F05A
:107C10000E94D92F6093BB047093BC048093BD0471
:107C20009093BE046AE170E082E50E94B731E59668
:107C30009FAF8EAFE5971816190644F08FEE9AE0C5
:107C400097CE60E070E088E492E4E4CF89E50E949A
:107C50005130882309F40AC10E94D92F2091530979
:107C60003091540940915509509156090F946E591D
:107C70004B015C0188E50E945130882309F4FFC064
:107C80000E94D92F20914F093091500940915109FC
:107C9000509152090F946E596B017C01CBA2DCA26A
:107CA000EDA2FEA28FA298A6A9A6BAA627E137EB5D
:107CB00041ED58EBC501B4010F94CF5B87FDE8C0DF
:107CC00027E030E040E753E4C501B4010F947D5252
:107CD00018160CF4DDC027E137EB41ED58EBC70176
:107CE000B6010F94CF5B87FDD3C027E030E040E7BB
:107CF00053E4C701B6010F947D5218160CF4C8C0A6
:107D000084E40E94033011E081270E94BA3280E0AF
:107D100090E0A0EAB0E48DA79EA7AFA7B8ABCE01D4
:107D20008D960F94042E80918408EC968FAFEC977B
:107D3000109284080E94C1C382E79AE00E94FE3438
:107D400089899A894A970CF0A6C063E68FE49AE085
:107D50000E9454B20F947C358B899C890E9448DC28
:107D600041E061E080E00F94280A882309F4A6C06E
:107D70000F9482420F947C351092A9101092AA1091
:107D80001092AB101092AC1089EA90E10E9460EE64
:107D90001BA5112309F4F5C020E030E040E751E4D1
:107DA0006091841070918510809186109091871059
:107DB0000F94695A21966CAF7DAF8EAF9FAF21971C
:107DC0001F3F09F0F9C481E08093000563E687EA6C
:107DD0009AE00E9454B268E873E182E090E00E9469
:107DE0001E7D80E1EDE9F0E1A5E3B8E001900D92A0
:107DF0008A95E1F7CE0101960F945F2EC12CD12C0C
:107E0000760180915F0982FDB1C068E873E182E08C
:107E100090E00E941E7D20E030E040E85EE360914B
:107E200041087091420880914308909144080F9452
:107E30006F59609341087093420880934308909370
:107E4000440820E030E040E85EE3C701B6010F944B
:107E50006F596B017C0120E030E84BE354E40F9450
:107E6000CF5B87FD73C01092000528C08090A110E1
:107E70009090A210A090A310B090A410FBCEC09040
:107E80009D10D0909E10E0909F10F090A01006CF13
:107E900085EC9AE06DCD63E682E69AE00E9454B2EA
:107EA0000F947C351093000589899A890E94A62F2A
:107EB00061E081E00F94A308811147CF6FEF89EB58
:107EC0009AE00E9454B28CA5811112C081E08CA767
:107ED0008D819E81AF81B885B0588DA79EA7AFA731
:107EE000B8ABBE01635D7F4F85E398E00E94802CB4
:107EF00080E090E0A0EAB0E480933D0890933E08D3
:107F0000A0933F08B09340081DA61EA61FA618AA5E
:107F1000BE01635D7F4F85E398E00E94802CEC9664
:107F20005FADEC97509384080E94C1C31092000586
:107F30008AA181111FCD10927208109271080E94BF
:107F400041C690E080E00E9448DC14CDCE01CD9681
:107F50000E9451F980E1EDE9F0E1A5E3B8E001907C
:107F60000D928A95E1F70E94C6DC4BCF0E9419B9A9
:107F700063E68AE99AE00E9454B20F947C3510922D
:107F80000005E6EBF4E085E0DF011D928A95E9F754
:107F900080E1EDE9F0E1A5E3B8E001900D928A956A
:107FA000E1F789859A85AB85BC8580933D089093E0
:107FB0003E08A0933F08B09340081DA61EA61FA62A
:107FC00018AABE01635D7F4F85E398E00E94802C74
:107FD000BE01635E7F4F85E398E00E94802C81E0C4
:107FE0008093000589A1882309F43CC420919D1049
:107FF00030919E1040919F105091A010AC962CAFE4
:108000003DAF4EAF5FAFAC978091A1109091A210A1
:10801000A091A310B091A410E0968CAF9DAFAEAF2D
:10802000BFAFE097A2EAB6E1A196BFAFAEAFA1970E
:10803000312C212CBFEF6C96BFAF6C97EFEFA4965D
:10804000EFAFA497FFEFE396FFAFE3972FE4EA9635
:108050002FAFEA9733ECEB963FAFEB9707E481E065
:1080600090E0A0E0B0E0022C04C0880F991FAA1F86
:10807000BB1F0A94D2F7C458DF4F88839983AA8321
:10808000BB83CC57D040A6EBB4E0E296BFAFAEAF17
:10809000E297EEE8F6E1A396FFAFEEAFA39710E00C
:1080A000C058DF4F2882C058D040E296AEADBFAD79
:1080B000E2978D91E296BFAFAEAFE29790E0B0E06D
:1080C000A0E0C458DF4F288139814A815B81CC57B9
:1080D000D04082239323A423B523892B8A2B8B2B77
:1080E00009F0E5C0A196AEADBFADA197CD90DD90F2
:1080F000ED90FC90A396AEADBFADA3972D913D91B1
:108100004D915C91A8962CAF3DAF4EAF5FAFA89755
:10811000A7019601AC966CAD7DAD8EAD9FADAC97D1
:108120000F946E592B013C01A8962CAD3DAD4EAD80
:108130005FADA897E0966CAD7DAD8EAD9FADE0973D
:108140000F946E594B015C01A3019201C301B2016E
:108150000F94E3522B013C01A5019401C501B40128
:108160000F94E3529B01AC01C301B2010F946F590C
:108170000F941D5C4B015C01A70196016BA17CA1D2
:108180008DA19EA10F946E596B017C01A8962CAD18
:108190003DAD4EAD5FADA8976FA178A589A59AA515
:1081A0000F946E592B013C01A7019601C701B6013E
:1081B0000F94E3526B017C01A3019201C301B20150
:1081C0000F94E3529B01AC01C701B6010F946F59A4
:1081D0000F941D5C20E030E040E751E40F94695AB1
:1081E000A50194010F946F596B017C018090BB0431
:1081F0009090BC04A090BD04B090BE0420E030E09C
:1082000040E85FE3C501B4010F94CF5B1816F4F4A6
:10821000C501B4010F94DB5A4B015C0160E070E0D2
:10822000CB01181419041A041B0434F40F94B44D30
:10823000A50194010F94E3580F9484529B01AC0163
:10824000B601C7010F946F596B017C01E3962FAD06
:10825000E397EA963FADEA97EB964FADEB97502F39
:10826000B601C7010F947D5287FF21C06C961FAFE6
:108270006C97C058DF4FB881C058D040A496BFAFAC
:10828000A497E696CFAEE697E796DFAEE797E89637
:10829000EFAEE897E996FFAEE997E396CFAEE397A6
:1082A000EA96DFAEEA97EB96EFAEEB970F2D1F5FE6
:1082B000A396EEADFFADA3973496A396FFAFEEAFB6
:1082C000A397153009F0F1CEFFEF2F1A3F0AA196C0
:1082D0002EAD3FADA1972C5F3F4FA1963FAF2EAF84
:1082E000A19735E02316310409F0B9CE6C964FAD55
:1082F0006C97E42FF0E0EA54FB4F208181E090E09E
:10830000A0E0B0E0A4960FACA49704C0880F991F1A
:10831000AA1FBB1F0A94D2F7822B8083A4965FAD5D
:10832000A49762965FAF629763964FAF6397E696A6
:108330008FADE697E7969FADE797E896AFADE897E4
:10834000E996BFADE99767968CAF9DAFAEAFBFAF73
:1083500067975F3F09F414C24F3F09F411C284E0EC
:108360004802F0011124E257F94E10810181328058
:10837000238027E137EB41ED58EB612F702F832DE0
:10838000922D0F94CF5B87FDFFC127E030E040E7DF
:1083900053E4612F702F832D922D0F947D52181668
:1083A0000CF4F2C1A4969FADA497A4E09A02F00148
:1083B0001124EE55F94EC080D180E280F38027E190
:1083C00037EB41ED58EBB601C7010F94CF5B87FD4A
:1083D000DBC127E030E040E753E4B601C7010F946A
:1083E0007D5218160CF4D0C120E030E040EA50E491
:1083F000B601C7010F946F59A0966FAFA097A296D0
:108400007FAFA297A5968FAFA597A9969FAFA99783
:10841000CB01A596AFADA597A996BFADA99721961B
:108420008CAF9DAFAEAFBFAF2197812F902FA32D03
:10843000B22D25968CAF9DAFAEAFBFAF2597A4965A
:10844000BFADA497B11150C26C96EFAD6C97E1111E
:1084500018C220E030E040EA50E4612F702F832DF5
:10846000922D0F946F59A4966FAFA497AD967FAFDE
:10847000AD97E1968FAFE197E3969FAFE3976C9648
:10848000FFAD6C97FF2309F4F1C26C963FAD6C977A
:10849000A096CFAEA097A296DFAEA297A596EFAE1C
:1084A000A597A996FFAEA99734300CF014C222ED1F
:1084B000822E23E5922E2BE7A22E21E4B22E2196C6
:1084C0004CAC5DAC6EAC7FAC219725962CAD3DAD30
:1084D0004EAD5FAD25976F962CAF3DAF4EAF5FAF02
:1084E0006F97A3019201B601C7010F946E592D96A3
:1084F0006CAF7DAF8EAF9FAF2D976F962CAD3DAD1E
:108500004EAD5FAD6F97612F702F832D922D0F941D
:108510006E5961966CAF7DAF8EAF9FAF6197A3012F
:10852000920160919D1070919E1080919F1090918A
:10853000A0100F946E592B013C016F962CAD3DADF0
:108540004EAD5FAD6F976091A1107091A2108091B8
:10855000A3109091A4100F946E596F966CAF7DAFDD
:108560008EAF9FAF6F97A0968FADA097A2969FAD4D
:10857000A297A596AFADA597A996BFADA9978DA7D0
:108580009EA7AFA7B8ABA4968FADA497AD969FADAD
:10859000AD97E196AFADE197E396BFADE39789ABB9
:1085A0009AABABABBCABC984DA84EB84FC84CDAAB8
:1085B000DEAAEFAAF8AE2DEC3CEC4CEC5CE3C50176
:1085C000B4010F94E35229813A814B815C810F946D
:1085D000E3522091A9103091AA104091AB10509114
:1085E000AC100F946F5969AF7AAF8BAF9CAFA301FA
:1085F0009201C301B2010F94E3522B013C016F962B
:108600002CAD3DAD4EAD5FAD6F97CA01B9010F9472
:10861000E3529B01AC01C301B2010F946F5920E0FA
:1086200030E040E050E40F94CF5B1816ACF420E04B
:1086300030E040E05FE3C701B6010F946F5929961F
:108640006CAF7DAF8EAF9FAF2997BE01635C7F4F4C
:10865000CE0101960E94892C89859A85AB85BC85BF
:1086600029968CAF9DAFAEAFBFAF29976B961CAE6E
:108670001DAE1EAE1FAE6B97BE01695A7F4FCE0175
:10868000CD960E94802CCE0101960F945F2EA09073
:108690007C10B0907D10C0907E10D0907F10E09044
:1086A0007810F090791000917A1010917B1097015A
:1086B000A801B501C6010F94CF5B181614F075011F
:1086C00086018090790290907A02A0907B02B0900F
:1086D0007C022DEC3CEC4CEC5DE3B701C8010F943F
:1086E000E3526093790270937A0280937B029093B5
:1086F0007C0240E0BE01675B7F4FCE018D960F94F8
:108700003D3680E1EDE9F0E1A5E3B8E001900D929E
:108710008A95E1F78092790290927A02A0927B0288
:10872000B0927C020E9460258111C8CB20E04FEFFF
:10873000BE016F5A7F4FCE0101960E944C2E20E061
:1087400041E0BE016F5A7F4FCE0101960E944C2E30
:108750002FEF40E0BE016F5A7F4FCE0101960E947D
:108760004C2E21E040E0BE016F5A7F4FCE010196B2
:108770000E944C2E0E94C6DC0E94602581119ECB77
:108780008091AD108093AE10E5964EAD5FADE5974C
:1087900041505109E5965FAF4EAFE597452B09F47F
:1087A0008DCB62968FAD629787FD88CB63968FAD38
:1087B000639787FF17CC82CB63E687E89AE00E9435
:1087C00054B20F947C3580E1EDE9F0E1A5E3B8E027
:1087D00001900D928A95E1F72D853E854F85588948
:1087E000609141087091420880914308909144083B
:1087F0000F946F5960934108709342088093430827
:1088000090934408CE01CD960E9451F92D853E8566
:108810004F855889609141087091420880914308C2
:10882000909144080F946E596093410870934208E8
:1088300080934308909344088CA58111A2CB81E0DA
:108840008CA78D819E81AF81B885B0588DA79EA7DA
:10885000AFA7B8ABBE01635D7F4F85E398E00E9490
:10886000802C8FCB2BA13CA14DA15EA1AC962CAF4F
:108870003DAF4EAF5FAFAC978FA198A5A9A5BAA5A4
:10888000CBCBC601D70121968CAF9DAFAEAFBFAFAA
:10889000219720E030E040EA50E4612F702F832DD3
:1088A000922D0F946E5925966CAF7DAF8EAF9FAF12
:1088B00025976C962FAD6C9724300CF4CACDA496F6
:1088C0001FAFA497AD960FAFAD97E1963FAEE1977E
:1088D000E3962FAEE39792ED892E93E5992E9BEFC9
:1088E000A92E90E4B92EEBCDA4964FADA4974430B9
:1088F0000CF46EC06C965FAD6C975430BCF120E008
:1089000030E040EA50E4B601C7010F946E59219659
:108910006CAF7DAF8EAF9FAF219720E030E040EA93
:1089200050E4612F702F832D922D0F946E59A496D1
:108930006FAFA497AD967FAFAD97E1968FAFE197FC
:10894000E3969FAFE3976C969FAD6C97A096CFAEE2
:10895000A097A296DFAEA297A596EFAEA597A9968F
:10896000FFAEA99794300CF0B6CFA1CDC601D701C8
:1089700021968CAF9DAFAEAFBFAF219720E030E026
:1089800040EA50E4612F702F832D922D0F946F5980
:1089900025966CAF7DAF8EAF9FAF25976C968FAD50
:1089A0006C978111BACF20E030E040EA50E4B60184
:1089B000C7010F946E59A0966FAFA097A2967FAF94
:1089C000A297A5968FAFA597A9969FAFA99777CFA6
:1089D0006C96AFAD6C97A1112BC020E030E040E267
:1089E00051E4A0966FADA097A2967FADA297A596F1
:1089F0008FADA597A9969FADA9970F946E59A09694
:108A00006FAFA097A2967FAFA297A5968FAFA597BD
:108A1000A9969FAFA997A4961FAFA497AD960FAF45
:108A2000AD97E1963FAEE197E3962FAEE3973FCD4A
:108A30006C96BFAD6C97B43034F120E030E040E28A
:108A400051E4A0966FADA097A2967FADA297A59690
:108A50008FADA597A9969FADA9970F946E592196B2
:108A60006CAF7DAF8EAF9FAF2197D5CFA096CFAE25
:108A7000A097A296DFAEA297A596EFAEA597A9966E
:108A8000FFAEA99728CFA4961FAFA497AD960FAFBE
:108A9000AD97E1963FAEE197E3962FAEE39782ED77
:108AA000882E83E5982E8BEFA82E81E4B82E07CD73
:108AB0008FE299E00C94FE34CF92DF92EF92FF9216
:108AC0000F931F93CF93DF9388E50E940330D82E36
:108AD00089E40E940330C82E8823D1F10E94D52F4B
:108AE000D82F89E50E940330182F8AE40E940330B2
:108AF000082F882309F455C00E94D52FC82F8AE576
:108B00000E940330E82EF12C811104C081E50E94FF
:108B10000330F82EC11001C000E0802F90E0D1108A
:108B200001C010E0810F911D019721F4E11062C096
:108B3000F11060C00E94584583E19EE0DF91CF9123
:108B40001F910F91FF90EF90DF90CF900C94FE3427
:108B5000D11002C0DFEFC5CF0E94D92F20914F095D
:108B60003091500940915109509152090F946E591A
:108B700020E030E040EA51E40F946E5920E030E00C
:108B80004EEB51E40F946F5922E936E74CEA5CE36F
:108B90000F94E3520F94DB5AD62F653008F4A1CF1F
:108BA000D9CF111102C0CFEFAACF0E94D92F2091A7
:108BB00053093091540940915509509156090F9429
:108BC0006E5920E030E040EA51E40F946E5920E005
:108BD00030E04EEB51E40F946F5922E936E74CEA4E
:108BE0005CE30F94E3520F94DB5AC62F653008F410
:108BF00086CFD9CFD7FD02C0C7FF05C00E94584518
:108C00008AEF9DE09BCF0E94D92F9B01AC010D2FD5
:108C1000DD0F110BAC2FCC0FBB0B60E070E0CB0174
:108C2000FF2091F065E0609FF001619FF00D11243D
:108C3000EA0FFB1FEE0FFF1FEE0FFF1FE153FA4F6E
:108C40006081718182819381E5E0E09FE001E19F95
:108C5000D00D1124CA0FDB1FCC0FDD1FCC0FDD1F81
:108C6000C153DA4F0F946F59688379838A839B834A
:108C7000DF91CF911F910F91FF90EF90DF90CF90F8
:108C8000089589E299E00C94FE34CF9384E50E9424
:108C90005130C0E08823D9F00E94B12FC82F181698
:108CA000B4F40E9441468DE40E94C5348091F404DE
:108CB0009091F5040F94923F6C2FCC0F770B8BEFB4
:108CC0009EE00E94FE3B8AE00E94C534CFEF8C2FCD
:108CD000CF9108954F925F926F927F928F929F9261
:108CE000AF92BF92CF92DF92EF92FF92CF93DF933A
:108CF000CDB7DEB72C970FB6F894DEBF0FBECDBF51
:108D000040904F095090500960905109709052095D
:108D10002091390230913A0240913B0250913C023D
:108D2000C301B2010F946F5969837A838B839C834B
:108D30008090530990905409A0905509B09056091D
:108D400020913D0230913E0240913F0250914002FD
:108D5000C501B4010F946F596D837E838F8398870B
:108D6000C0905709D0905809E0905909F0905A09DD
:108D700020914102309142024091430250914402BD
:108D8000C701B6010F946F5969877A878B879C87D3
:108D9000209145023091460240914702509148028D
:108DA000C301B2010F946F592B013C01209149027C
:108DB00030914A0240914B0250914C02C501B401DE
:108DC0000F946F594B015C0120914D0230914E027E
:108DD00040914F0250915002C701B6010F946F5954
:108DE0006B017C010E9441468CE49EE00E94FE34AF
:108DF00083E50E940330882321F00E94C52F8093D1
:108E0000370280913702811151C083E39EE00E94B6
:108E1000FE3484E49EE00E94FE3449815A816B81D5
:108E20007C818FEE9BE20E94E8364D815E816F81EE
:108E3000788588ED90E40E94E83649855A856B85EF
:108E40007C8585ED90E40E94E83682E49EE00E94F5
:108E5000FE348AE39EE00E94FE34B301A2018FEE4D
:108E60009BE20E94E836B501A40188ED90E40E94DF
:108E7000E836B701A60185ED90E40E94E8368AE065
:108E80002C960FB6F894DEBF0FBECDBFDF91CF9109
:108E9000FF90EF90DF90CF90BF90AF909F908F901A
:108EA0007F906F905F904F900C94C53487E39EE065
:108EB000AECF2F923F924F925F926F927F928F929E
:108EC0009F92AF92BF92CF92DF92EF92FF920F9359
:108ED0001F93CF93DF93CDB7DEB76A970FB6F894A1
:108EE000DEBF0FBECDBF83E50E940330182F309048
:108EF0009C10882319F00E94C52F382E40909D1099
:108F000050909E1060909F107090A0108091A110C2
:108F10009091A210A091A310B091A4108B8B9C8B68
:108F2000AD8BBE8B8091A5109091A610A091A7103B
:108F3000B091A8108F8B988FA98FBA8F112329F029
:108F4000311003C080E00E94BA3286E50E940330EF
:108F5000888B0E94B533882309F4BFC083E40E9444
:108F60000330882309F498C00E94D92F6B017C013B
:108F7000AFECB5E0BF83AE83B987A887F5E0FD838A
:108F80001D861E8628EC2F8702EC1A86212C88EC81
:108F90008B8792E49C87A885B985BA8BA98B15E04D
:108FA000E989FA8981909190A190B190FA8BE98B2F
:108FB0002A85322D4B855C85C501B4010F947D5205
:108FC00087FF04C08A86292CAB86BC862D853E850A
:108FD0004F85502FC501B4010F94CF5B181624F4B0
:108FE0008D869E86AF860B2D1150D1F6FD81F150F6
:108FF000FD8388859985449699878887F111CBCF21
:109000002D853E854F85502F6A85722D8B859C85D9
:109010000F946F5920E030E040E05FE30F94E3529B
:10902000A70196010F946F596B017C012DEB37E37B
:1090300046E855EB0F94CF5B87FD0AC02DEB37E375
:1090400046E855E3C701B6010F947D52181624F582
:1090500080E00E94BA3215E0AE80BF8005E0D50105
:109060006D917D918D919D915D014D01B4E08B1AC3
:109070009108A70196010F946E59F40160837183E2
:1090800082839383015059F711508E819F814496BA
:109090009F838E831111E0CFA889AA2351F00E94EB
:1090A000B533882331F080ED9CE00E94FE340E94AD
:1090B0004B368AE50E940330882359F00E94D92F4D
:1090C00069837A838B839C8360E0CE0101960E9442
:1090D000D532832D0E94BA320BC0311003C098895B
:1090E000992339F30E94414686EE9CE00E94FE34AB
:1090F000332051F080919C10811106C00E94584588
:1091000081EB9CE00E94FE340E94414683EA9CE091
:109110000E94FE3480919C100E94CA360E944146F3
:1091200086E99CE00E94FE34C0906708D0906808F1
:10913000E0906908F0906A0820E030E0A901C701DA
:10914000B6010F94CF5B18160CF053C042E0C70174
:10915000B6010F948C078DE00E94C5348AE00E940E
:10916000C534A301920160919D1070919E10809171
:109170009F109091A0100F947D5281111FC02B89D8
:109180003C894D895E896091A1107091A2108091F7
:10919000A3109091A4100F947D5281110FC02F89BC
:1091A000388D498D5A8D6091A5107091A6108091CF
:1091B000A7109091A8100F947D5281110E9409FB75
:1091C0006A960FB6F894DEBF0FBECDBFDF91CF9188
:1091D0001F910F91FF90EF90DF90CF90BF90AF90D5
:1091E0009F908F907F906F905F904F903F902F90C7
:1091F000089581E99CE00E94FE34B3CFCF93C82F3D
:1092000082E0C11184E040E060E00E94C3840E94DB
:10921000414689E999E0CC2311F08EEA99E0CF919B
:109220000C94FE34FF920F931F93CF93DF93EC01C6
:109230008B01F42E0E9421D50E94584589E099E0C7
:109240000E94FE340115110511F40EE61FE320976C
:1092500011F4C0E0D9E00E940CB91F930F93DF9383
:10926000CF9380EF98E09F938F9381E08F930E943C
:1092700039B20E94DA83C0915416C695C6958FE420
:1092800096E10E948527DC2FDD0F1D2F1C0FEDB707
:10929000FEB737960FB6F894FEBF0FBEEDBF83E062
:1092A0000E94692644E653E16C2F80E00E94302A38
:1092B00010928A16D0938B1681EE98E00E941528A2
:1092C00010928A1610938B1684ED98E00E94152850
:1092D00083E596E10F94363D8111E1CF61E087EFA0
:1092E00098E00E94C63589EE93E030E6019729F0B8
:1092F000232F2A950000E9F7F9CFF89489EE93E03F
:1093000038EE019729F0232F2A950000E9F7F9CFCD
:109310000E9421D5FF2041F00E9430340E94B221EA
:10932000909905C0A895FCCF0E94B021F7CF909BE3
:1093300002C0A895FCCFF0E0E0E0DF91CF911F9153
:109340000F91FF9019945F926F927F928F929F92EC
:10935000AF92BF92CF92DF92EF92FF920F931F9343
:10936000CF93DF931F92CDB7DEB77C0139018B011C
:109370005B01A40EB51ED12CC12CA016B10609F4B8
:1093800050C0F70180809180F80151908F0159827F
:10939000C4010F949B585816B9F1652DC4010F9460
:1093A000A358FFEFCF1ADF0AC6018F779927892BC1
:1093B00021F162E070E080E090E00F941035C4018C
:1093C0000F949B5899818917F9F00E94414683E7D1
:1093D00096E00E94FE3481E00F90DF91CF911F91C3
:1093E0000F91FF90EF90DF90CF90BF90AF909F9044
:1093F0008F907F906F905F90089562E070E080E0C2
:1094000090E00E94FA33DBCFBE016F5F7F4FC30154
:109410000F945325F7018081918101969183808378
:10942000ACCF80E0D9CF8091AD109091AE102FEFEE
:109430003FEF981751F0E92FF0E0E355FF4E2281FE
:1094400030E09F5F9F779093AE10C90108951F92FF
:109450000F920FB60F9211240F900FBE0F901F9016
:1094600018951F920F920FB60F9211240BB60F9200
:109470002F933F934F935F936F937F938F939F931C
:10948000EF93FF939091C6005091AE103091AD10C4
:1094900041E0430F4F7720917D04213108F099C0BE
:1094A000E22FF0E08827E85AF54B8F4F0D9466596C
:1094B000694A924AA14AB04AB74AE94ABB4AE94ACC
:1094C000BF4AC34AE94AC74ACB4ACF4AD64AE94AC1
:1094D000E14A903229F0F8F49A3011F09D3001F50C
:1094E000541731F0E32FF0E0E355FF4E9283342F11
:1094F0003093AD10FF91EF919F918F917F916F917C
:109500005F914F913F912F910F900BBE0F900FBE27
:109510000F901F9018959D3481F081E09E3471F07A
:1095200080E10CC09A3338F49033D0F69032C1F217
:109530009D32B1F7D5CF9D3499F782E080937D04B9
:10954000CFCF913359F018F4903251F2E9CF88E03F
:109550009433A1F38BE0983389F3E2CF83E0EECF2D
:1095600084E0903359F386E0913341F3D9CF85E01D
:109570009833B1F6E3CF87E0923391F6DFCF89E0FD
:10958000913371F6DBCF8AE0903351F6D7CF8CE080
:10959000973331F6D3CF8DE0963311F6CFCF90329B
:1095A00009F49ECF8EE0933549F2BACF80ED890F52
:1095B0008A3008F095CF2FE020937D0480937C04BF
:1095C0008FCF9A3019F09D3009F08ACF10927D0428
:1095D00087CF9A3019F09D3009F082CF80918D1697
:1095E0008823A1F3273001F138F4253079F7109260
:1095F000710210924F08EACF2A30D1F02F3031F7A4
:1096000020917C0480914D0810924D08823089F39E
:10961000843091F08130D1F6222319F02130B1F657
:1096200082E080934E08D2CF81E080934106CECF76
:1096300081E080934006CACF65E27EE17093C60761
:109640006093C507C3CF8EBD0DB407FEFDCF08954F
:109650008FEF8EBD0DB407FEFDCF8EB508959091AE
:1096600064009B7F90936400982F906A96959CBDB0
:1096700080FD03C091E0863009F490E09DBD08951F
:10968000CF93DF93EB010E94FE34CE01DF91CF91A7
:109690000C949ECEAF92BF92CF92DF92EF92FF9248
:1096A0000F931F93CF93DF93CDB7DEB7E6970FB637
:1096B000F894DEBF0FBECDBF0091F7041091F804FF
:1096C000F80101900020E9F731976F01C01AD10A23
:1096D000F801CF01801B910B8C159D053CF4819105
:1096E0008F32B9F7DF0111971C92F3CF8BE1E2EED5
:1096F000F6E1DE015C9601900D928A95E1F7F12C7E
:10970000E12CEC14FD040CF05DC0F801EE0DFF1D22
:109710008081811103C08FEFE81AF80A5801AE0C5E
:10972000BF1CF5018081882309F44CC0FFEFEF1ABC
:10973000FF0AF801EE0DFF1D7F01E01AF10A819189
:109740008111FACFCE014C960E9404D38BE1FE0129
:109750007C96DE01119601900D928A95E1F7B50194
:10976000CE0101960E9410CBCE0101960E940332D9
:109770008FE20E94C5348091211381113BC08CE59A
:1097800093E00E949ECE8091C11684FF1BC0198277
:109790001C8221E0A501BE01645E7F4FCE010196CF
:1097A0000F94AD05811129C08AE00E94C5340E9442
:1097B0004146B50189EB94E10E94404BCE010196F0
:1097C0000E9403328AE00E94C534CE014C960E946A
:1097D0000332E6960FB6F894DEBF0FBECDBFDF9121
:1097E000CF911F910F91FF90EF90DF90CF90BF909E
:1097F000AF90089581E293E1C4CFCE014C960E94D0
:1098000006D28BE1FE013196DE015C9601900D924D
:109810008A95E1F7CE0101960E94033272CF2F9212
:109820003F924F925F926F927F928F929F92AF92F0
:10983000BF92CF92DF92EF92FF920F931F93CF933D
:10984000DF9300D000D000D01F921F92CDB7DEB7BB
:10985000B82E80919A11843008F0D1C10F9443350D
:109860006B017C0180919A11811108C08091AD102B
:109870009091AE10891B8F7709F463C681E6A82EFC
:1098800013C08A3019F08D3009F0F6C0109295118E
:109890008091331190913411FC01E15DFE4E1682EE
:1098A000892BF1F40E9463F280919A11843008F0C0
:1098B000ECC08091AD109091AE10891B8F7709F4A8
:1098C000E4C00E94134A97FFDCCF0E94584589EB01
:1098D00097E00E94FE348091AD108093AE10E4CFEB
:1098E000109234111092331105E311E1F8018191C6
:1098F000803209F446C08E3409F0A9C064EB77E0E9
:10990000C8010F94FA514C01892B41F06EE470E0CC
:10991000C80104960F94BD5C009709F4C8014AE0A1
:1099200050E070E060E001960F946A4F2B013C011B
:1099300080912F1190913011A0913111B09132117D
:109940000196A11DB11D481659066A067B0629F02D
:1099500060E081E897E0892851F16AE270E0C8018F
:109960000F94EC5C9C01009729F1982F901B912C8F
:10997000992349F09150F801E90FF11D8081982653
:10998000F7CF8F01B3CF4AE050E070E060E0C9014B
:1099900001960F946A4F292D30E050E040E06217A5
:1099A00073078407950751F060E082E697E00F9413
:1099B000202A7ACF60E088E397E0F9CF40922F1118
:1099C00050923011609231117092321180910808DA
:1099D0008130E1F067E470E0C8010F94BD5C00974E
:1099E000A9F04AE050E070E060E001960F946A4F01
:1099F000643071058105910548F487E996E00E947D
:109A0000FE3460E08DE896E00E9454B2C0925408A3
:109A1000D0925508E0925608F0925708809135117F
:109A20008B3309F441CF80919A11843008F03CCFF8
:109A300080919C118A9DC001112465E371E18356D8
:109A40009E4E0F94C85C80E00F94DA292DCF809150
:109A5000C11680FFBBCF61EF7EE3C8010F94FA51BE
:109A6000009731F0FC01838180538A3008F0AECF3B
:109A700060E08EE097E09BCF23E331E145E351E1E5
:109A800065E971E10E943F210FCF8091C11682FFED
:109A9000B6C01A82198271E6F72EE0E1EE2EF9E6E1
:109AA000DF2E80919A11843008F0A9C00E9477219E
:109AB0008111A5C041E050E0BE016B5F7F4F86E29F
:109AC00098E10E943ECF0D8110E0019711F00FEF59
:109AD0001FEF80912E1890912F18A0913018B091FF
:109AE00031188093BD169093BE16A093BF16B09305
:109AF000C0160E9477210F3F100749F4811107C05B
:109B00000E94584587ED97E00E94FE34CACF4091ED
:109B10009C11242F30E00A3061F00D3051F0882381
:109B200009F45FC089819A81009719F001969A83A0
:109B3000898310927E0489819A81F29EF001F39EBE
:109B4000F00D1124E656FE4EE80FF91F1382892B03
:109B500069F50E9463F20E947721882309F4A1CF5E
:109B60000E94C6DC86E298E10E9406D28091B81677
:109B7000882391F181508093B8168D9DC0011124E6
:109B800062E08C5C984F0F944243E091B81624E059
:109B9000E29FF0011124E05DF84F608171818281C4
:109BA00093810E94A4230E9479CA7BCF1A821982D2
:109BB00081E00F94DA298091BD169091BE16A09194
:109BC000BF16B091C0168093961190939711A093F1
:109BD0009811B0939911BFCF0E940FD2E09208085C
:109BE00060CF4F9DA001112443565E4E9E012F5F12
:109BF0003F4F6EE774E0802F0E943F2152CF0F94B9
:109C000043356B017C01B11004C080914E0688235E
:109C100051F0C0924508D0924608E0924708F09271
:109C20004808BB24B3948091D1049091D204A091B0
:109C3000D304B091D4040097A105B10551F140912E
:109C40004508509146086091470870914808840F74
:109C5000951FA61FB71FA7019601281B390B4A0B9A
:109C60005B0BDA01C901B7FD14C00E945845609131
:109C700052087091530882E398E00E94404B8AE0BA
:109C80000E94C53440E070E060E090E080E00E9417
:109C900012498091100290911102A0911202B0918C
:109CA0001302892B8A2B8B2B79F0909117168091B8
:109CB0001816981709F4ACC1C0924508D09246080E
:109CC000E0924708F092480880918F0490919004A8
:109CD0009099E0C101969093900480938F048091B5
:109CE0008F04909190048E3E92406CF00E945845F3
:109CF0008FE098E00E94FE3440E070E060E090E089
:109D000080E00E9412490F9443354B015C01809121
:109D10004F08811108C0209117169091181681E004
:109D2000291301C080E02091D3153091D41591E022
:109D300089272A3A31050CF480E091E040918304B0
:109D4000509184046091850470918604452B462BC4
:109D5000472B09F490E0981789F0882309F4A0C1F3
:109D6000D501C40180569444A24FBF4F8093830411
:109D700090938404A0938504B09386044090A91026
:109D80005090AA106090AB107090AC1020917F049E
:109D9000309180044091810450918204C301B2014A
:109DA0000F947D52882319F180918304909184044B
:109DB000A0918504B091860440927F045092800463
:109DC0006092810470928204892B8A2B8B2B09F478
:109DD00049C0D501C40180569444A24FBF4F80931F
:109DE000830490938404A0938504B09386048091A7
:109DF000830490918404A0918504B0918604009717
:109E0000A105B10579F1881A990AAA0ABB0AB7FC1B
:109E100029C0109283041092840410928504109239
:109E200086048AEF97E00E94FE3460E086EE97E0B9
:109E30000E9454B28091D5159091D6151816190626
:109E400024F490E080E00E9448DC809171089091B9
:109E500072081816190634F41092720810927108DC
:109E60000E9441C680918B0490918C04A0918D0436
:109E7000B0918E0446015701881A990AAA0ABB0AB2
:109E8000D501C401B7FD9CC12091171690911816F9
:109E90008091600240916102291306C190918D0961
:109EA000899FC0011124880F892F881F990B9195D4
:109EB0008D8380918E09489FC0011124880F892FBE
:109EC000881F990B91958E830F94433569837A830C
:109ED0008B839C8340E0BE016F5F7F4FCE01059670
:109EE0000E941ADD6D8170E089E00F943A3441E000
:109EF000BE016F5F7F4FCE0105960E941ADD6E8115
:109F000070E087E00F943A3480914D06882309F47D
:109F10004AC10091330210913402C8010297209186
:109F2000D5153091D615281739070CF43CC180900F
:109F300018168F82188619861A861B868091171626
:109F40009F80891509F4CAC0892D90E03BE6A32EB5
:109F5000A89EF001A99EF00D1124EE55F64F4589FB
:109F600056896789708D452B462B472B81F4418D8F
:109F7000528D638D748D452B462B472B41F4458DB7
:109F8000568D678D70A1452B462B472BE1F12BE6B3
:109F9000B22EB89E9001B99E300D1124A9014E55E4
:109FA000564F1A01FA0161817281838194810F9465
:109FB0001D5C4B015C01F10161A172A183A194A11F
:109FC0000F9482522B013C01F10165A176A187A17A
:109FD00090A50F9482529B01AC01C301B2010F9472
:109FE000695AA50194010F94E3524B015C01288545
:109FF00039854A855B850F94CF5B181624F48886D3
:10A000009986AA86BB868F818F5F8F708F8396CF4C
:10A01000BB2019F01092910457CE0F944335009154
:10A0200045081091460820914708309148088090D3
:10A03000100290901102A0901202B0901302080D2D
:10A04000191D2A1D3B1D601B710B820B930B97FD85
:10A05000E1CF80919104811137CE81E0809391040A
:10A060005F9A8091C3078E7F8093C3078A9A8091FD
:10A07000C3078D7F8093C30780910801809581700D
:10A08000809306018091C3078B7F8093C3070E9452
:10A09000B0211ACE181619060CF021CE01971BCE4E
:10A0A00080E090E0DC0162CE209118165BE6259FEF
:10A0B000900111242E55364FF901EF59FF4F908131
:10A0C000899FC0011124880F892F881F990B9195B2
:10A0D0008D832E593F4FF9018081EDCE20912D02C5
:10A0E00030912E0240912F0250913002688579857F
:10A0F0008A859B850F94E3524B015C01B801012EC8
:10A10000000C880B990B0F9484529B01AC01C50184
:10A11000B4010F946F5969837A838B839C83409138
:10A12000310250913202B801CE0101960E94ECD565
:10A1300089809A80AB80BC804090870450908804CE
:10A140006090890470908A04A3019201C501B40152
:10A150000F947D5287FF16C028E431EE4AE75FE393
:10A16000C301B2010F94E35220E037ED43EA5CE310
:10A170000F946F59A50194010F94E35269837A8378
:10A180008B839C8369817A818B819C816093870416
:10A19000709388048093890490938A040F94DB5A07
:10A1A000CB010E9448DCF4E6CF0ED11CE11CF11C6F
:10A1B000C0928B04D0928C04E0928D04F0928E04B5
:10A1C0000E9463F280910808882309F47AC1909173
:10A1D0000901892F8095817010910802181709F4E0
:10A1E0005AC02091C11620622093C11680930802A4
:10A1F00090FD10C064EF71E080E090E00E94FA33BF
:10A200000E9431D28091C11683FDBEC1112309F491
:10A2100042C002C00E9420D2123008F46BC100E09C
:10A220000E94AB2683E080937D020F9443356C59E6
:10A230007F4F8F4F9F4F6093FC047093FD0480937A
:10A24000FE049093FF04002331F1123021F5809138
:10A25000C11683FF20C00F947C40882379F081E0F1
:10A260000F94983F42EB50E06DE978E087EC96E17F
:10A270000E943ECF87EC96E10E9406D20E94F13107
:10A28000811144C10E94DB310F94874181E08093AA
:10A29000B7160F94C9410F9443356B017C0110919F
:10A2A0000F021123F1F0809150088823D1F04091E2
:10A2B0009204509193046091940470919504460126
:10A2C0005701841A950AA60AB70AB501A40177FDB9
:10A2D0001AC0833009F430C10CF01FC181300CF07A
:10A2E00024C1212F30E0A8EEB3E00F941559C60E1B
:10A2F000D71EE81EF91EC0929204D0929304E092F9
:10A300009404F092950480916508813009F073C03F
:10A310000F9443356B017C0180919A0490919B04CA
:10A32000A0919C04B0919D04A7019601281B390BB4
:10A330004A0B5B0BDA01C901B7FD3AC0D701C60170
:10A34000805F984DAF4FBF4F80939A0490939B04CA
:10A35000A0939C04B0939D048090C2059090C30587
:10A36000A090C405B090C5050E9484FDAB01BC015E
:10A370004093C2055093C3056093C4057093C5050F
:10A380008091B4079091B507A091B607B091B70737
:10A3900088199909AA09BB09840F951FA61FB71F21
:10A3A0008093B4079093B507A093B607B093B7070F
:10A3B0008091960490919704A0919804B09199048B
:10A3C00046015701881A990AAA0ABB0AD501C40195
:10A3D000B7FD11C020E8C20E2EEED21E26E3E21E0B
:10A3E000F11CC0929604D0929704E0929804F092E7
:10A3F00099040E94CADB0F9415020E945EB68091F8
:10A40000D004882379F10F9443356B017C0180914E
:10A41000CC049091CD04A091CE04B091CF0446011C
:10A420005701881A990AAA0ABB0AD501C401B7FDC7
:10A4300019C02091D00430E0A8EEB3E00F94155974
:10A44000C60ED71EE81EF91EC092CC04D092CD04D1
:10A45000E092CE04F092CF0480E00F9430088AE0BE
:10A460000E94C5348091CB04882359F10F94433561
:10A470006B017C018091C7049091C804A091C9042C
:10A48000B091CA04A7019601281B390B4A0B5B0B3C
:10A49000DA01C901B7FD15C02091CB0430E0A8EE68
:10A4A000B3E00F941559C60ED71EE81EF91EC092D0
:10A4B000C704D092C804E092C904F092CA040F9471
:10A4C0009F402B960FB6F894DEBF0FBECDBFDF9135
:10A4D000CF911F910F91FF90EF90DF90CF90BF90A1
:10A4E000AF909F908F907F906F905F904F903F9034
:10A4F0002F90089560E08FE698E00E9454B280911A
:10A500000A0581118CCE0E94DA8389CE8CE898E00E
:10A510009093C6078093C507BECE843009F0E1CE84
:10A520000E94414683E998E004C00E94414682ECC3
:10A5300098E00E94FE34D5CE0E9441468BEA98E016
:10A54000F8CF8091540890915508A0915608B09189
:10A550005708A7019601281B390B4A0B5B0BDA0140
:10A56000C901885E9340A109B109B7FD87C981ED92
:10A5700097E00E94FE34C0925408D0925508E092B1
:10A580005608F09257087AC9123028F460E08DE737
:10A5900098E00E9454B201E043CECF93DF93C82FDE
:10A5A000D62F8091531083FD14C080919F09811193
:10A5B00010C08091820290918302AC0141505109F8
:10A5C0002091D5153091D6152417350714F40E9423
:10A5D00048DC40E06D2F8BE00E94C384CC2339F02F
:10A5E00040E061E080E0DF91CF910D94280A8091F6
:10A5F0009F0991E0892780937102809171028823DD
:10A6000089F08091D3159091D4152091D515309172
:10A61000D615821B930B97FF03C0919581959109E5
:10A62000029744F4109271028091531083FF06C088
:10A63000C1E01AC080E00E940F4CDFCFC0919F099B
:10A64000C11112C0809182029091830201972091E2
:10A65000D5153091D6152817390754F70E94414671
:10A6600088E899E00E94FE348C2FDF91CF91089505
:10A67000AF92BF92CF92DF92EF92FF920F931F9310
:10A68000CF93DF93CDB7DEB764970FB6F894DEBFF4
:10A690000FBECDBF0E944546D82E87FDB5C08AE5C6
:10A6A0000E945130882309F4C0C040E050E0BA0154
:10A6B0008AE50E946C307B018C014D2D63E085E0C2
:10A6C0000E94C3842091A5103091A6104091A7103C
:10A6D0005091A81060E070E08AE793E40F946E59FF
:10A6E0005B016C019701A8010F94CF5B181614F061
:10A6F0007501860120E030E0A901B701C8010F947F
:10A70000CF5B181624F4E12CF12C00E010E0B70127
:10A71000C8010F94DB5A072E000C880B990B0F947D
:10A7200084526D837E838F83988720E030E0A90177
:10A730000F947D52882321F0CE0105960E94F223CA
:10A7400080E090E0A0EAB1E489879A87AB87BC8774
:10A750001D861E861F86188A8CE40E94033088237B
:10A7600009F468C00E94D92F6B017C0120E030E021
:10A77000A901C701B6010F94CF5B87FF04C0F7FAA8
:10A78000F094F7F8F094C98ADA8AEB8AFC8A20916F
:10A79000D5153091D6152430310574F08091D3153C
:10A7A0009091D415821B930B97FF03C091958195CF
:10A7B000910901E004970CF400E063E080E00E945E
:10A7C000CD52811140C083E080932402109209058C
:10A7D0000E94DA836D817E818F8198858B019C0137
:10A7E000305809831A832B833C8320E030E0A90191
:10A7F0000F947D52882321F0CE0101960E94F2230E
:10A80000109209050E94DA8364960FB6F894DEBFB1
:10A810000FBECDBFDF91CF911F910F91FF90EF90B1
:10A82000DF90CF90BF90AF900895E12CF12C00E223
:10A8300011E443CFC090CA05D090CB05E090CC0581
:10A84000F090CD0593CF83E0E82E22E0AE01475F84
:10A850005F4FBE016F5E7F4FCE010D960F94242C8B
:10A86000B9CF6F927F928F929F92AF92BF92CF9209
:10A87000DF92EF92FF920F931F93CF93DF9300D05D
:10A8800000D01F921F92CDB7DEB75C014B013A0199
:10A89000F22E68010091460610924206109243067D
:10A8A0001092440610924506109246060F944F35BA
:10A8B0008091D5159091D6158C159D051CF4C60177
:10A8C0000E9448DC60E080E00E94CD5281112DC1E1
:10A8D000109209050E94DA831C141D0444F4C60179
:10A8E0000E9448DC40E060E080E00F94280A40E0ED
:10A8F00060E088E00E94C38460E081E00E94CD5265
:10A9000080E090E0A0E7B2E489839A83AB83BC83C4
:10A9100080E090E0A0E8B0EC8D839E83AF83B887A1
:10A92000BE016F5F7F4FCE0105960E9438F287E02F
:10A930000E9478F0811158C08091A5109091A610C6
:10A94000A091A710B091A8104091AA045091AB0417
:10A950006091AC047091AD04C090A604D090A7049F
:10A96000E090A804F090A904C0923508D09236086F
:10A97000E0923708F09238084093390850933A082B
:10A9800060933B0870933C0880933D0890933E0889
:10A99000A0933F08B093400880E090E0A8E4B2E4C0
:10A9A00089839A83AB83BC83CE0101960E9451F9BF
:10A9B0008091AE049091AF04A091B004B091B10425
:10A9C00080933D0890933E08A0933F08B0934008C1
:10A9D00080E090E0A0EAB0E489839A83AB83BC83F3
:10A9E000CE0101960E9451F9C12CD12C80E7E82EAE
:10A9F00082E4F82EC982DA82EB82FC8280E090E069
:10AA0000A0E8B0E48D839E83AF83B887BE016F5FFB
:10AA10007F4FCE0105960E9438F220E030E0A90178
:10AA20006091B2047091B3048091B4049091B50424
:10AA30000F947D5287FF0BC0C982DA82EB82FC82C1
:10AA4000BE016F5F7F4F82EB94E00E9438F28091ED
:10AA5000B2049091B304A091B404B091B504809372
:10AA6000A9109093AA10A093AB10B093AC10809350
:10AA7000410890934208A0934308B093440881E4AE
:10AA800098E00E9460EE8091CE0581110F94C23F44
:10AA9000109209050E94DA8361E081E39AE00E9446
:10AAA000C63580914E06815080934E0646EE5DE19C
:10AAB00069E37AE085E00F942F2D80914E0688237C
:10AAC00039F00E9479CA80914E06815080934E06DB
:10AAD0008091A504882351F01092A5048091A304CD
:10AAE00080938D098091A40480938E0980916508DC
:10AAF000823011F40E9446FE0F9482420E94DA8353
:10AB000028960FB6F894DEBF0FBECDBFDF91CF9170
:10AB10001F910F91FF90EF90DF90CF90BF90AF907B
:10AB20009F908F907F906F900895E12C2F2DA3011F
:10AB3000B401C5010F94242CCFCE4F925F926F9237
:10AB40007F92AF92BF92CF92DF92EF92FF921F93CC
:10AB5000CF93DF9300D000D01F921F92CDB7DEB706
:10AB60005C01E62EF42E642F80E00E94CD52182F57
:10AB700081111BC0EE2021F0109209050E94DA839A
:10AB8000812F28960FB6F894DEBF0FBECDBFDF91A0
:10AB9000CF911F91FF90EF90DF90CF90BF90AF903B
:10ABA0007F906F905F904F900895EE2029F040E0E5
:10ABB0006F2D83E00E94C38480E090E0A0E7B2E4C0
:10ABC0008D839E83AF83B88780E090E0A0E8B0ECEF
:10ABD00089839A83AB83BC83BE016B5F7F4FCE01B9
:10ABE00001960E9438F268E873E180E090E00E94EC
:10ABF000FA33C12CD12C88ECE82E81E4F82ECD82DA
:10AC0000DE82EF82F88680E090E0A0E8B0E48983FD
:10AC10009A83AB83BC83BE016B5F7F4FCE010196ED
:10AC20000E9438F240908C1050908D1060908E10E1
:10AC300070908F10C0928C10D0928D10E0928E1078
:10AC4000F0928F1080E090E0A0E2B2E48D839E83CA
:10AC5000AF83B887F50180819181A281B381898317
:10AC60009A83AB83BC83BE016B5F7F4FCE0101969D
:10AC70000E9438F240928C1050928D1060928E108B
:10AC800070928F10129A64E670E080E090E00E946B
:10AC9000FA3376CFBF92CF92DF92EF92FF920F936B
:10ACA0001F93CF93DF9300D01F92CDB7DEB77C0107
:10ACB0006B018A01B22E61E084E29AE00E94C635FF
:10ACC00046EE5DE16BE27AE085E00F942F2D9091E6
:10ACD0004E0681E0890F80934E068091C11682FF57
:10ACE00006C08B7F8093C1169E5F90934E060E9494
:10ACF0007EFE80E1EDE9F0E1A6EAB4E001900D927C
:10AD00008A95E1F70E94C6DC8091A50481110FC0ED
:10AD100081E08093A50480918D098093A304109213
:10AD20008D0980918E098093A40410928E0920E0F1
:10AD300030E0A901F70160817181828193810F94D4
:10AD40007D528823F1F080919F0981110CC0809180
:10AD500082029091830201972091D3153091D415EE
:10AD60002817390774F080E090E0A0E7B2E4898307
:10AD70009A83AB83BC83BE016F5F7F4FC7010E9484
:10AD800038F287E00E9478F0811103C0B6010F9479
:10AD90005A0120E030E0A901F801608171818281CF
:10ADA00093810F947D52882329F042E06B2DC801D6
:10ADB0000E949D55129A64E670E080E090E00E9447
:10ADC000FA3381E00F900F900F900F90DF91CF91A9
:10ADD0001F910F91FF90EF90DF90CF90BF9008955B
:10ADE000CF92DF92EF92FF92CF93DF936B017C01C2
:10ADF000D42FC091500883E08093500881E0809365
:10AE00004F08C114D104E104F10431F00F9443352B
:10AE1000C60ED71EE81EF91E80914F08882389F0C0
:10AE2000C114D104E104F10421F48D2F0E940F4CD0
:10AE3000F3CF0F9443356C197D098E099F0997FD57
:10AE4000F4CF10924F08C0935008DF91CF91FF903C
:10AE5000EF90DF90CF9008951F93CF93DF93D82F7B
:10AE6000C62F0E94FE4861E08C2F0E9409320F9489
:10AE70004335685370458F4F9F4F609342067093E0
:10AE8000430680934406909345061092460610911F
:10AE9000500883E08093500830E020E04FE450E415
:10AEA00066E17AE082E00E940D3681E080934F08EF
:10AEB00080914F08882309F463C060E08C2F0E94C2
:10AEC000093280914606882309F456C040E060E0CC
:10AED0008AE00E94C3840E9441468CEF99E00E9460
:10AEE000FE3430E020E046EE59E06DEE79E082E09D
:10AEF0000E940D3641E060E070E0CB010E94F05608
:10AF000030E020E050E040E069ED79E085E00E942B
:10AF10000D3610924206109243061092440610928B
:10AF20004506109246060F944F3560E080E00E947F
:10AF3000CD528D2F0E94FE480F94433568537045C3
:10AF40008F4F9F4F60934206709343068093440651
:10AF5000909345061092460630E020E04FE450E41E
:10AF60006DEC79E082E00E940D3681E080934F081D
:10AF700061E08C2F0E94093281E00E940F4C98CF33
:10AF800010935008DF91CF911F910895CF92DF92D7
:10AF9000EF92FF920F931F93CF93DF93CDB7DEB75E
:10AFA000A0970FB6F894DEBF0FBECDBF0E944546F6
:10AFB00087FDD1C0482F61E081E00E94C38485E411
:10AFC0000E940330882309F4D5C00E94D92F6B0159
:10AFD0007C0120E030E0A9010F94CF5B87FF04C023
:10AFE000F7FAF094F7F8F094F7FAF094F7F8F09491
:10AFF000C98ADA8AEB8AFC8A8CE0E8E8F2E0DE01B2
:10B00000119601900D928A95E1F78AE50E945130E0
:10B01000882351F040E050E0BA018AE50E946C308C
:10B0200069877A878B879C8788E50E9451308823BF
:10B0300051F040E050E0BA0188E50E946C3069832D
:10B040007A838B839C8389E50E945130882351F059
:10B0500040E050E0BA0189E50E946C306D837E8348
:10B060008F83988785E50E940330882309F489C07F
:10B070000E94D92F6B017C0120E030E0A901C701BB
:10B08000B6010F94CF5B87FF04C0F7FAF094F7F88E
:10B09000F094F7FAF094F7F8F094CD8ADE8AEF8A0C
:10B0A000F88E198E1A8E1B8E1C8E8CE40E94033033
:10B0B000882309F46FC00E94D92F6B017C0120E026
:10B0C00030E0A901C701B6010F94CF5B87FF04C030
:10B0D000F7FAF094F7F8F094CD8EDE8EEF8EF8A2AA
:10B0E00062E070E082E40E94B731F82E80914E0653
:10B0F000811131C021E0AE014B5E5F4FBE016F5F39
:10B100007F4FCE0141960E944A56882321F16F2D30
:10B1100081E00E942C5782E50E945130882309F477
:10B1200042C00E94D52F40E050E060EA71E44D87B4
:10B130005E876F87788B20914E06222361F08C0109
:10B140002F2DAE01435F5F4FBE01635E7F4FCE0187
:10B1500049960E943154A0960FB6F894DEBF0FBEF8
:10B16000CDBFDF91CF911F910F91FF90EF90DF90B6
:10B17000CF900895C12CD12C80E8E82E80E4F82EE1
:10B1800033CFC090C605D090C705E090C805F090B9
:10B19000C90572CFC090CA05D090CB05E090CC0510
:10B1A000F090CD058CCF90E080E0BDCFCF92DF92C4
:10B1B000EF92FF920F931F93CF93DF93CDB7DEB73C
:10B1C0006C970FB6F894DEBF0FBECDBF8CE40E9423
:10B1D0000330882309F4C3C00E94D92F6B017C017E
:10B1E00020E030E0A9010F94CF5B87FF04C0F7FA9D
:10B1F000F094F7F8F094F7FAF094F7F8F094C98E19
:10B20000DA8EEB8EFC8E8CE0E8E8F2E0DE0111963F
:10B2100001900D928A95E1F788E50E9451308823CC
:10B22000A1F040E050E0BA0188E50E946C30209126
:10B230004F093091500940915109509152090F9492
:10B240006E5969837A838B839C8389E50E94513090
:10B250008823A1F040E050E0BA0189E50E946C30FB
:10B2600020914F0930915009409151095091520954
:10B270000F946E596D837E838F8398878AE50E9431
:10B280005130882351F040E050E0BA018AE50E9435
:10B290006C3069877A878B879C87F090C116F2FAA9
:10B2A000FF24F0F840E061E080E00E94C38460E0A9
:10B2B00080E50E94C631E82E1D861E861F86188AEC
:10B2C00080914E0681113CC02E2DAE01435F5F4F31
:10B2D000BE016F5F7F4FCE0149960E944A56882378
:10B2E00079F18091CE0581110F94C23FFF2011F0BA
:10B2F000EE2031F160E080E00E942C57898D9A8D1C
:10B30000AB8DBC8DB0588D8B9E8BAF8BB88F198A4F
:10B310001A8A1B8A1C8A1D861E861F86188A80919F
:10B320004E06882369F010E000E020E0AE014B5E9D
:10B330005F4FBE016F5E7F4FCE010D960E9431546C
:10B340006C960FB6F894DEBF0FBECDBFDF91CF91E4
:10B350001F910F91FF90EF90DF90CF900895C12C37
:10B36000D12C80E8E82E80E4F82E45CF2F923F9232
:10B370004F925F926F927F928F929F92AF92BF9205
:10B38000CF92DF92EF92FF920F931F93CF93DF93B1
:10B39000CDB7DEB7E1970FB6F894DEBF0FBECDBFD5
:10B3A00089AB2091500828AB21E020935008809170
:10B3B000F6048D3409F463C4843511F40C94996E49
:10B3C000873409F044C18091F4049091F5048A31E6
:10B3D000910509F4D7C108F03DC18430910508F00A
:10B3E00030C1209108088230910508F451C1213004
:10B3F00009F054C111E0029709F010E00E94833077
:10B4000019821A821B821C821D821E821F8218864C
:10B4100082E50E945130882309F453C10E94D92F3C
:10B420006B017C0120E030E0A9010F947D5288235C
:10B4300009F4EAC040909D1050909E1060909F10BB
:10B440007090A0108091A1109091A210A091A310D3
:10B45000B091A41088A799A7AAA7BBA78090350888
:10B4600090903608A0903708B0903808809139083D
:10B4700090913A08A0913B08B0913C088CA79DA7F9
:10B48000AEA7BFA7A5019401C301B2010F947D52DD
:10B4900081110DC02CA53DA54EA55FA568A579A578
:10B4A0008AA59BA50F947D52882309F4ADC0A30102
:10B4B0009201C501B4010F946E5920E030E040E0E4
:10B4C0005FE30F94E3526CA37DA38EA39FA328A5F3
:10B4D00039A54AA55BA56CA57DA58EA59FA50F9452
:10B4E0006E5920E030E040E05FE30F94E3522B011F
:10B4F0003C0120E030E0A901C701B6010F947D5264
:10B50000881F8827881F181709F4D2C080E090E0B0
:10B51000A0E8BFEB88A799A7AAA7BBA72CA13DA12C
:10B520004EA15FA1CA01B9010F94E3524B015C0126
:10B53000A3019201C301B2010F94E3529B01AC013C
:10B54000C501B4010F946F590F941D5C4B015C0150
:10B55000AC019B01C701B6010F946E596CA77DA782
:10B560008EA79FA7A5019401C701B6010F946F593B
:10B570009B01AC016CA57DA58EA59FA50F94E35200
:10B580006B017C0120E030E0A9010F94CF5B87FDC7
:10B5900094C0C701B6010F941D5C6B017C01C3010F
:10B5A000B2019058A50194010F94695A28A539A5B4
:10B5B0004AA55BA50F94E352A70196010F94E352AD
:10B5C0002CA13DA14EA15FA10F946F5969837A838D
:10B5D0008B839C83A50194016CA17DA18EA19FA169
:10B5E0000F94695A28A539A54AA55BA50F94E35283
:10B5F000A70196010F94E352A30192010F946F5992
:10B600006D837E838F83988720E030E0A901698174
:10B610007A818B819C810F947D52811166C020E0DC
:10B6200030E0A9016D817E818F8198850F947D52D4
:10B6300081115BC00E9458458EE09FE00E94FE345D
:10B640002DC08430910509F463C0459739F10F94FA
:10B65000162C24C08A32910509F4ECC158F48C31BF
:10B66000910509F4AAC008F490C04D9781F70E9493
:10B67000AD7114C08B35910509F459C28C35910513
:10B6800009F459C28A35910511F71092660806C06F
:10B69000213021F40E9483300E949EF639A9311195
:10B6A00002C00F94A43588A9809350080C94CE66EC
:10B6B00080E090E0A0E8BFE32DCFC12CD12C760133
:10B6C0006ECF89E40E945130882331F00E94D92F37
:10B6D00069837A838B839C838AE40E945130882318
:10B6E00009F492CF0E94D92F8BCF412FBE016F5FFB
:10B6F0007F4F85E398E00F943D360F944335609378
:10B700004508709346088093470890934808C6CF31
:10B7100080E50E945130C12CD12C7601882321F084
:10B720000E9450256B017C0183E50E9451308823E3
:10B7300061F00E94D92F20E030E04AE754E40F94F2
:10B74000E3520F94E25A6B017C010E94C6DC8091A7
:10B750006413811105C060E084E29FE00E9454B24E
:10B760000F944335C60ED71EE81EF91E0F944335BD
:10B770006C197D098E099F0997FF90CF80E00E9488
:10B780000F4CF4CF0E94083C89CF0F94A442811142
:10B7900085CF8CE0E4E9F2E0DE01119601900D9294
:10B7A0008A95E1F770E060E080E50E945E30BE01BE
:10B7B0006F5F7F4F0F945A0171CF87E00E9478F03E
:10B7C000811106C060E08FE40E94C631811166CF0E
:10B7D0000E94C6DC1092380260919C108CE40E949A
:10B7E000C631982E80E00E94BA320F9443356093A0
:10B7F00045087093460880934708909348088091C5
:10B80000790290917A02A0917B02B0917C028093A0
:10B81000C3049093C404A093C504B093C60480915C
:10B820007302909174029093C2048093C10484E6E1
:10B8300090E0909374028093730281E08093C1073B
:10B840000E940BFC8AE50E940330A82E88E50E9426
:10B850000330182F89E50E940330B82E181308C052
:10B86000B12EA11205C011E0BB24B394AA24A39465
:10B8700082E50E945130882309F4D2C00E94D92F5A
:10B880006C8F7D8F8E8F9F8F20E030E0A9010F9409
:10B890007D52882349F0111103C0BB2009F494C0E4
:10B8A000CE014C960F94042E112309F488C0BB20BE
:10B8B00009F482C010929D1010929E1010929F1059
:10B8C0001092A0101092A1101092A2101092A3102A
:10B8D0001092A4100E9461F2E1ECF7E2C590D590BD
:10B8E000E590F490E5ECF7E2459055906590749002
:10B8F000A7019601C301B2010F947D5287FF95C045
:10B90000A7019601C301B2010F94695A9B01AC01D2
:10B910000F94E35220E030E040E85FE30F946F596A
:10B920000F941D5C20E030E048E452E40F94E352B1
:10B9300069837A838B839C838091A5109091A61054
:10B94000A091A710B091A8108CA39DA3AEA3BFA3F4
:10B9500020E030E040EC5FE3C301B2010F94E3521A
:10B960002B013C0177FA709477F8709420E030E076
:10B9700040EC5FE3C701B6010F94E3529058DE013B
:10B9800011966D01ECA0FDA00EA11FA1A3019201D3
:10B990000E9461F10E9476FD10929D1010929E10FF
:10B9A00010929F101092A0101092A1101092A2104D
:10B9B0001092A3101092A41080E00E94B8F9BB204E
:10B9C00019F081E00E94B8F9AA2019F082E00E94E3
:10B9D000B8F90E9461F28091C0078093C107892D58
:10B9E0000E94BA328091C3049091C404A091C5040E
:10B9F000B091C6048093790290937A02A0937B025F
:10BA0000B0937C028091C1049091C204909374021F
:10BA10008093730283E080937D020E9409FB3ECEF7
:10BA200060E070E080E890E42BCFA3019201C701B1
:10BA3000B6016ACF80910808813009F02FCE89E4E1
:10BA40000E945130082F10E0882319F00E94D52F52
:10BA5000182F8AE40E945130F82E882339F00E9472
:10BA6000D52F011106C0853068F005C080E00023A5
:10BA700049F0153028F08DE29FE00E94FE340ECE92
:10BA8000F110F1CF90E1EDE9F0E1A5E3B8E001902C
:10BA90000D929A95E1F7002391F0B4E01B02F001BA
:10BAA0001124EE55F94E408151816281738140939A
:10BAB0003508509336086093370870933808FF2094
:10BAC00091F024E08202F0011124E257F94E8081C6
:10BAD0009181A281B3818093390890933A08A09311
:10BAE0003B08B0933C0840E050E0BA0186E40E9475
:10BAF0006C306B017C0120E030E0A9010F94CF5B3A
:10BB000018168CF420E030E040E752E4C701B6019B
:10BB10000F94695A69837A838B839C83CE01019643
:10BB20000E9451F9BBCD60E070E0CB01F3CF8FE014
:10BB300080936608B3CD8091F304882381F1893026
:10BB400009F0ACCD60EAA62E62E0B62E7DE9C72EE4
:10BB500070E1D72EE12C00E010E0D5018D915D0160
:10BB60000E945130F82E882361F0133011F4082F11
:10BB7000FE2C0E94D92FF601608371838283938308
:10BB8000EF2C1F5FF4E0CF0ED11C143031F7EE2004
:10BB900009F457C00E9461F20E9409FB7FCD50EA70
:10BBA000C52E52E0D52EF12CE12C00E010E0D6019C
:10BBB0008D916D010E945130382E8823D9F10E9459
:10BBC000D92F4B015C01133059F0F701E15BF64FBF
:10BBD00020813181428153810F946E594B015C0168
:10BBE000F701E356FF4E2081318142815381C50127
:10BBF000B4010F946E592B013C012DEB37E346E85D
:10BC000055EB0F94CF5B87FD0AC02DEB37E346E879
:10BC100055E3C301B2010F947D5218165CF4133042
:10BC2000C1F48092A9109092AA10A092AB10B09289
:10BC3000AC10032D1F5FB4E0EB0EF11C143009F0C3
:10BC4000B6CF002309F4A8CF89EA90E10E9460EE04
:10BC5000A3CFF701EB57F74F5F01A301920160817A
:10BC60007181828193810F946F59D5016D937D937A
:10BC70008D939C931397812F0E9458F0DBCF809176
:10BC8000F4049091F5048837910511F40C94DC6864
:10BC900008F077C28D34910509F4ADC708F0D3C020
:10BCA0008A31910509F4CFC608F094C0843191051A
:10BCB00009F415C608F071C08131910509F4D6C5A3
:10BCC00008F044C0029708F0C2CC80E50E945130D1
:10BCD000C12CD12C7601882321F00E9450256B01C4
:10BCE0007C0183E50E945130882361F00E94D92FA6
:10BCF00020E030E04AE754E40F94E3520F94E25A14
:10BD00006B017C010E94C6DC8091F7049091F804DD
:10BD1000009709F4A5C50F9450428091F4049091C6
:10BD2000F5046EE47FE0892B11F466E47FE030E0F7
:10BD300020E04FE450E482E00E940D3640E0C7016D
:10BD4000B6010E94F0560F948242A8CC429709F0A7
:10BD50007ECC83E50E945130882311F40C94136843
:10BD60000F944335609345087093460880934708C5
:10BD7000909348080E94D92F20E030E04AE754E42D
:10BD80000F94E3520F94E25A6093100270931102E1
:10BD9000809312029093130281CC8731910509F4AC
:10BDA000D3C570F48531910509F4CAC5469709F0E9
:10BDB0004ECC8091C11682FD71CC0E9420D26ECCF7
:10BDC0008831910509F4D5C5499709F040CC0E9406
:10BDD000D65864CC8F31910509F4DAC6D0F48C3191
:10BDE000910509F49DC608F441C68D31910509F409
:10BDF0009FC64E9709F02BCC8091C11683FF4ECC85
:10BE00000F94FC2B8091F7049091F8040F941F413C
:10BE100045CC8934910509F4DAC650F48032910595
:10BE200009F48DC6819709F012CC0E944A4B36CC9A
:10BE30008B34910509F4DBC68C34910509F007CCED
:10BE40000E947EFE2BCC8B36910509F4C0C708F00A
:10BE50000FC18435910509F47CCF40F581359105FA
:10BE600011F40C94F36790F48E34910509F0EFCB44
:10BE700070E060E083E50E94B7318E34910509F0EF
:10BE8000BFC60E94ECDB0F94824208CC823591053C
:10BE900011F40C940B688335910509F0D8CB80918F
:10BEA00066088F7E806280936608F8CB883691059D
:10BEB00009F42AC708F09CC08535910511F40C944B
:10BEC00056688C35910509F0C2CB0E94454687FD26
:10BED000E5CB8091EF0484FD0AC08091F10487FDD9
:10BEE00006C08091F204837011F40C94846820EAF7
:10BEF000C22E22E0D22E34E5E32E30E1F32E10E004
:10BF0000D6018D916D010E945130882309F466C0DD
:10BF1000133011F00C947B680E94D92F4B015C0107
:10BF200020E030E040EA51E40F947D5287FF4EC09C
:10BF3000A501940160917410709175108091761034
:10BF4000909177100F94695A2B013C01AC019B0131
:10BF5000609181097091820980918309909184098F
:10BF60000F94E3526093810970938209809383094F
:10BF700090938409A30192016091841070918510BF
:10BF800080918610909187100F94E35260938410F3
:10BF900070938510809386109093871060916D093F
:10BFA00070916E0980916F09909170090F9482527F
:10BFB000A30192010F94E3520F94E25A60936D092A
:10BFC00070936E0980936F0990937009809274103A
:10BFD00090927510A0927610B09277101F5FF4E0E7
:10BFE000EF0EF11C143009F08BCF0E94A2DC56CB6F
:10BFF0008936910509F4C0C68A36910509F027CB28
:10C0000080E50F94382DF82E81E08F1508F446CB8B
:10C0100081E40E94033060918D09062F10E08111A8
:10C0200002C00FEF10E089E40E945130882311F420
:10C030000C94CB6E0E94B12F90E01816190614F4E0
:10C0400081E090E026E0289FF001299FF00D112467
:10C05000E75FF74F04811581EF2DF0E0E357F64FCE
:10C060000F3F110519F010F00FEF10E0008316CB11
:10C070008137910509F40DC708F068C08E36910527
:10C0800009F4B3C608F059C08C36910509F406CB03
:10C090008D36910509F0DBCA8091531083FDFECAED
:10C0A0000E944546F82E87FDF9CA89E40E94513066
:10C0B000882311F40C94B96E0E94B12F90E01816E9
:10C0C000190614F481E090E026E0289FF001299FF2
:10C0D000F00D1124E75FF74F8081918110E00E94FD
:10C0E00048DC61E081E00F9491462091D5153091B4
:10C0F000D6158091D3159091D415821793070CF023
:10C1000032C68FE390E19F938F938AE490E19F93EF
:10C110008F931F920E9439B20F900F900F900F9043
:10C120000F9001E00F945A46002309F4B7CA40E08B
:10C13000612F8F2D0F94280AB1CA8F36910509F40B
:10C1400067C68037910509F4A9CA81CA8537910568
:10C1500009F4E7C758F48237910509F4DAC7833741
:10C16000910509F074CA0E94253598CA8637910551
:10C1700009F4E9C78737910509F069CA0E94EFFB06
:10C180008DCA8039E1E09E0711F40C941B6C08F015
:10C19000ECC18D3C910511F40C94E66908F0A6C041
:10C1A0008B39910509F4F8C640F58D37910509F4EE
:10C1B0000ECE58F48937910509F049CA1092C1078B
:10C1C0001092C0070E940BFC69CA8C38910509F4D3
:10C1D0007FC68139910509F03ACA70E060E083E5D5
:10C1E0000E94B731823010F40C94E4680E945845E4
:10C1F00080EA90E10E94FE3451CA893C910511F415
:10C200000C945169B0F58E3B910509F487C6883CC2
:10C21000910509F01CCA0E944546182F87FD3ECAA9
:10C220000091840884E40E945130F82E8823C1F0E4
:10C230000E94D92F4B015C0120E030E0A9010F944E
:10C240007D52882311F40C944E6924E01202F0010F
:10C250001124E058F74F80829182A282B3820F2D81
:10C26000602F83E50E94C631809384080E94C1C379
:10C2700015CA8B3C910511F40C947B698C3C91059B
:10C2800009F0E5C98091F00487FF02C00C949E6913
:10C290008091F1048E7011F00C949E694091881089
:10C2A0005091891060918A1070918B1085EC90E10B
:10C2B0000E94E83640918C1050918D1060918E1044
:10C2C00070918F1082EC90E10E94E83640919010BE
:10C2D0005091911060919210709193108EE79CE2B2
:10C2E0000E94E8368AE00E94C534D8C9823221E033
:10C2F000920711F40C94576B80F58C3D910511F465
:10C300000C94BD6A60F48E3C910511F40C946D6A36
:10C31000833D910509F09BC90E946A46BFC98D3DC6
:10C32000910511F40C94006B8A3F910509F08FC9B7
:10C3300083E40E940330882321F00E94D52F0E94BD
:10C340007A26609151027091520281E591E10E943A
:10C35000FE3B8AE00E94C534A1C98E32A1E09A0753
:10C3600011F40C94D16B08F083C08C32E1E09E078D
:10C3700011F40C94B36B8D32914009F068C985E4D7
:10C380000F94382D81110C94C96B80E50E94033005
:10C39000882351F00E94D92F6093D8157093D91536
:10C3A0008093DA159093DB1589E40E94033088238B
:10C3B00081F00E94D92F2CEA35EC47E25EE30F941E
:10C3C000E3526093DC157093DD158093DE15909336
:10C3D000DF1584E40E940330882381F00E94D92F66
:10C3E0002CEA35EC47E25EE30F94695A6093E0155E
:10C3F0007093E1158093E2159093E3150E944146F6
:10C400004091D8155091D9156091DA157091DB15CE
:10C410008FE291E10E94E8362CEA35EC47E25EE3D8
:10C420006091DC157091DD158091DE159091DF151E
:10C430000F94695AAB01BC018BE291E10E94E8368E
:10C440002CEA35EC47E25EE36091E0157091E1156E
:10C450008091E2159091E3150F94E352AB01BC017A
:10C4600087E291E10E94E8368AE00E94C53416C94D
:10C470008F3221E0920711F40C94176C80339140B5
:10C4800009F0E5C880E50E940330882351F00E943E
:10C49000D92F6093740870937508809376089093F1
:10C4A000770889E40E940330882381F00E94D92F05
:10C4B0002CEA35EC47E25EE30F94E3526093780890
:10C4C0007093790880937A0890937B0884E40E94A3
:10C4D0000330882381F00E94D92F2CEA35EC47E203
:10C4E0005EE30F94695A60937C0870937D08809393
:10C4F0007E0890937F080E944146409174085091B5
:10C50000750860917608709177088DE491E10E943A
:10C51000E8362CEA35EC47E25EE3609178087091EA
:10C52000790880917A0890917B080F94695AAB0141
:10C53000BC0189E491E10E94E8362CEA35EC47E23F
:10C540005EE360917C0870917D0880917E089091F7
:10C550007F080F94E352AB01BC0185E491E10E9496
:10C56000E8368AE00E94C53499C8883FA1E09A075E
:10C5700011F40C944E6D08F047C08C3AE1E09E0730
:10C5800011F40C94236CC8F48D3921E0920711F456
:10C590000C947C6E28F48A39914009F47FC857C8FE
:10C5A000843AB1E09B0711F40C941F6C853A9140DA
:10C5B00009F04DC80E945C4571C8853FF1E09F07B6
:10C5C00011F40C94466D68F4863E31E0930711F443
:10C5D0000C94D46C843F914009F039C80E9498D8DB
:10C5E0005DC8863FB1E09B0711F40C944A6D873F0C
:10C5F000914009F02CC861E083E50E94C63191E0CA
:10C6000089270F94B60B4AC88C36F3E09F0709F4CC
:10C6100045C808F0D5C08B3532E0930711F40C946F
:10C62000716D70F48C30B2E09B0711F40C94606D66
:10C630008835924011F00C94275B0E94C6572EC893
:10C640008D3BF2E09F0711F40C94F16D8E3B92400C
:10C6500011F00C94275B0E944546182F87FD1EC8D9
:10C660008AE50E945130812C912C90E2A92E91E410
:10C67000B92E882341F040E050E0BA018AE50E94DB
:10C680006C304B015C01412F64E083E00E94C38465
:10C6900020E030E0A901C501B4010F94CF5B18166A
:10C6A0007CF580E090E0A0EAB0E489839A83AB83D4
:10C6B000BC832091A5103091A6104091A7105091F5
:10C6C000A810C501B4010F946F596B017C0120E0E3
:10C6D00030E04AE753E40F947D5287FD06C0C12C39
:10C6E000D12C8AE7E82E83E4F82ECC8EDD8EEE8EF8
:10C6F000FF8EBE016F5F7F4FCE014C960E9419F2F4
:10C7000085E50E940330882311F40C94F56D0E9496
:10C71000D92F6B017C0120E030E0A901C701B601EF
:10C720000F94CF5B87FF04C0F7FAF094F7F8F0940A
:10C73000F7FAF094F7F8F094C982DA82EB82FC827F
:10C7400044E061E0CE0101960E949D5520E030E07A
:10C75000A901C501B4010F94CF5B18165CF580E008
:10C7600090E0A0EAB0E489839A83AB83BC83A501FF
:10C7700094016091A5107091A6108091A7109091DE
:10C78000A8100F946E596B017C0120E030E0A901E4
:10C790000F94CF5B18161CF0C12CD12C7601CC8ED7
:10C7A000DD8EEE8EFF8EBE016F5F7F4FCE014C9609
:10C7B0000E9419F2109209050E94DA830C944E5BD4
:10C7C000873E33E0930711F40C946C6EC8F4843800
:10C7D000B3E09B0711F40C94016E803A934011F082
:10C7E0000C94275B2091F7043091F8049091C116C6
:10C7F00092609093C116C9010F94F9420C944E5B5C
:10C80000883EF3E09F0711F40C94956E893E9340A7
:10C8100011F00C94275B0F94C94181110C944E5B6D
:10C820000E94DB310F9487410E9484FD6D337105B6
:10C830008105910520F081E392E10E941F6F8DE256
:10C8400092E10E941F6F84EE8093010589E192E1DD
:10C850000E94FE3485E192E10E941F6F0C944E5BB2
:10C8600060E086E59FE00E9454B257CA8091EF04D1
:10C8700084FD17C08091F10487FD13C08091F204FC
:10C88000837079F460E089E69FE00E9454B25F987B
:10C890008A988091080181708093060112980C9407
:10C8A0004E5B88E50E94033081115F9889E50E9404
:10C8B000033081118A988AE50E940330882329F089
:10C8C0008091080181708093060185E40E94033005
:10C8D000882311F40C944E5B12980C944E5B80915B
:10C8E000C11683FF25C081E89FE00E94FE3480913D
:10C8F000C11683FF17C082EE96E10E9404D38BE13C
:10C90000E2EEF6E1DE01119601900D928A95E1F7D3
:10C9100070E060E0CE0101960F94A506CE0101966D
:10C920000E94033282E79FE00E94FE340C944E5B2B
:10C930000E94414682E99FE00E94FE340C944E5BC7
:10C940000E9431D20C944E5B8091F7049091F804D0
:10C95000FC012191222331F02032D9F7DF01119718
:10C960001C92F7CF60E00F944243109201050C94A3
:10C970004E5B83E50E945130882321F00E9471258F
:10C980000E94A42384E50E9451308823A9F00E94CC
:10C9900071256B017C010E942BFEC092BE05D092D6
:10C9A000BF05E092C005F092C105CD28CE28CF2862
:10C9B00019F081E08093650880914E068823F9F094
:10C9C00080E090E0A0EAB1E489839A83AB83BC83E2
:10C9D0001C8E1D8E1E8E1F8E18A219A21AA21BA2BB
:10C9E00010E000E020E0AE014F5F5F4FBE01645EEB
:10C9F0007F4FCE0180960E9431540C944E5B0E9472
:10CA00004934882381F00E9479CA0E946D348BEDED
:10CA100098E00F94D84010929611109297111092AE
:10CA200098111092991161E08EE19EE10E94C63545
:10CA300046EE5DE16CE97FE085E00F942F2D0F94C9
:10CA400082420C944E5B8091C11683FD02C00C940F
:10CA50004E5B83E50E945130882311F40C944E5BA9
:10CA60000E9471250E94A4230C944E5B83E40E94D3
:10CA70000330882361F182EB9FE00E94FE348091B5
:10CA800029188823F9F0BE016F5F7F4F86E298E195
:10CA90000E9497D2CE0101960E949ECECE010196B1
:10CAA0000F94224280912113882339F080E20E9462
:10CAB000C53481E293E10E949ECE8AE00E94C53493
:10CAC0000C944E5B88EA9FE00E94FE34F6CF83E52B
:10CAD0000E945130882301F10E94B12F182F8C330E
:10CAE00008F08CE38093CB040F9443356B017C01F9
:10CAF000212F30E0A8EEB3E00F941559C60ED71ED3
:10CB0000E81EF91EC092C704D092C804E092C9047E
:10CB1000F092CA040C944E5B0F949F400C944E5BB1
:10CB20008091F7049091F8040F94F9420C944E5BB5
:10CB30008091C1168E7F8093C1160C944E5B8091BC
:10CB4000C11682FD0E94C6DC8091C11683FD02C021
:10CB50000C944E5B60E080E50E94C631182F682F70
:10CB60008091F7049091F8040F94424383E50E946A
:10CB70005130882321F00E9471250E94A4230E9435
:10CB800079CA11110C944E5B0E946D340C944E5B6B
:10CB90000E9484FD6C8F7D8F8E8F9F8FBE016F5F93
:10CBA0007F4FCE014C960E94372ACE0101960F94FA
:10CBB00050420E944146BE016F5F7F4F81EC9FE073
:10CBC0000E94404B8AE00E94C5340C944E5B80E585
:10CBD0000E940330882311F40C944E5B0E94B12F05
:10CBE000853608F084E6809301050C944E5B0E9424
:10CBF0006D340C944E5B81E00E94B6FD0C944E5B4C
:10CC00008CE290E10E94FE346091B0077091B10710
:10CC100083E290E10E94D6366091B2077091B3072B
:10CC200086E190E10E94D6366091B0077091B1071D
:10CC30008091B2079091B307681B790B80916508CA
:10CC4000815021E030E0823010F030E020E0621BC3
:10CC5000730B8BE090E10E94D6368AE00E94C534C7
:10CC600083E090E10E94FE348091B4079091B50773
:10CC7000A091B607B091B7078C8F9D8FAE8FBF8FF5
:10CC8000BE016F5F7F4FCE014C960E94372ABE01D6
:10CC90006F5F7F4F86EF9FE00E94404B8091B80707
:10CCA0009091B907A091BA07B091BB078C8F9D8F67
:10CCB000AE8FBF8FBE016F5F7F4FCE014C960E943B
:10CCC000372ABE016F5F7F4F86EE9FE00E94404B88
:10CCD00020E030E04AE754E46091BC077091BD0762
:10CCE0008091BE079091BF070F94695AAB01BC01B8
:10CCF0008EEC9FE00E94E8368DE60E94C5348AE003
:10CD00000E94C5340C944E5B8091531083FF02C087
:10CD10000C944E5B0E94454687FF02C00C944E5B0C
:10CD200089E40E945130882311F40C94AE6E0E9465
:10CD3000B12F90E01816190614F481E090E026E077
:10CD4000289FF001299FF00D1124E75FF74F8081A4
:10CD500091810E9448DC61E080E00F9491460F943D
:10CD60005A460C944E5B84E390E1112309F4CBC93D
:10CD7000012FD8C9182FD6C90E944546182F87FD04
:10CD80000AC08FE490E10E94FE34812F0F94300896
:10CD90008AE00E94C53438A930935008E1960FB656
:10CDA000F894DEBF0FBECDBFDF91CF911F910F91E1
:10CDB000FF90EF90DF90CF90BF90AF909F908F90BB
:10CDC0007F906F905F904F903F902F90089580E5F7
:10CDD0000F94382D823010F00C944E5BE82FF0E069
:10CDE000E357F64F10820C944E5B8EE40E94513054
:10CDF000882311F40C944E5B0E94712560932F11CF
:10CE00007093301180933111909332110C944E5BDA
:10CE100083E50E940330882329F083E50F94382DA1
:10CE2000809353100E94414680E690E10E94FE34B8
:10CE300080915310882351F110E000E020E08091B0
:10CE4000531090E0B0E0A0E0002E04C0B695A79586
:10CE5000979587950A94D2F780FF12C0FF24F39428
:10CE6000F20E222319F08CE20E94C534F801EE0F75
:10CE7000FF1FEA5AFF4E859194910E94FE342F2D98
:10CE80000F5F1F4F05301105D1F617CE82E590E1F7
:10CE90001BCE83E50E945130882369F00E94B12F98
:10CEA0008D3320F480930F020C944E5B8CE38093BF
:10CEB0000F020C944E5B0E94414660910F0287E680
:10CEC00090E10E94E0368AE00E94C5340C944E5BEB
:10CED0008091531083FF02C00C944E5B89E40E9442
:10CEE0005130882309F463C70E94B12F90E01816CF
:10CEF000190614F481E090E026E0289FF001299FB4
:10CF0000F00D1124E75FF74F828193810E94A62FD5
:10CF100061E080E00F9491460C944E5B8091531039
:10CF200083FF02C00C944E5B89E40E945130882339
:10CF300009F447C70E94B12F90E01816190614F49F
:10CF400081E090E026E0289FF001299FF00D112458
:10CF5000E75FF74F8281938110E00E94A62F60E087
:10CF600081E00F9491462091710830917208809170
:10CF70006F0890917008821793071CF48DE790E179
:10CF800002C08EE690E160E00E9454B260E0812F22
:10CF90000F94A3080C944E5B83E50E9451308823C4
:10CFA00011F40C944E5B0E94B12F182F8C3308F0B3
:10CFB0008CE38093D0040F9443356B017C01212FC7
:10CFC00030E0A8EEB3E00F941559C60ED71EE81E48
:10CFD000F91EC092CC04D092CD04E092CE04F0921F
:10CFE000CF040C944E5B0E9421D50E94D7DC81E0D7
:10CFF0000E94B6FD0E94803468EE73E080E090E00D
:10D000000E94FA330E94B22160E08CE890E10E9415
:10D0100054B20C944E5B809166088F7D8061809342
:10D0200066080C944E5B8091EF0484FD0CC08091E7
:10D03000F10487FD08C08091F204837021F40E94FE
:10D04000D7DC0C944E5B0E94C6DC88E50E9403305E
:10D05000882331F05F9A8091C3078E7F8093C30746
:10D0600089E50E940330882331F08A9A8091C307B2
:10D070008D7F8093C3078AE50E940330882359F08F
:10D080008091080180958170809306018091C3078B
:10D090008B7F8093C30785E40E940330882311F4BB
:10D0A0000C944E5B0E94B0210C944E5B83E50E9471
:10D0B0000330882311F40C944E5B0F944335609336
:10D0C00045087093460880934708909348080E944B
:10D0D000D92F20E030E04AE754E40F94E3520F9454
:10D0E000E25A6093D1047093D2048093D304909356
:10D0F000D4040C944E5B0E94D92FF701648B758B7E
:10D10000868B978B0C94EE5F81E00F94C12B0C946F
:10D110004E5B0F945C2B89E296E10E94EED70C9453
:10D120004E5B8091F7049091F804009741F0DC0188
:10D130002C91222321F00F9450420C944E5B0F94BB
:10D1400082420C944E5B0091F7041091F80494E035
:10D15000F12C40E09150F9F0F8018081282F2B7FCD
:10D16000213499F421812133B1F4813411F18534D2
:10D1700009F441E098012E5F3F4F89012F5F3F4F37
:10D18000F80180818032C9F3E5CF803521F48181B7
:10D1900080538A3078F341110E944146FF2021F0EC
:10D1A0008DE990E10E94FE34C8010E94CC340C94B9
:10D1B0004E5BFF24F394DECF2093C1072093C0077A
:10D1C0000E940BFC0C944E5B8C01112788E40E949A
:10D1D00051308823C1F00E94D52F8A3A91050CF472
:10D1E0004BC00E94D52F843B91400CF048C00E9458
:10D1F000D52F26E0209FF001219FF00D1124E75F3D
:10D20000F74F9183808382E40E9451308823A9F0F4
:10D210000E94D52F0597B4F10E94D52F8D38910526
:10D22000A4F50E94D52F26E0209FF001219FF00D4C
:10D230001124E75FF74F9383828386E40E94513085
:10D24000882311F40C944E5B0E94D52F97FD20C0CB
:10D250000E94D52F8F3F910509F0ECF40E94D52F45
:10D2600026E0209FF001219FF00D1124E75FF74F8A
:10D27000958384830C944E5B8AEA90E0BACF83EB6B
:10D2800091E0B7CF85E090E0CECF8CE890E0CBCFB7
:10D2900090E080E0E5CF8FEF90E0E2CF80E00C946B
:10D2A00034610E94454687FF02C00C944E5B00EA41
:10D2B00012E084E5E82E80E1F82E94EAC92E92E08F
:10D2C000D92ED8018D918D010E940330882359F009
:10D2D0000E94D92F0F94E25AF701608371838283F1
:10D2E00093830E9454DCF4E0EF0EF11CC016D106CB
:10D2F00041F70C944E5B0E94454687FF02C00C9498
:10D300004E5BB0EAEB2EB2E0FB2E10E000E0D7015E
:10D310008D917D010E940330882349F00E94D92F0E
:10D32000F801EC5AFF4E64A375A386A397A30C5F84
:10D330001F4F0031110559F70C944E5B83E50E9495
:10D340005130882391F00E94D92F609388107093F8
:10D35000891080938A1090938B1060939010709333
:10D360009110809392109093931080E50E94513019
:10D37000882351F00E94D92F6093881070938910F0
:10D3800080938A1090938B1082E50E9451308823FD
:10D3900051F00E94D92F60938C1070938D10809360
:10D3A0008E1090938F1084E50E945130882311F4E1
:10D3B0000C944E5B0E94D92F609390107093911043
:10D3C00080939210909393100C944E5B8091EF0495
:10D3D000827151F48091F1048C7831F48091F204DF
:10D3E000837011F40C944E5B82E40E940330882316
:10D3F00051F00E94502560936410709365108093E3
:10D4000066109093671083E50E940330882351F0E3
:10D410000E94D92F6093941070939510809396106A
:10D420009093971084E50E940330882351F00E9466
:10D43000D92F609398107093991080939A109093BD
:10D440009B1088E50E940330882351F00E94D92F59
:10D4500060937509709376098093770990937809A2
:10D4600089E50E940330882351F00E94D92F6093F0
:10D47000790970937A0980937B0990937C098AE5F6
:10D480000E9403308823B1F00E94D92F60937D0958
:10D4900070937E0980937F09909380092DEC3CEC7A
:10D4A0004CEC5DE30F947D52181624F085ED90E16D
:10D4B0000E94FE3485E40E940330882311F40C940A
:10D4C0004E5B0E94D92F60938109709382098093EB
:10D4D0008309909384090C944E5BA1E9EA2EA8E09D
:10D4E000FA2E10E088E5810F0E940330882351F066
:10D4F0000E94D92FF7016083718382839383812FE8
:10D500000E9458F01F5FF4E0EF0EF11C133051F74A
:10D510008091F10487FF02C00C94CC5D8091F204ED
:10D52000837011F00C94CC5D409191085091920859
:10D53000609193087091940887E091E10E94E83629
:10D5400040919508509196086091970870919808BD
:10D5500088ED90E40E94E8364091990850919A082D
:10D5600060919B0870919C0885ED90E40E94E836DC
:10D570008AE00E94C5340C944E5B82E40E94033022
:10D58000882341F080917302909174029093150268
:10D590008093140282E50E940330882341F0809139
:10D5A000140290911502909374028093730283E5A4
:10D5B0000E945130882331F00E94D52F909374023D
:10D5C000809373028091EF049091F004A091F10494
:10D5D000B091F204892B8A2B8B2B11F00C944E5BAB
:10D5E00060917302709174028EE091E10E94FE3BA3
:10D5F00085E20E94C5348AE00E94C5340C944E5BDB
:10D600000E944546082F87FF02C00C944E5B83E5BD
:10D610000E945130002E000C110B7801EE0CFF1C03
:10D62000882359F10E94D52FF701EB5CFD4F9183C0
:10D630008083000F111F000F111F980122583D4FCA
:10D640007901BC01990F880B990B0F9484522AE041
:10D6500037ED43E25CE30F94E35206541A4FD801CE
:10D660002D913D914D915C910F94E352F7016083B0
:10D670007183828393830C944E5B0E94414685E4C0
:10D680000E94C53480E3800F0E94C534F701EB5C33
:10D69000FD4F6081718182E191E10E94FE3B85E254
:10D6A0000E94C5348AE00E94C5340C944E5B8AE522
:10D6B0000E945130882331F10E94D92F20E030E0C0
:10D6C00040E050EC0F947D5287FD3CC00E94D92F62
:10D6D00020E030E040E050E40F94CF5B1816BCF13E
:10D6E0000E94D92F209170103091711040917210CA
:10D6F000509173100F94E3520F94DB5ACB010F94A7
:10D70000F73505C083E50E9451308111D5CF809156
:10D71000F10487FD21C08091F2048370E9F40E9436
:10D720004146409133065091340660913506709120
:10D7300036068AE191E10E94E8368AE00E94C5340B
:10D740000C944E5B60E070E080E090ECCBCF60E04A
:10D7500070E080E090E4C6CF82E50E940330811142
:10D76000DECF0C944E5B64E071E083E50E945E3096
:10D770008C0168EE73E080E50E945E308938F3E149
:10D780009F0710F088E893E1B8010E941E7D0C9479
:10D790004E5B0E94584583E391E10E94FE340C9455
:10D7A0004E5B83E50E940330182F882369F00E94A6
:10D7B000D52F9C01909383028093820291E0232BCA
:10D7C00009F090E090939F0980E50E940330882340
:10D7D00061F02091820230918302232B11F00E948C
:10D7E000C52F80939F090C944E5B11110C944E5BD6
:10D7F0000E9441468CE791E10E94FE3480919F098E
:10D80000882391F084E691E10E94FE3460918202C7
:10D81000709183028BE691E10E94FE3B87E691E1E5
:10D820000E94FE340C944E5B80E691E1EDCF0E94A5
:10D830000A370C944E5B0E94C6DC0C944E5B0E942F
:10D8400059470C944E5B0F94A44281110C944E5B8B
:10D8500070E9C72E77E2D72E2DE930E13DA32CA346
:10D86000CE0101961C017C0110E000E0F6016591FB
:10D87000759185919491ACA1BDA18D909D90AD9035
:10D88000BD90BDA3ACA3A50194010F946E592B01CB
:10D890003C01F701408251826282738220E030E0D5
:10D8A00040EA51EC0F94CF5B87FD0AC020E030E0E6
:10D8B00040EA51E4C301B2010F947D52181684F47A
:10D8C000F801E15FFF4BE4911E1654F4B7FAB094EF
:10D8D000B7F8B094D7018D929D92AD92BC921397F8
:10D8E000F70181909190A190B1907F0120E030E00C
:10D8F00040EA51ECC501B4010F94CF5B87FD3FC0F6
:10D9000020E030E040EA51E4C501B4010F947D52BB
:10D910001816ACF10F5F1F4FF4E0CF0ED11C03308F
:10D92000110509F0A3CF61E9E62E68E0F62E10E0BC
:10D93000F10181919191A191B1911F01F701819321
:10D940009193A193B1937F01812F0E9458F01F5FA3
:10D95000133071F70E9409FB60E08FE891E10E94AB
:10D9600054B263E972E084E690E00E941E7D6AEBA7
:10D9700072E084E690E00E941E7D0C944E5B0E9453
:10D9800058458DEA91E10E94FE3461E08FE991E112
:10D990000E9454B20E94DA8368E270E088EC90E062
:10D9A0000E941E7D0C944E5B84E50E940330882308
:10D9B000A1F0109203051092040510920505109233
:10D9C0000605109207058FEF0E94B22361E070E018
:10D9D00084E50E94B7318093070583E50E940330F8
:10D9E000882321F00E94D52F0E94B22383E40E9455
:10D9F0000330882331F080912302803210F40E949A
:10DA00007E3280E50E940330882331F00E94D52FBA
:10DA1000803210F40E947E3285E50E940330882314
:10DA200011F40C944E5B0E94D52F803210F00C94B0
:10DA30004E5B41E050E060E070E0082E04C0440F0F
:10DA4000551F661F771F0A94D2F740955095609531
:10DA50007095009103051091040520910505309102
:10DA600006054023512362237323409303055093FB
:10DA700004056093050570930605909123028913B0
:10DA80000C944E5B109252100C944E5B0F94DD126E
:10DA90000C944E5B0E9416FC0C944E5B2093370650
:10DAA0000F94D11210923706882311F40C944E5B18
:10DAB0000E9441468BEC91E10E94FE340C944E5B37
:10DAC0008091C11682FF05C080648093C1160C94BA
:10DAD0004E5B83FD02C00C944E5B0F94FC2B0C94A8
:10DAE0004E5B0E944546082F87FF02C00C944E5B98
:10DAF00085E50E940330882359F10E94D92F4B01FC
:10DB00005C01E02E002E000CFF0820E030E0A901AF
:10DB10000F94CF5B87FF04C0B7FAB094B7F8B09406
:10DB200020E030E84BE354E4C501B4010F94CF5B2F
:10DB3000970153E0220F331F5A95E1F72A533A4FCA
:10DB40001816D4F1D9018D929D92AD92BC92139783
:10DB50008CE40E940330882311F40C944E5B0E94E5
:10DB6000D92F6B017C01002E000C110B20E030E05E
:10DB7000A9010F94CF5B87FF04C0F7FAF094F7F880
:10DB8000F09420E030E84BE354E4C701B6010F9471
:10DB9000CF5B980143E0220F331F4A95E1F72A53E8
:10DBA0003A4F18169CF0D9011496CD92DD92ED9261
:10DBB000FC9217970C944E5B80E090E8ABE3B4E4E2
:10DBC000F90180839183A283B383C2CF80E090E880
:10DBD000ABE3B4E4F90184839583A683B7830C9403
:10DBE0004E5B0E9438530C944E5B28E01202F00109
:10DBF0001124EA53FA4FC080D180E280F3800C9464
:10DC00008B63A0908509B0908609C0908709D09059
:10DC100088098BE40E945130882339F10E94D92F62
:10DC20007B018C0120E030E0A9010F94CF5B87FDE0
:10DC30000AC020E030E040E251E4B701C8010F948F
:10DC40007D521816A4F48FE30E94C5348BE40E9421
:10DC5000C53481EE91E10E94FE3489ED91E10E948C
:10DC6000FE3486ED91E10E94FE3475018601970134
:10DC7000A801B501C6010F947D52882361F00E946E
:10DC8000C6DCC701D8018093850990938609A093CB
:10DC90008709B09388098091EF049091F004A091D6
:10DCA000F104B091F204892B8A2B8B2B11F00C9488
:10DCB0004E5B0E94414640918509509186096091D2
:10DCC00087097091880985EF91E10E94E8368AE022
:10DCD0000E94C5340C944E5B81E08093080810923A
:10DCE000B91360E083E50E94C63181110C944E5B4C
:10DCF0000F94032A0C944E5B83E50E940330882323
:10DD000041F00E94C52F8093CE050E94E3310C9410
:10DD10004E5B0E94414680E092E10E94FE34809179
:10DD2000CE050E94CA360C944E5B0E94916F0C94F3
:10DD30004E5B1091F4040F94433560934508709343
:10DD400046088093470890934808112311F40C94D7
:10DD50004E5B812F0E94D7D40C944E5B83E50E94CA
:10DD60005130882311F40C94AF660E94D52F0C9487
:10DD7000A96683E50E945130182F811108C082E501
:10DD80000E945130082F882311F40C94BA660E9427
:10DD9000D52F0C946F6083E50E945130882311F4D5
:10DDA0000C942C600E9471258B010C942C6083E5EF
:10DDB0000E945130882311F40C944E5B0E94D52FA1
:10DDC000A5C883E50E945130182F811107C082E554
:10DDD0000E945130882311F40C944E5B0E94D52F81
:10DDE000BCC8DF92EF92FF920F931F93CF93DF9304
:10DDF000EC01E0905208F09053088AE0D82E6AE0D7
:10DE000070E0CE010F94BD5C8C01009711F0FC0115
:10DE10001082CE010E94162B81E00E94B659011596
:10DE2000110519F0E801D992EACFC701DF91CF912E
:10DE30001F910F91FF90EF90DF900C94162B4F9253
:10DE40005F926F927F928F929F92AF92BF92CF928A
:10DE5000DF92EF92FF920F931F93CF93DF93CDB793
:10DE6000DEB77C014DB65EB66090520870905308E4
:10DE70008DB69EB66AE070E0C7010F94B8516C0190
:10DE80008C010E191F09892B21F4C7010F94CA5167
:10DE90008C01C80101962DB73EB7281B390B0FB670
:10DEA000F8943EBF0FBE2DBF8DB79EB701965C01A3
:10DEB000A801B7010F94EB51F501E00FF11F10829B
:10DEC000C5010E94162B81E00E94B659C114D104ED
:10DED00051F076019FEFE91AF90A0FB6F8949EBE49
:10DEE0000FBE8DBEC5CF0FB6F8949EBE0FBE8DBEC1
:10DEF000C3010E94162B0FB6F8945EBE0FBE4DBE36
:10DF0000DF91CF911F910F91FF90EF90DF90CF9015
:10DF1000BF90AF909F908F907F906F905F904F9049
:10DF200008954F925F926F927F928F929F92AF92DD
:10DF3000BF92CF92DF92EF92FF920F931F93CF93F6
:10DF4000DF93CDB7DEB7C059D1090FB6F894DEBF65
:10DF50000FBECDBF0E94F131882369F083E50E9496
:10DF60000330882301F120E040E070E060E084E0CD
:10DF700094E80E94C67FC057DF4F0FB6F894DEBF0B
:10DF80000FBECDBFDF91CF911F910F91FF90EF900A
:10DF9000DF90CF90BF90AF909F908F907F906F90C9
:10DFA0005F904F90089583E40E940330882319F016
:10DFB0000E94F983E0CF8090440990904509A09099
:10DFC0004609B090470980914D0980FF05C09091A6
:10DFD00053109860909353108695817080939F0999
:10DFE00080EF9EE00E941F6F8091D3089091D4082B
:10DFF0009E012F5F3F4F7901009799F09F938F9378
:10E0000087EE9EE09F938F933F932F930F9414522C
:10E01000C7010E94F16E0F900F900F900F900F901C
:10E020000F908091D1089091D208009799F09F931A
:10E030008F938EED9EE09F938F93FF92EF920F94BC
:10E040001452C7010E94F16E0F900F900F900F9025
:10E050000F900F906E0131E8C30ED11C6091B00893
:10E060007091B1088091B2089091B308860123E0C5
:10E0700041E00F944A4D9F938F938CEC9EE09F93C9
:10E080008F93FF92EF920F941452C7010E94F16E8A
:10E0900084EC9EE00E941F6F87E08093C30780930B
:10E0A000B1050F900F900F900F900F900F908091EF
:10E0B000CC088823F9F06091CD087091CE0880914A
:10E0C000CF089091D00823E041E00F944A4D9F93F0
:10E0D0008F938BEB9EE09F938F93FF92EF920F9421
:10E0E0001452C7010E94F16E0F900F900F900F9085
:10E0F0000F900F908091D5088823A1F01F928F93E5
:10E100001F921F928EEA9EE09F938F93FF92EF9251
:10E110000F941452C7010E94F16E0FB6F894DEBF3F
:10E120000FBECDBF8091D6088823A9F01F928F9390
:10E130001F9281E08F938EEA9EE09F938F93FF92D0
:10E14000EF920F941452C7010E94F16E0FB6F8942B
:10E15000DEBF0FBECDBF4090D7085090D80860906A
:10E16000D9087090DA0820E030E0A901C301B201BB
:10E170000F947D52811104C080914D0982FF20C00F
:10E18000860121E041E0C301B2010F944A4D9F9303
:10E190008F9380914D0982FB882780F91F928F937E
:10E1A00081EA9EE09F938F93FF92EF920F94145217
:10E1B000C7010E94F16E0FB6F894DEBF0FBECDBF4F
:10E1C0006091A2087091A3088091A4089091A5087D
:10E1D0008E010F581F4F23E041E00F944A4D782ED7
:10E1E000692E60919E0870919F088091A00890917F
:10E1F000A108860123E041E00F944A4D6F927F927F
:10E200009F938F9380E99EE09F938F93FF92EF926D
:10E210000F941452C7010E94F16E6091A60870918C
:10E22000A7088091A8089091A90823E041E00F94E5
:10E230004A4D85E89EE00E941F6FDF92CF928BE7E8
:10E240009EE09F938F93FF92EF920F941452C70119
:10E250000E94F16E8091AF088F938091AE088F93EA
:10E2600084E79EE09F938F93FF92EF920F94145256
:10E27000C7010E94F16E6091AA087091AB0880916D
:10E28000AC089091AD0823E041E00F944A4D9F9374
:10E290008F938AE69EE09F938F93FF92EF920F9465
:10E2A0001452C7010E94F16E8CE0E4EBF8E0A1E9A2
:10E2B000B8E001900D928A95E1F78CE0E0ECF8E08F
:10E2C000A5E8B8E001900D928A95E1F780E00E9400
:10E2D00058F081E00E9458F082E00E9458F080914E
:10E2E0004C098093660881E08093CE050E94E3315B
:10E2F0008BED98E09F938F9380EC97E39F938F93A0
:10E30000FF92EF920F9414520FB6F894DEBF0FBE37
:10E31000CDBFC7010E94F16E80914B098F93809110
:10E320004A098F93809149098F93809148098F936F
:10E33000BF92AF929F928F928CE59EE09F938F93B6
:10E34000FF92EF920F941452C7010E94F16E0FB624
:10E35000F894DEBF0FBECDBF0ECE4F925F926F928C
:10E360007F928F929F92AF92BF92CF92DF92EF9265
:10E37000FF920F931F93CF93DF9300D000D01F9293
:10E380001F92CDB7DEB783E50F94382D863028F085
:10E3900083EE9DE00E94FE343FC0833009F464C1E7
:10E3A000B0F4813021F1823009F450C080ED9DE05D
:10E3B0000E94FE340E94B5338823A1F080919C1006
:10E3C0000E94CA360E944B360E9409FB25C0843049
:10E3D00009F490C1853051F780E00E94BA320E9462
:10E3E000AA32F2CF82EC9DE00E94FE34EDCF0E9473
:10E3F000AA3210920E0210920D0280910205811134
:10E4000025C08EE40E94033081111DC080EB9DE089
:10E410009093C6078093C50728960FB6F894DEBF81
:10E420000FBECDBFDF91CF911F910F91FF90EF9065
:10E43000DF90CF90BF90AF909F908F907F906F9024
:10E440005F904F90089586EB9DE0E2CF80910D02A2
:10E4500090910E0297FF03C087E89DE09BCF009745
:10E4600009F0A8C01D821E821F8218868DEC9CECCC
:10E47000ACE4BEE389839A83AB83BC83BE016B5F4C
:10E480007F4FCE0101960E9419F280910D0290916A
:10E490000E02893191050CF0B3C021E020933802BF
:10E4A0009C012F5F3F4F30930E0220930D0265E0D9
:10E4B0000F94305980FF03C024E0291B922F24E0E1
:10E4C0009202F0011124EE55F94E80809180A280D5
:10E4D000B38094E08902F0011124E257F94E4080A4
:10E4E0005180628073808DEC9CECACE4BEE38D8344
:10E4F0009E83AF83B88719821A821B821C82CE0149
:10E5000001966C01E12CF12C00EA10E4A3019201C8
:10E51000C501B4010E9461F119821A821B821C821A
:10E52000B601CE0105960E9419F280929D1090923C
:10E530009E10A0929F10B092A0104092A1105092F5
:10E54000A2106092A3107092A41010920205009184
:10E550000D0210910E0289E1E82EF12C093111050E
:10E560000CF47801B70180E29DE00E94FE3B69E176
:10E5700070E08BE19DE00E94FE3B8AE00E94C53482
:10E58000101611060CF020CF1F9289E18F93FF9295
:10E59000EF9284E09DE09F938F9382E19DE09F93B3
:10E5A0008F931F920E9439B20FB6F894DEBF0FBE50
:10E5B000CDBF0ACF815065E00F94305980FF03C072
:10E5C00024E0291B922F25E09202F0011124E80F8C
:10E5D000F11D87FDFA95EE0FFF1FEE0FFF1FE153B0
:10E5E000FA4F8091A5109091A610A091A710B0911C
:10E5F000A81080839183A283B3831092380245CF01
:10E6000080E090E0A0EAB0E48093A5109093A6107B
:10E61000A093A710B093A81089E792E00E9446F15A
:10E620000E94C6DC8FEF9FEF90930E0280930D0245
:10E6300083E79DE00E94FE3481E69DE00F94504206
:10E6400063E972E084E690E00E941E7D6AEB72E06E
:10E6500084E690E00E941E7D8BE59DE00E941F6F86
:10E6600081E00E94BA3271CF89E40E945130882340
:10E6700071F00E94D52F182F853068F064E070E0AB
:10E6800088E49DE00E94FE3B85E49DE083CE8AE421
:10E690000E94C035C1CE8AE40E9451308823B9F36C
:10E6A0000E94D52F082F853048F064E070E082E3A7
:10E6B0009DE00E94FE3B8FE29DE06CCE8AE50E94C9
:10E6C00051308823A9F00E94D92F25E01202F001D1
:10E6D0001124E00FF11D07FDFA95EE0FFF1FEE0F5D
:10E6E000FF1FE153FA4F60837183828393836CCE63
:10E6F0008AE5CECF8AE50E9451308823C9F30E9473
:10E70000D92F609333067093340680933506909327
:10E7100036065ACECF93DF93C0919B11C093600908
:10E7200081E6C89FE0011124C356DE4E809153104C
:10E7300080FF05C00E944146CE010E94CC34CE012C
:10E740000E94162B80E0DF91CF910C94B6598F92E6
:10E750009F92AF92BF92CF92DF92EF92FF92CF93B0
:10E760006B017C0120E030E0A9010F947D5287FF0E
:10E77000A3C06DEB77E386E095EBA70196010F94BC
:10E780006F596B017C0120E030E040E251E40F94CE
:10E79000E35220E030E048EC52E40F94E3524B01A6
:10E7A0005C0120E030E040E251ECC701B6010F947B
:10E7B0007D52181654F420E030E048EC52E4C701D2
:10E7C000B6010F94CF5B87FD8BC020E030E0A9013C
:10E7D000C701B6010F947D5287FF73C060E070E0FF
:10E7E00080EA90ECA50194010F946F5920E030E08D
:10E7F00040E251E40F94695A0F94DB5A6B017C019B
:10E80000F7FC64C020E137E240E050E00F94E358A9
:10E81000CA01B9012AE030E040E050E00F94E3582B
:10E82000605D6093AA05C701B60128EE33E040E0C1
:10E8300050E00F94E3589AE0892E912CA12CB12C32
:10E84000CA01B901A50194010F94E358605D60937A
:10E85000AB05C701B60124E630E040E050E00F947C
:10E86000E358CA01B901A50194010F94E358605D12
:10E870006093AC058EE28093AD05C701B601A5019A
:10E8800094010F94E358C62FCA01B901A501940160
:10E890000F94E358605D6093AE05C05DC093AF0513
:10E8A0008AEA95E0CF91FF90EF90DF90CF90BF90F4
:10E8B000AF909F908F9008956DEB77E386E095E39E
:10E8C0005CCF60E070E080EA90E48CCFF094E0945C
:10E8D000D094C094C11CD11CE11CF11C6DE2A1CFED
:10E8E00020E030E0A901C701B6010F947D5287FFF7
:10E8F0006AC060E070E080EA90ECA50194010F949A
:10E900006F5920E030E040E251E40F94695A0F94CF
:10E91000DB5A4B015C0120E030E0A901C701B601E0
:10E920000F94CF5B87FD0BC020E030E040E251E464
:10E93000C701B6010F947D5260E287FD13C0B7FC9A
:10E9400047C0C501B40128EE33E040E050E00F9429
:10E95000E358CA01B9012AE030E040E050E00F94EA
:10E96000E358605D6093AB05C501B40124E630E077
:10E9700040E050E00F94E3588AE0C82ED12CE12CFF
:10E98000F12CCA01B901A70196010F94E358605D0B
:10E990006093AC058EE28093AD05C501B401A7017B
:10E9A00096010F94E358C62FCA01B901A701960139
:10E9B0000F94E358605D6093AE05C05DC093AF05F2
:10E9C0008BEA95E06FCF60E070E080EA90E495CF4D
:10E9D000B094A09490948094811C911CA11CB11CB3
:10E9E0006DE2C0CF6091350270913602072E000CA7
:10E9F000880B990B0F9484522AE037ED43E25CE3D5
:10EA00000F94E3522091BA053091BB054091BC05AB
:10EA10005091BD050F94E35260937E0270937F0284
:10EA200080938002909381020895E0913008E23053
:10EA300030F4F0E0E357F64F809126088083089584
:10EA40008091B6168823C1F081508093B616E2EE0D
:10EA5000F6E1882351F08150990B2BE1289FF001BA
:10EA6000299FF00D1124E85EF84E8BE1ADEFB6E181
:10EA700001900D928A95E1F72091B616211105C0FB
:10EA80008091C11680628093C11681E090E0A0E081
:10EA9000B0E0211103C080E090E0DC0180931E080B
:10EAA00090931F08A0932008B09321081092230888
:10EAB00081E080931D0883E080937D020895CF93C9
:10EAC000DF93EC01CB01BA010F94845229EC38ECAE
:10EAD00048EC5EE30F94695A20E030E040E05FE3E9
:10EAE0000F946F590F94E25A6883DF91CF91089584
:10EAF00080915102909152020C947A26E091300854
:10EB000086E0E802F0011124E75FF74F80912608C4
:10EB100090E0958384830895CF93DF93EC01CB013C
:10EB2000BA010F94845220E030E0A9010F946F598C
:10EB30000F94E25A6883DF91CF9108958F929F924C
:10EB4000AF92BF92CF92DF92EF92FF92CF936B0181
:10EB50007C0120E030E0A9010F947D5287FD9FC029
:10EB60006DEB77E386E095E3A70196010F946F596B
:10EB70006B017C0120E030E040E251E40F94E3526D
:10EB800020E030E048EC52E40F94E3524B015C018A
:10EB900020E030E0A901C701B6010F947D5220E0CA
:10EBA00030E040EA50E487FF04C020E030E040EA73
:10EBB00050ECC501B4010F946F5920E030E040E201
:10EBC00051E40F94695A0F94DB5A6B017C018BE27C
:10EBD000F7FE09C0F094E094D094C094C11CD11CFD
:10EBE000E11CF11C8DE28093A905C701B60120E16B
:10EBF00037E240E050E00F94E3588AE0882E912CF1
:10EC0000A12CB12CCA01B901A50194010F94E358BC
:10EC1000605D6093AA05C701B60128EE33E040E0CD
:10EC200050E00F94E358CA01B901A50194010F9473
:10EC3000E358605D6093AB05C701B60124E630E0A0
:10EC400040E050E00F94E358CA01B901A5019401D6
:10EC50000F94E358605D6093AC058EE28093AD0540
:10EC6000C701B601A50194010F94E358C62FCA014C
:10EC7000B901A50194010F94E358605D6093AE055E
:10EC8000C05DC093AF0589EA95E0CF91FF90EF900A
:10EC9000DF90CF90BF90AF909F908F9008956DEBD5
:10ECA00077E386E095EB60CF8F929F92AF92BF9211
:10ECB000CF92DF92EF92FF92CF936B017C0120E025
:10ECC00030E0A9010F947D5287FDAAC06DEB77E378
:10ECD00086E095E3A70196010F946F596B017C01C3
:10ECE00020E030E0A9010F947D5287FF9EC0C7014C
:10ECF000B601905820E030E040E251E40F94E35236
:10ED000020E030E040E251E40F94E35220E030E0B4
:10ED100040EA50E40F946F5920E030E040E251E4C3
:10ED20000F94695A0F94DB5A6B017C0180E2809347
:10ED3000A90560E280E1C81687E2D806E104F10483
:10ED40008CF0C701B60120E137E240E050E00F94BB
:10ED5000E358CA01B9012AE030E040E050E00F94E6
:10ED6000E358605D6093AA0560E288EEC81683E010
:10ED7000D806E104F1048CF0C701B60128EE33E0B7
:10ED800040E050E00F94E358CA01B9012AE030E0B6
:10ED900040E050E00F94E358605D6093AB0560E2A3
:10EDA00084E6C816D104E104F1048CF0C701B60171
:10EDB00024E630E040E050E00F94E358CA01B90186
:10EDC0002AE030E040E050E00F94E358605D60934B
:10EDD000AC058AE0882E912CA12CB12CC701B6017C
:10EDE000A50194010F94E358C62FCA01B901A501EA
:10EDF00094010F94E358605D6093AD058EE28093BB
:10EE0000AE05C05DC093AF0589EA95E0CF91FF9054
:10EE1000EF90DF90CF90BF90AF909F908F9008952C
:10EE20006DEB77E386E095EB55CF20E030E040E2F4
:10EE300051E4C701B60162CFCF93DF93EC01CB0160
:10EE4000BA010F94845220E030E040E251E40F9484
:10EE5000695A20E030E0A9010F946F5968837983E3
:10EE60008A839B83DF91CF910895CF93DF93EC0149
:10EE7000CB01BA010F94845220E030E040E251E42B
:10EE80000F94695A20E030E0A9010F946F5968830C
:10EE900079838A839B83DF91CF9108950F94845265
:10EEA00020E030E040E251E40F94695A20E030E085
:10EEB000A9010F946F590C945476CF93DF93EC0112
:10EEC000CB01BA010F94845220E030E0A9010F94E5
:10EED0006F59688379838A839B83DF91CF910895EB
:10EEE000CF93DF93EC01CB01BA010F94845220E061
:10EEF00030E0A9010F946F59688379838A839B83DB
:10EF0000DF91CF910895CF93DF93EC01CB01BA014C
:10EF10000F9484522AE037ED43E25DE30F94695A7F
:10EF200020E030E0A9010F946F590F94E25A6883F2
:10EF300079838A839B83DF91CF910895CF93DF9369
:10EF4000EC01CB01BA010F9484522AE037ED43E281
:10EF50005DE30F94695A20E030E0A9010F946F59E6
:10EF6000688379838A839B83DF91CF910895CF93C0
:10EF7000DF93EC01CB01BA010F94845220E030E022
:10EF8000A9010F946F59688379838A839B83DF91EA
:10EF9000CF910895CF93DF93EC01CB01BA010F9489
:10EFA000845220E030E048EC52E40F94695A20E0AB
:10EFB00030E0A9010F946F59688379838A839B831A
:10EFC000DF91CF910895CF93DF93EC01CB01BA018C
:10EFD0000F94845220E030E048EC52E40F94695AD8
:10EFE00020E030E0A9010F946F59688379838A8308
:10EFF0009B83DF91CF9108950F94845220E030E0FD
:10F0000048EC52E40F94695A20E030E0A9010F94D3
:10F010006F590C949E75CF93DF93EC01CB01BA012D
:10F020000F94845220E030E0A9010F946F590F949F
:10F03000DB5A79836883DF91CF910895CF93DF9373
:10F04000EC01CB01BA010F94845220E030E04AE792
:10F0500054E40F94695A20E030E0A9010F946F59ED
:10F06000688379838A839B83DF91CF9108950F947E
:10F07000845220E030E048EC52E40F94695A20E0DA
:10F0800030E0A9010F946F590C94A7732CEA35EC6A
:10F0900047E25EE36091970570919805809199052C
:10F0A00090919A050F94695A6093E0157093E11559
:10F0B0008093E2159093E31508952CEA35EC47E22E
:10F0C0005EE360919B0570919C0580919D059091F8
:10F0D0009E050F94E3526093DC157093DD158093C9
:10F0E000DE159093DF1508952CEA35EC47E25EE3D8
:10F0F00060919705709198058091990590919A0576
:10F100000F94695A6093E0157093E1158093E215AE
:10F110009093E31508952CEA35EC47E25EE36091A5
:10F120009B0570919C0580919D0590919E050F9483
:10F13000E3526093DC157093DD158093DE15909398
:10F14000DF150895E0919005E63010F581E08E0F0F
:10F150008093900540911E0850911F0860912008EF
:10F16000709121089091230880911C0828E0E29F6B
:10F17000F0011124EF5AFA4F20914D1630914E169E
:10F18000318320834283538364837583968387838B
:10F190000895FC01A081B1811C92A281B3818C9160
:10F1A0008F5F8C930280F381E02D90818CE0989F9B
:10F1B000800D1124EFE4F6E113AE84AF0895CF92F1
:10F1C000DF92EF92FF92CF93DF9300D01F92CDB7E3
:10F1D000DEB76B017C0120E030E0A9010F947D5285
:10F1E00087FD1CC06DEB77E386E095E3A7019601F0
:10F1F0000F946F5969837A838B839C8360E2CE017D
:10F2000001960E9416FF0F900F900F900F90DF91C4
:10F21000CF91FF90EF90DF90CF9008956DEB77E363
:10F2200086E095EBE3CF0F94845220E030E04AE78C
:10F2300054E40F94695A20E030E0A9010F946F590B
:10F240000C94DF78CF92DF92EF92FF926B017C01FA
:10F2500020E030E0A9010F947D5287FD26C06DEBC0
:10F2600077E386E095E3A70196010F946F596B0150
:10F270007C0120E030E0A9010F947D5220E030E0D5
:10F2800040E05FE387FF04C020E030E040E05FEB58
:10F29000C701B6010F946F590F94DB5ACB01FF9051
:10F2A000EF90DF90CF900D94D8006DEB77E386E080
:10F2B00095EBD9CF0F94845220E030E0A9010F9450
:10F2C0006F590C9422790F94845220E030E0A90108
:10F2D0000F946F590F94DB5ACB010D94D8000F9403
:10F2E000845229EC38EC48EC5EE30F94695A20E034
:10F2F00030E040E05FE30F946F590F94E25A862F9D
:10F300000D942F010D944F350D944F356FEF809173
:10F3100026080D94E0326CEF71EB82E00D943644D8
:10F3200061E072EB81E00D94364466E072EB80E0C0
:10F330000D94364467EB7FEA83E00D943644CF9218
:10F34000DF92EF92FF92CF93DF9300D01F92CDB761
:10F35000DEB76B017C0120E030E0A9010F947D5203
:10F3600087FD1BC06DEB77E386E095E3A70196016F
:10F370000F946F5969837A838B839C83CE010196A6
:10F380000E94B2FF0F900F900F900F90DF91CF91DE
:10F39000FF90EF90DF90CF9008956DEB77E386E0DC
:10F3A00095EBE4CF0F94845220E030E040E251E44A
:10F3B0000F94695A20E030E0A9010F946F590C9422
:10F3C0009F798091171690911816891B8F7011F4F0
:10F3D0000C941E3481E0089580917D02882351F0C1
:10F3E000609195057091960530E020E041E081E064
:10F3F0000C947728089584E00D94AF3183E00D9448
:10F40000AF3182E00D94AF310F94845220E030E0B0
:10F41000A9010F946F590F94E25A862F0D940D0194
:10F4200090919C1081E089270C94BA3261E086E2C9
:10F4300098E00C94D5320F94442A0C9461F280E049
:10F4400090E0A0E8B0E48093A5109093A610A0935C
:10F45000A710B093A8108CED92E00E9446F1E091C5
:10F46000A00580E090E0A6EEB2E4E43009F44AC0E2
:10F4700080E090E0A0EBB1E480939D1090939E100B
:10F48000A0939F10B093A0108093A1109093A2100E
:10F49000A093A310B093A410EE0FFF0BE454FD4F04
:10F4A000808191818330910549F184309105D9F1B2
:10F4B000029761F480E090E0A0E5B3E480939D10B2
:10F4C00090939E10A0939F10B093A01084EC92E0B4
:10F4D0000E9446F11092A5101092A6101092A7104B
:10F4E0001092A8108CED92E00E9446F18091A00548
:10F4F0008F5F8530ECF48093A005089580E090E064
:10F50000A0E5B3E480939D1090939E10A0939F106C
:10F51000B093A0108093A1109093A210A093A31079
:10F52000B093A410D3CF80E090E0A0E5B3E4F2CF95
:10F530001092A0050895CF93DF9300D01F92CDB70E
:10F54000DEB70F94E25A0F94825269837A838B83D9
:10F550009C83CE0101960E9493FE0F900F900F9016
:10F560000F90DF91CF9108950F9484522AE037EDE8
:10F5700043E25DE30F94695A20E030E0A9010F9463
:10F580006F590C949B7ACF92DF92EF92FF92CF93B8
:10F59000DF9300D01F92CDB7DEB76B017C0120E076
:10F5A00030E0A9010F947D5287FD1BC06DEB77E31E
:10F5B00086E095E3A70196010F946F5969837A83DA
:10F5C0008B839C83CE0101960E9493FE0F900F9037
:10F5D0000F900F90DF91CF91FF90EF90DF90CF9041
:10F5E00008956DEB77E386E095EBE4CF0F948452BA
:10F5F0002AE037ED43E25DE30F94695A20E030E002
:10F60000A9010F946F590C94C37A0F94845220E08F
:10F6100030E0A9010F946F590C94C37ACF92DF9216
:10F62000EF92FF926B017C0120E030E0A9010F9482
:10F630007D5287FD26C06DEB77E386E095E3A70159
:10F6400096010F946F596B017C0120E030E0A90115
:10F650000F947D5220E030E040E05FE387FF04C07C
:10F6600020E030E040E05FEBC701B6010F946F5936
:10F670000F94DB5ACB01FF90EF90DF90CF900D9469
:10F680002E006DEB77E386E095EBD9CF0F94845293
:10F6900020E030E0A9010F946F590C940E7B0C947C
:10F6A000A2DC0C94A2DC0C94A2DC0C94A2DC0C94E2
:10F6B00054DC0C9454DC0C9454DC0C9454DCCF9249
:10F6C000DF92EF92FF92CF93C82F0F9443356B01D7
:10F6D0007C0124EA30E74DE75FE3609125027091F9
:10F6E000260280912702909128020F947D5287FD77
:10F6F00018C08AEF90E0A0E0B0E08C0D9D1DAE1D1B
:10F70000BF1D80933B0590933C05A0933D05B093AE
:10F710003E05C0931E02CF91FF90EF90DF90CF90F7
:10F72000089580E090E0DC01E8CFCF92DF92EF9285
:10F73000FF920F931F930F94433500910C05109186
:10F740000D0520910E0530910F056B017C01C01A4B
:10F75000D10AE20AF30A9701860137FD11C0209110
:10F760000B05209520930B056A547C4F8F4F9F4FBC
:10F7700060930C0570930D0580930E0590930F0513
:10F7800081E090910B05911101C080E01F910F91D4
:10F79000FF90EF90DF90CF9008950F9482421092E7
:10F7A0004F08109271020E944934882351F08091D1
:10F7B000C11682FD06C085E29EE19093C607809344
:10F7C000C50761E08EE19EE10E94C6350C9446FEBD
:10F7D0004F925F926F927F928F929F92BF92CF9241
:10F7E000DF92EF92FF920F931F93CF93DF9300D09E
:10F7F00000D01F921F92CDB7DEB77C016A0149018C
:10F80000FB0190818CE0989F800D1124982FF701C7
:10F810002081822F880F820F880F80938A16909301
:10F820008B164115510571F1FA82E9827C836B8355
:10F83000011121C0AE014B5F5F4FB401C6010E94B0
:10F8400081256C016D817E818F819885611571059F
:10F8500081059105B9F00E941427F70180818F5F1F
:10F860008083853138F3CE0101960E94C978E2CFBA
:10F87000B12C860129C08A01B12C26C04528462812
:10F880004728B1F728960FB6F894DEBF0FBECDBF5C
:10F89000DF91CF911F910F91FF90EF90DF90CF906C
:10F8A000BF909F908F907F906F905F904F90089542
:10F8B000B39407C0B1102EC001151105C9F20F5F36
:10F8C0001F4F01151105A9F2AE014B5F5F4FB40147
:10F8D000C6010E9481256C014D805E806F80788416
:10F8E0004114510461047104A9F0F0E24F1651046F
:10F8F00061047104F9F2D301C2018D97A109B10924
:10F900000297A105B10530F04BE2441651046104A1
:10F91000710471F6F7018081482F4B0D5527551F53
:10F920004631510534F0853020F0CE0101960E9419
:10F93000C97881E0411451046104710409F480E044
:10F94000B80EF70180818B0D8083BB2009F496CF20
:10F95000BA94AE014B5F5F4FB401C8010E9481258C
:10F960008C016D817E818F8198850E941427EDCF57
:10F97000EF92FF920F931F93CF93DF9300D000D0AD
:10F9800000D01F921F92CDB7DEB77C0120912408D2
:10F99000422F022E000C550B80912508833099F1DF
:10F9A000843051F18EEA91E25F932F939F938F936E
:10F9B0008E010F5F1F4F1F930F930F941452C701B7
:10F9C0000E9448DC4FE350E0B80187EC97E00F94C9
:10F9D000DD5C0F900F900F900F900F900F902B9673
:10F9E0000FB6F894DEBF0FBECDBFDF91CF911F9150
:10F9F0000F91FF90EF9008958AEB91E227FDD4CF0D
:10FA000085EA91E2D1CF83EC91E2CECFE09130084C
:10FA100085E1E802F0011124E153FA4E86819781D5
:10FA20000C94B87CE091300886E0E802F0011124E3
:10FA3000E75FF74F808191810C94B87C0F931F93FF
:10FA4000CF93DF938C01EB0190913B1620913C16F4
:10FA5000921305C00F9415020E9463F2F5CF8091B6
:10FA60003A1634E0839FF0011124E35CF94E1183D0
:10FA70000083D383C2839F5F90933B168F5F2817C9
:10FA800039F080933A16DF91CF911F910F9108952D
:10FA900010923A16F8CF63E972E084E690E00E9493
:10FAA0001E7D6AEB72E084E690E00C941E7D81116D
:10FAB0000C944B7D68EB71E084E190E00C941E7D2A
:10FAC0000E9498D80C94577D0F94DD120C94577DAA
:10FAD0000E9416FC0C944B7DCF93DF93CDB7DEB71D
:10FAE00020E2488559856F818E810F94EC2EDF913D
:10FAF000CF910895282F10922E0880911E08909182
:10FB00001F08A0912008B0912108B7FF08C01092EB
:10FB10001E0810921F081092200810922108809150
:10FB2000A805882331F080911E0880932208109246
:10FB30001D0880911C081816FCF4082E000C990B67
:10FB4000821B910920912208022E000C330B2817EA
:10FB5000390794F097FF02C090E080E0809322087C
:10FB6000092E000CAA0BBB0B80931E0890931F0854
:10FB7000A0932008B0932108809122086623A9F061
:10FB800090912308891714F4809323082091230867
:10FB9000022E000C330B2C5F3F4F482F082E000C19
:10FBA000550B241735071CF48450809323080895BF
:10FBB000AF92BF92CF92DF92EF92FF920F931F937B
:10FBC000CF93DF9361E081E00E947A7DC0912308AA
:10FBD00005E00C0FD1E08EEEE82E81E2F82E12E067
:10FBE0001C1B93EEC92E91E2D92EBD2EBC1AAC2E51
:10FBF000A194C11130C0DD23D9F0809122081816DC
:10FC0000BCF040911E0850911F086091200870912F
:10FC100021084F5F5F4F6F4F7F4F40931E085093F7
:10FC20001F0860932008709321088F5F809322083B
:10FC300080917D02882341F030E020E041E067EFD1
:10FC400071E28A2D0E947728CF5F0C13D2CF83E018
:10FC500080931C081FC0C13041F59091220891305B
:10FC600069F080917D028823C9F11F92DF92CF92C3
:10FC7000BF9281E0913051F180E028C080911B0853
:10FC800010921B08882369F3C0934E0880911D08C9
:10FC9000882339F3DF91CF911F910F91FF90EF905F
:10FCA000DF90CF90BF90AF900895C23069F69091E9
:10FCB00022089230A9F080917D02882379F01F926A
:10FCC000FF92EF921F9381E09230B1F68F930E94E2
:10FCD0006C7D0F900F900F900F900F90D0E0B4CFED
:10FCE00080911B0810921B08882329F3C0934E08AB
:10FCF00080911D088823F9F2CDCF2F923F924F9229
:10FD00005F926F927F928F929F92AF92BF92CF92AB
:10FD1000DF92EF92FF920F931F93CF93DF934C01EB
:10FD20000F94CA5101968401080F191FC8010F943E
:10FD3000CA5101966801C80ED91EF8016080C1E061
:10FD4000611001C0C0E0F6013080D1E0311001C087
:10FD5000D0E0AA24A3946110A12C60E085E00E9469
:10FD60007A7D50902308752C9EE0E92EF12C252CED
:10FD700021948A2D90E001965C01AC0EB11CAD0E71
:10FD8000B11C71101DC080917D028823A1F0E0910B
:10FD90002402E25067E072E2E33038F4F0E0EE0F64
:10FDA000FF1FEC51FD4F6081718130E020E043E0A6
:10FDB000822D0E947728D1E0611013C0D2E011C0DB
:10FDC000D2E06110D1E0D7110CC080917D02882370
:10FDD00041F030E020E041E0B4018D2F85190E9410
:10FDE0007728C1E0CD0F472C4518662079F0C71160
:10FDF0000BC080917D02882339F030E020E041E0A3
:10FE0000B801842D0E947728C2E0CD0F332071F015
:10FE1000C7110BC080917D02882339F030E020E0CB
:10FE200041E0B601842D0E947728CF5FF3E0AF1642
:10FE3000B1040CF4CF5FC71162C080917D028823AA
:10FE400009F45AC030E020E042E064E172E2842D1F
:10FE50000E947728D091090593EF9E0D9093080595
:10FE60008EEF8E0D80932F08209187162E151F047C
:10FE700011F00CF041C0209189169217E8F59EE32D
:10FE800090938A1680938B1665E470E080E090E092
:10FE90000E94142761E36D0F062E000C770B880B70
:10FEA000990B0E94142760E270E080E090E00E94CD
:10FEB00014278091D3159091D4150F94D8000E94E7
:10FEC000EF286FE270E080E090E00E9414270E942B
:10FED000957B811109C085E08D9FF0011124EE5BB7
:10FEE000F94F8481811108C08091D5159091D61564
:10FEF0000F94D8000E94EF2892E090937D02ECE0EE
:10FF0000EE0EF11C7394FAE4EF16F10409F039CF08
:10FF1000CF5FC0931C08DF91CF911F910F91FF908D
:10FF2000EF90DF90CF90BF90AF909F908F907F9099
:10FF30006F905F904F903F902F9008958FE192E2E5
:10FF40000C947D7E8CE292E20C947D7E8EE492E2B3
:10FF50000C947D7E89EE92E20C947D7E84EA92E29E
:10FF60000C947D7E81ED92E20C947D7E84E293E29E
:10FF70000C947D7E87E093E20C947D7E87E892E28C
:10FF80000C947D7E88E692E20C947D7E8F929F9207
:10FF9000AF92BF92EF92FF920F931F93CF93DF9395
:10FFA000EC018B01E42EF22E80914D1690914E16AD
:10FFB0008C179D0709F43EC02091010527FD109282
:10FFC000010522EBC23DD20709F03FC0805E9B4B8A
:10FFD00071F40F9443356E517B4F8F4F9F4F609359
:10FFE0009105709392058093930590939405D09317
:10FFF0004E16C0934D1630E020E000931E0810937B
:020000021000EC
:100000001F082093200830932108E0922308F092E3
:100010001C08C05EDB4B21F410920A05109290057B
:1000200082E080937D0281E080931D081092A505F7
:1000300010929F05DF91CF911F910F91FF90EF904C
:10004000BF90AF909F908F9008952BEBC03ED2074A
:1000500071F6825D924B19F0C0EEDBEBC8CF0F94C6
:1000600043358090910590909205A0909305B090B3
:100070009405681979098A099B0997FFEDCF80914A
:10008000C3078770873041F7C5E5D0E8B0CFCF937D
:10009000DF93EC010E94A27820E040E070E060E095
:1000A000CE01DF91CF910C94C67F20E040E070E05C
:1000B00060E080EC9EEA0E94C67F81E080930A05A2
:1000C00010924C0810924B08089520E040E070E038
:1000D00060E08AE999E70C94C67F80919F098111BD
:1000E00014C0809182029091830201972091D315D0
:1000F0003091D4152817390744F420E040E070E02F
:1001000060E085EC9AEB0C94C67F0C94658021E04E
:1001100020930A05FC0180819181A281B3818093A3
:10012000250290932602A0932702B093280220E094
:1001300040E070E060E08091190890911A080C94FA
:10014000C67FCF93DF9300D01F92CDB7DEB78DEC83
:100150009CECACECBCE389839A83AB83BC83CE017B
:1001600001960E9487800F900F900F900F90DF9163
:10017000CF910895CF93DF9300D01F92CDB7DEB714
:100180008DEC9CECACECBDE389839A83AB83BC83A0
:10019000CE0101960E9487800F900F900F900F90D4
:1001A000DF91CF910895CF93DF9300D01F92CDB709
:1001B000DEB780E090E0A0E8BFE389839A83AB8359
:1001C000BC83CE0101960E9487800F900F900F9004
:1001D0000F90DF91CF910895CF93DF9300D01F92BE
:1001E000CDB7DEB780E090E0A0E2B1E489839A83E6
:1001F000AB83BC83CE0101960E9487800F900F9045
:100200000F900F90DF91CF9108958FEF8093260884
:1002100020E040E070E060E08BE496E90C94C67F5B
:1002200081E080930A051092C3071092B10520E087
:1002300040E070E060E087E491E80E94C67F88E6D5
:1002400096E29093C6078093C507089581E0809356
:100250000A058091C3078770873051F01092C30759
:100260001092B10588E696E29093C6078093C50781
:1002700080919C108093A10580E00E94BA3220E01A
:1002800040E070E060E088E992E80C94C67F8091DD
:100290007D02882341F030E020E041E062E570E239
:1002A00082E00E9477288091B1058770873041F401
:1002B00020E040E070E060E08AE791E80C94C67FBF
:1002C000089520E040E070E060E081E991E80E945C
:1002D000C67F81E0809302058091A205811107C04D
:1002E00087E390E29093C6078093C50708958DE356
:1002F00090E2F8CF80917D02882341F030E020E049
:1003000041E063E470E281E00E94772880911B085D
:1003100010921B08882321F01092A2050C94618191
:1003200008950F931F93CF93DF9300D000D000D098
:100330001F92CDB7DEB780917D028823F1F01F9226
:1003400089E18F938091A20590E001969F938F930E
:100350008FE290E29F938F938E010F5F1F4F1F9349
:100360000F930F941452B80184E290E20E94F32894
:100370000FB6F894DEBF0FBECDBF84E080937D0240
:1003800080910205811108C020E040E070E060E04B
:1003900087ED91E80E94C67F2A960FB6F894DEBFDB
:1003A0000FBECDBFDF91CF911F910F910895CF92D6
:1003B000DF92EF92FF92CF93DF9300D01F92CDB7E1
:1003C000DEB780911B0810921B08882331F18091C1
:1003D000A2058F5F8093A2058931E0F081E08093D0
:1003E000020520E040E070E060E08BE092EB0E94CC
:1003F000C67F8EE190E29093C6078093C5070F9069
:100400000F900F900F90DF91CF91FF90EF90DF90C2
:10041000CF9008950E946181F2CF60911E08709183
:100420001F088091200890912108611571058105B0
:10043000910509F43EC00F9484522DEC3CEC4CEC39
:100440005CE30F94E3522091A5103091A6104091E7
:10045000A7105091A8100F946F596B017C0120E0F8
:1004600030E040E850EC0F947D5287FD53C020E00F
:1004700030E040E850E4C701B6010F94CF5B181696
:100480000CF44FC0C092A510D092A610E092A71015
:10049000F092A8108CED92E00E9446F182E08093E9
:1004A0007D0210921E0810921F08109220081092D0
:1004B000210880917D02882309F4A1CFC090A51066
:1004C000D090A610E090A710F090A81020E030E0A7
:1004D000A901C701B6010F947D5227E137EB41ED29
:1004E00058E387FF04C027E137EB41ED58EBC70124
:1004F000B6010F946F5969837A838B839C836BE277
:10050000CE0101960E9416FFBC0187E190E20E9495
:10051000F32875CFC12CD12C90E8E92E90ECF92E60
:10052000B1CFC12CD12C80E8E82E80E4F82EAACFE0
:1005300080917D02882341F030E020E041E062E5D7
:1005400070E282E00E9477288091B1058770873041
:1005500079F41092A00520E040E070E060E087E9C7
:100560009BEB0E94C67F81E080939F050C941F7ACD
:1005700008952F923F924F925F926F927F928F9247
:100580009F92AF92BF92CF92DF92EF92FF920F9322
:100590001F93CF93DF9300D000D0CDB7DEB71C01FF
:1005A0007A8369832B833C834D835E8327013801E3
:1005B00081E080931D080E94A27883E080937D02F1
:1005C00030928F0520928E0589819A8190938D05B6
:1005D00080938C058B819C81AD81BE818093880541
:1005E00090938905A0938A05B0938B05409284056A
:1005F000509285056092860570928705F12CE12C5A
:10060000C0921E08D0921F08E0922008F0922108A4
:10061000B0924E16A0924D1690928305809282055C
:100620008C8D8093810526960FB6F894DEBF0FBEA1
:10063000CDBFDF91CF911F910F91FF90EF90DF9091
:10064000CF90BF90AF909F908F907F906F905F9072
:100650004F903F902F9008952F923F924F925F922C
:100660006F927F928F929F92AF92BF92CF92DF92C2
:10067000EF92FF920F931F93CF93DF9300D000D0A0
:1006800000D0CDB7DEB71C017987688769011A836E
:100690000983EB82BA01550F880B990B0F94845292
:1006A00020E030E0A9010F946F594B015C0120E07C
:1006B00030E040E05FEC0F94CF5B18162CF0812CFB
:1006C000912CA12C2FECB22EC501B4010F94DB5A52
:1006D0002B013C01B601DD0C880B990B0F94845261
:1006E00020E030E0A9010F946F594B015C0120E03C
:1006F00030E040E05FE40F947D5287FD05C0812C1F
:10070000912CA12C9FE4B92EE885F9856081718137
:10071000072E000C880B990B0F94845220E030E0D8
:10072000A9010F946F596B017C01C301B2010F94B1
:1007300084529B01AC01C701B6010F946E590F940E
:10074000E25A6C837D838E839F83C501B4010F942D
:10075000DB5A7B018C01E418F50806091709FB81B7
:10076000FF9389809A808AEAA82E8EEAB82ECC80E0
:10077000DD80A301920168857985C1010E94B9825B
:100780000F9029960FB6F894DEBF0FBECDBFDF9154
:10079000CF911F910F91FF90EF90DF90CF90BF907E
:1007A000AF909F908F907F906F905F904F903F9011
:1007B0002F90089520E040E070E060E080EE9BEB39
:1007C0000C94C67F0E9480340E9421D50C94DA8359
:1007D00088E598E00E9481CA0E94DA830D948242E3
:1007E0000E94DA8384EB94E29093C6078093C50756
:1007F00008950E94DB310F94874181E08093B71602
:100800000F94C9410C94DA836F927F928F929F92DA
:10081000AF92BF92CF92DF92EF92FF920F931F930E
:10082000CF93DF9381E080930A0561E00E947A7D97
:10083000C091230885E0882E8C0ED1E009EF13E8E3
:100840009AEBE92E94E2F92E82E0982E9C1A20EF82
:10085000C22E23E8D22E35ECA32E34E2B32E7D2E09
:100860007C1A6C2E6194C11130C0DD23D9F08091C7
:1008700022081816BCF040911E0850911F08609184
:100880002008709121084F5F5F4F6F4F7F4F40935B
:100890001E0850931F0860932008709321088F5FF3
:1008A0008093220880917D02882341F030E020E08F
:1008B00041E062ED74E2862D0E947728CF5F8C12B2
:1008C000D2CF83E080931C0823C0C13081F5809192
:1008D0002208813089F080917D02882309F444C088
:1008E000DF92CF92BF92AF927F9281E090912208E7
:1008F000913089F180E02FC080911B0810921B0875
:10090000882349F30E94F08380911D08882319F3FE
:10091000DF91CF911F910F91FF90EF90DF90CF90DB
:10092000BF90AF909F908F907F906F900895C2304E
:1009300029F6809122088230C9F080917D028823B7
:1009400099F01F930F93FF92EF929F9281E0909105
:100950002208923079F68F930E946C7D0F900F9051
:100960000F900F900F900F90D0E0A8CF80911B08B0
:1009700010921B08882309F30E94F98380911D08B7
:100980008823D9F2C5CF61116093240240930905F1
:100990008C3008F03AC0E82F880FFF0B8827EC5204
:1009A000FB478F4F0D9466590785E084EB840A85D9
:1009B000EE84F184F4840085F7840585FA84FD844F
:1009C00082EA9FE721E020930A0520E040E070E002
:1009D00060E00C94C67F8AEA9FE7F4CF8EEA9FE737
:1009E000F1CF82EB9FE7EECF86EB9FE7EBCF8AEB71
:1009F0009FE7E8CF8EEB9FE7E5CF82EC9FE7E2CF62
:100A000010924E0888ED9DE7DDCF0C94DA838EE9D5
:100A10009FE7D8CF86EA9FE7D5CFCF930E9416FCF9
:100A20000E9498D8C82F882319F080E00F94B60B45
:100A30008C2F0E94577DCF910C94DA830F931F93D4
:100A4000CF93DF93CDB7DEB76E970FB6F894DEBFC6
:100A50000FBECDBF282F082E000C330B90911F0224
:100A6000409120028F3F39F0F901EE0FFF1FEF5D3B
:100A7000FD4F908141814F939F933F938F9389E5E1
:100A80009EE19F938F938E010F5F1F4F1F930F93D4
:100A90000F9414524FE350E0B80187EC97E00F94A5
:100AA000DD5C0E94DA830FB6F894DEBF0FBECDBFC7
:100AB0006E960FB6F894DEBF0FBECDBFDF91CF911B
:100AC0001F910F9108958FEF0C941E85809130082F
:100AD0000C941E85E0919005EE2389F0E150E0939F
:100AE000900588E0E89FF0011124EF5AFA4F6281E7
:100AF000738127814681808191810C94C67F0C94FB
:100B0000DA832F923F924F925F926F927F928F92F1
:100B10009F92AF92BF92CF92DF92EF92FF920F938C
:100B20001F93CF93DF9300D01F92CDB7DEB761E064
:100B300081E00E947A7D209123082B832C83822FD1
:100B40008B5F898389E0821B8A8388E0782E721A02
:100B500087E0682E621A86E0582E521A85E0482EE9
:100B6000421A84E0382E321A222E21942B81211130
:100B70005BC080912208882399F180917D028823AF
:100B800059F081E090912208911180E024E045E045
:100B900057E2622D0F94EC2E80918D0980932608E8
:100BA0008B81853009F0A2C0109230088091220814
:100BB000853009F45FC180917D02882309F43AC22F
:100BC00011E080912208853009F010E0809126081C
:100BD0000F942F0100E09C0142EE56E2642D83C089
:100BE00080911B0810921B08882339F20E946A85A5
:100BF00080911D08882309F4C0CF0F900F900F90AB
:100C00000F90DF91CF911F910F91FF90EF90DF90A8
:100C1000CF90BF90AF909F908F907F906F905F909C
:100C20004F903F902F9008958B818130C1F5809136
:100C300022088130E1F080917D02882309F4ACCF55
:100C400011E080912208813009F010E08091730258
:100C5000909174020F94D80061E02C81621B00E037
:100C60009C014FEF56E2812F0E94722995CF80910F
:100C70001B0810921B088823F1F2E12C10E000E021
:100C800027EE33E04AE050E063E772E08FEF96E250
:100C90000E942C8380911D08882369F2AECF8B813E
:100CA000823009F08AC180912208823009F44EC056
:100CB00080917D028823D1F011E08091220882305A
:100CC00009F010E06091330670913406809135068A
:100CD000909136060E94DF7862E02C81621B00E072
:100CE0009C0149EF56E2812F0E94722980918E0962
:100CF000809326089B81963009F0E6C081E08093BE
:100D0000300880912208863009F4C9C080917D02A4
:100D1000882391F011E080912208863009F010E0DC
:100D2000809126080F942F0100E09C0142EE56E2CC
:100D3000652D812F0E9472299B819F5F9B83298152
:100D4000291314CF8AE080931C0857CF80911B0889
:100D500010921B08882309F4ABCF20E030E04AE76B
:100D600054E4609133067091340680913506909179
:100D700036060F94E35220E030E0A9010F946F593A
:100D800020E030E04AE754E40F946F590F94E25AA0
:100D90001F92912C812C8EE6A82E8EEAB82E6B0124
:100DA00010EDE12E17E0F12E00E010E028E13CEF1D
:100DB0004FEF5FEF63E376E089EF96E20E94B9823E
:100DC0000F9080911D08882309F472CF16CF80916F
:100DD00022088330C9F080917D02882309F486CFF0
:100DE00011E080912208833009F010E08091D51540
:100DF0009091D6150F94D80063E02C81621B00E01F
:100E00009C0142EF56E22FCF80911B0810921B08E5
:100E1000882309F30F94612FE12C04E819E723EBF1
:100E200031E050E040E065ED75E182EF96E20E942E
:100E30002C8380911D08882371F2DFCE80911B08DE
:100E400010921B08882309F4C4C00F94612FE12C71
:100E500001E416EC2CE830E050E040E061E778E097
:100E60008EEE96E20E942C8380911D08882309F45F
:100E7000B0C0C3CE80911B0810921B08882309F4D0
:100E80009ACE0F94612F65E175E782EE96E20F949A
:100E90006B3180911D08882309F48DCEAECE8091F0
:100EA0001B0810921B08882309F430CF0F94612F80
:100EB00065E175E782EE96E20F946B3180911D0833
:100EC000882309F423CF99CE2B81273099F580917F
:100ED00022088730B9F080917D02882309F42CCF55
:100EE00011E080912208873009F010E080913502EE
:100EF000909136020F94D80000E09C014DED56E22F
:100F0000662D17CF80911B0810921B08882319F3B8
:100F1000E12C02EF14E727EE33E04AE050E065E30E
:100F200072E08DED96E20E942C8380911D0888234B
:100F300091F263CE8B81883009F062C080912208E3
:100F40008830D9F080917D02882309F4F5CE11E034
:100F500080912208883009F010E060918509709135
:100F6000860980918709909188090E94A77300E003
:100F70009C0143ED56E2672DDCCE80911B08109258
:100F80001B088823F9F265E879E083ED96E20F9477
:100F9000253180911D088823A9F22FCE80911B084E
:100FA00010921B088823A1F185E590E80E944780F4
:100FB00080911D08882361F120CE8B81833009F454
:100FC00006CF843009F0E8CD80912208843009F4FE
:100FD00035CF80917D02882309F488CE11E080917D
:100FE0002208843009F010E0809171089091720815
:100FF0000F94D80000E09C014EEE56E2632D33CEF4
:101000009B81993009F098CE80912208893031F285
:1010100080917D02882309F48FCE81E0909122088F
:10102000993009F080E023E048EC56E26A810F94A1
:10103000EC2E82CE80918E09809326087DCE5F9221
:101040006F927F928F929F92AF92BF92CF92DF92D8
:10105000EF92FF920F931F93CF93DF93D1E0809194
:10106000D5159091D615892B09F4D0E061E081E087
:101070000E947A7DC09123088C2E45E0942E9C0E10
:10108000AA24A39484E0F82EFC1A83E0D82EDC1A5C
:1010900082E0C82ECC1A7A2C7C1A6C2E619487E0E0
:1010A000B82EBC1AC111B9C080912208882309F456
:1010B00096C080917D02882359F081E090912208AA
:1010C000911180E024E043EC56E2662D0F94EC2E63
:1010D00080918E0980932608C430E9F4A0923008EC
:1010E00080912208843009F448C180917D028823D0
:1010F00091F011E080912208843009F010E0809195
:1011000026080F942F0100E09C014CEA56E26F2D57
:10111000812F0E94722910E000E035E0E32E5C2E62
:10112000581800932608CE111FC0F801EE0FFF1FBC
:10113000E154F04C8591949190933208809331085A
:10114000809122088C1709F42DC180917D0288239B
:1011500059F081E0909122089E1180E023E042EA5C
:1011600056E2652D0F94EC2E8E2D0F5F1F4F96E0EB
:10117000E92E8630B1F68091710890917208892B22
:1011800019F4DD2309F42EC1C73009F58091220836
:10119000873009F418C180917D028823C1F082EE66
:1011A00093E89F938F9389E996E29F938F93BF92E1
:1011B00081E090912208973009F080E08F930E949F
:1011C0006C7D0F900F900F900F900F900F9088E014
:1011D000D1E0CF5FC91166CF80931C080EC080910B
:1011E0001B0810921B08882309F463CF0E946A85AC
:1011F00080911D08882309F45CCFDF91CF911F9166
:101200000F91FF90EF90DF90CF90BF90AF909F90A5
:101210008F907F906F905F900895C13009F060C00B
:1012200080912208813009F43FC080917D0288239B
:1012300009F44ECF11E080912208813009F010E0CE
:101240008091D5159091D6150F94D80000E09C019F
:101250004CEB56E2672D812F0E94722980918D09F7
:1012600080932608C33009F033CF10923008809164
:101270002208833009F46CC080917D02882309F430
:101280004ACF11E080912208833009F010E080916C
:1012900026080F942F0100E09C014CEA56E26D2DC8
:1012A000812F0E94722914CF80911B0810921B0875
:1012B000882309F4BACF0F94612FE12C02E819E7D3
:1012C00023EB31E050E040E065ED75E18CEB96E218
:1012D0000E942C8380911D08882309F4A6CF8DCF0E
:1012E000C23009F0BBCF809122088230B9F08091E2
:1012F0007D02882309F4ECCE11E08091220882302F
:1013000009F010E080917108909172080F94D80054
:1013100000E09C0148EB56E26C2D9DCF80911B08AC
:1013200010921B08882319F30F94612FE12C01E41C
:1013300016EC2CE830E050E040E061E778E088EB24
:1013400096E20E942C8380911D08882381F255CF5C
:1013500080911B0810921B08882309F48DCF0F94ED
:10136000612F65E175E78CEA96E20F946B3180910D
:101370001D08882309F480CF40CF80911B0810926C
:101380001B08882309F4B1CE0F94612F65E175E73E
:101390008CEA96E20F946B3180911D08882309F442
:1013A000A4CE2BCF80911B0810921B08882309F430
:1013B000CCCE84EF99E80E94478080911D08882355
:1013C00009F4C3CE1ACF80911B0810921B08882302
:1013D00009F4E1CE0E94E28380911D08882309F47C
:1013E000DACE0BCF87E0F5CE4F925F926F927F926D
:1013F0008F929F92AF92BF92CF92DF92EF92FF9225
:101400000F931F93CF93DF930091260861E081E053
:101410000E947A7DC091230810E0000F111F015433
:10142000104C95E0592E5C0E2FE7E22E26E2F22EAC
:10143000D3E0DC1B36E8C32E39E7D32E41E7A42ED8
:1014400046E2B42E82E0782E7C1A52EA852E56E2CD
:10145000952E81E0682E6C1A4C2E4194C11137C034
:10146000809122088823B1F080917D02882359F071
:1014700081E090912208911180E024E04DE856E24D
:10148000642D0F94EC2ECF5F5C12E8CF84E0809344
:101490001C080CC080911B0810921B08882321F3A4
:1014A0000E946A8580911D088823F1F2DF91CF9117
:1014B0001F910F91FF90EF90DF90CF90BF90AF9072
:1014C0009F908F907F906F905F904F900895C13064
:1014D00059F5F801859194919093320880933108E1
:1014E00080912208813081F080917D02882359F219
:1014F0001F929F928F926F9281E09091220891307B
:1015000009F474C080E072C080911B0810921B081F
:10151000882351F380912608682F0F94E032809140
:101520001D08882309F3C2CFC23009F042C0F80178
:10153000859194919093320880933108809122088C
:101540008230D1F080917D02882309F49CCFDF9214
:10155000CF92BF92AF927F9281E090912208923019
:1015600009F080E08F930E946C7D0F900F900F9098
:101570000F900F900F9087CF80911B0810921B083F
:10158000882301F30E94867980911D088823D1F277
:101590008DCF80911B0810921B088823C1F06091A9
:1015A00026088FEF0F94E03280911D08882379F090
:1015B0007DCFC33009F067CFF80185919491909366
:1015C00032088093310880912208833011F3809192
:1015D0007D02882309F457CF1F92FF92EF92DF9389
:1015E00081E090912208933009F08CCF8F930E9474
:1015F0006C7D0F900F900F900F900F9044CF9F92A3
:10160000AF92BF92CF92DF92EF92FF920F931F9310
:10161000CF93DF9361E081E00E947A7DC09123083F
:10162000CC2E85E0982E9C0E99E2A92E96E2B92E3A
:10163000D7E0DC1B16E01C1B05E00C1B84E0F82E39
:10164000FC1A82E0E82EEC1A81E0D82EDC1AC111D7
:1016500033C0809122088823B9F080917D028823CD
:1016600061F06C2D619581E090912208911180E0EC
:1016700024E04CE656E20F94EC2ECF5FC911E7CF81
:1016800088E080931C080CC080911B0810921B08F6
:10169000882319F30E946A8580911D088823E9F246
:1016A000DF91CF911F910F91FF90EF90DF90CF903E
:1016B000BF90AF909F900895C13011F5809122089E
:1016C000813079F080917D028823B9F281E0909198
:1016D0002208913009F080E023E047E95FE36D2DB7
:1016E000CACF80911B0810921B08882359F382E609
:1016F0009CE80E94478080911D08882319F3D0CF71
:10170000C23009F0BFC090912208923071F08091F0
:101710007D02882309F4B1CF81E0923009F080E0A6
:1017200020E24EE556E26E2DA6CF80911B08109266
:101730001B08882361F328E636E23093C60720931E
:10174000C50780911D08882311F3AACF9091220824
:10175000933079F080917D02882309F48ECF63E085
:101760006C1981E0933009F080E020E242E556E216
:1017700082CF80911B0810921B08882359F329E51A
:1017800036E23093C6072093C50780911D08882351
:1017900009F386CF90912208943071F080917D02F8
:1017A000882309F46ACF81E0943009F080E020E2D8
:1017B00046E456E26F2D5FCF80911B0810921B0804
:1017C000882361F32DE436E23093C6072093C507E2
:1017D00080911D08882311F363CF909122089530E2
:1017E00071F080917D02882309F447CF81E0953024
:1017F00009F080E020E24AE356E2602F3CCF80917E
:101800001B0810921B08882361F321E436E2309311
:10181000C6072093C50780911D08882311F340CF88
:1018200080912208863081F080917D02882309F41E
:1018300024CF81E090912208963009F080E023E0E7
:101840004DE256E2612F17CF80911B0810921B08C2
:10185000882351F38EE79DE80E94478080911D0800
:10186000882311F31DCF80911B0810921B08882339
:10187000D9F0B092C607A092C50780911D088823B1
:1018800099F00ECFC33009F461CFC43009F482CF90
:10189000C53009F4A2CFC63019F2C73009F0EDCE39
:1018A000909122089730F9F280917D02882309F403
:1018B000E4CE81E0973009F080E020E248E156E292
:1018C0006D2FD9CEAF92BF92CF92DF92EF92FF925F
:1018D0000F931F93CF93DF9361E081E00E947A7DA5
:1018E000C091230885E0C82ECC0ED5E0DC1B93E028
:1018F000D92E14E01C1BBD2CBC1A82E0F82EFC1A59
:1019000081E0E82EEC1AAC2EA194C1112BC080917D
:101910002208882381F080917D02882369F181E08B
:1019200090912208911180E024E041E156E26A2D75
:101930000F94EC2E21C080911B0810921B08882365
:1019400051F30E946A8580911D08882321F3DF915D
:10195000CF911F910F91FF90EF90DF90CF90BF90AC
:10196000AF900895C130A1F590912208913059F0BF
:1019700080917D02811119C0CF5FCC11C6CF86E066
:1019800080931C08E4CF80911B0810921B088823C9
:1019900079F3809137028C2780933702D0927D02B1
:1019A00080911D08882321F3D2CF81E0913009F086
:1019B00080E09091370220E036E2911102C02CEFD6
:1019C00035E201E043E056E26E2D0E947229D4CF49
:1019D000C23009F077C080912208823079F080917E
:1019E0007D02882349F281E090912208923009F02B
:1019F00080E023E048EB5FE36F2D9ACF80911B08D6
:101A000010921B08882359F385E999E70E944780C3
:101A100080911D08882319F39ACF80912208833082
:101A200081F080917D02882309F4A6CF81E0909116
:101A30002208933009F080E023E041EB5FE36B2D57
:101A400077CF80911B0810921B08882351F380E9FF
:101A500099E70E94478080911D08882311F377CF72
:101A600080912208843081F080917D02882309F4DE
:101A700083CF81E090912208943009F080E023E048
:101A80004AEA5FE3612F54CF80911B0810921B0834
:101A9000882351F38BE899E70E94478080911D08C5
:101AA000882311F354CF80911B0810921B088823C0
:101AB000A9F08DE690E80E94478080911D08882358
:101AC00069F045CFC33009F4A8CFC43049F2C5301E
:101AD00009F052CF80912208853029F380917D0250
:101AE000882309F449CF81E090912208953009F0CC
:101AF00080E023E041EA5FE36D2F1ACF2F923F92FF
:101B00004F925F926F927F928F929F92AF92BF920D
:101B1000CF92DF92EF92FF920F931F93CF93DF93B9
:101B200000D01F921F92CDB7DEB78091C307877098
:101B300089830E94B533682E61E081E00E947A7D3E
:101B4000209123082C83722E2B5F2A8383E0871930
:101B50008B835524539482E0282E2718452C471850
:101B6000372C31948C81811141C0809122088823C7
:101B7000C9F080917D02882359F081E0909122087C
:101B8000911180E024E04AED50E2632D0F94EC2E99
:101B9000662009F452C08981873009F462C193E05C
:101BA0009D834DC080911B0810921B08882309F368
:101BB0000E946A8580911D088823D9F20F900F90AA
:101BC0000F900F900F90DF91CF911F910F91FF9089
:101BD000EF90DF90CF90BF90AF909F908F907F90CD
:101BE0006F905F904F903F902F9008959C8191301F
:101BF00011F580912208813079F080917D0288234F
:101C000039F281E090912208913009F080E023E0E0
